:100000000C949D080C94BC080C94BC080C94070B31
:100010000C943D0B0C94BC080C94BC080C94BC08CC
:100020000C94BC080C94BC080C94BC080C94BC0840
:100030000C94BC080C94BC080C94BC080C94970E4F
:100040000C94BC080C94BC080C94BC080C94BC0820
:100050000C94B6590C94C2500C94BC080C94BC0877
:100060000C94BC080C9498510C94BC080C948C51C2
:100070000C94BC080C94BC080C94BC080C94BC08F0
:100080000C9479650C94BC080C94BC080C94BC08C6
:100090000C94D6510C94BC080C94CA510C94BC0816
:1000A0000C94BC080C94BC080C94BC080C94BC08C0
:1000B0000C94BC080C94BC080C94BC080C94BC08B0
:1000C0000C94BC080C94BC080C94BC080C94BC08A0
:1000D0000C94BC080C94BC080C94BC080C94BC0890
:1000E0000C94BC080C946F590C9479590C94655974
:1000F0000C941F590C94AA590C949B590C948F5929
:100100000C9483590C94BC080C94BC080C94BC0847
:100110000C94BC080C94BC080C94BC080C94BC084F
:10012000084AD73B3BCE016E84BCBFFDC12F3D6C5E
:1001300074319ABD56833DDA3D00C77F11BED9E4C4
:10014000BB4C3E916BAAAABE000000803F076342F1
:1001500036B79BD8A71A39685618AEBAAB558C1D5E
:100160003CB7CC5763BD6DEDFD753EF6177231BFE0
:10017000000000803F08000000BE922449123EAB00
:10018000AAAA2ABECDCCCC4C3E00000080BEABAAB1
:10019000AAAA3E00000000BF000000803F0000004F
:1001A0000000084178D3BB4387D1133D190E3CC3EF
:1001B000BD4282AD2B3E68EC8276BED98FE1A93E6E
:1001C0004C80EFFFBE01C4FF7F3F000000000050E5
:1001D0003A20256C642050612020252D372E326670
:1001E000206D0A002563002563004932433A200050
:1001F000256300256C642050612020252D372E3288
:1002000066206D00256C6420432000256300545F48
:1002100052483D252D342E3166200052483D252D73
:10022000342E31662000256300256300507772313B
:100230003D25730A0044656275673D3078252D7849
:100240000A00496E7075742050313D25730A0048CC
:10025000554D5F5057525F414C574159533D25739F
:100260000A0025730A006175746F0A004C6F6720DD
:100270006D6F64653D00496E74722E205365633A5C
:1002800020202050303D252D372E33662050313D23
:10029000252D372E33660A00496E74722E20546F56
:1002A00074616C3A2050303D252D6C642050313DF6
:1002B000252D6C640A005553425F5057523D2573FB
:1002C0000A00565F4D43553D252D352E32660A00F6
:1002D000565F494E3D252D352E32660A0052657017
:1002E0006F7274204D61736B3D3078252D6C7820D2
:1002F000005265706F727420496E74657276616C1D
:100300003D252D640A0052494D4520616464723DCB
:10031000252D642E252D640A004E65696768626F7D
:1003200072207461626C652073697A653D25640A88
:1003300000545820506F7765723D25640A00436869
:10034000616E3D25640A004932433A200049443D2C
:100350000053797374656D2053756D6D6172790A00
:100360000025630025630043757272656E74207208
:1003700065706F727420696E74657276616C3D256C
:100380002D64207365630A004E6577207265706F77
:10039000727420696E74657276616C3D252D6420DF
:1003A0007365630A002563005573696E6720726583
:1003B000706F72743D3078252D6C7820004E657713
:1003C000207265706F72743D3078252D6C78200036
:1003D000256300256300256300256300204F5343F8
:1003E00043414C3D2564200020467573653A2065E5
:1003F000653D253032782068663D25303278206CA6
:10040000663D25303278206C623D25303278004DD3
:1004100043553D2530366C7800256300252D31305D
:100420006C7520252D31306C7520252D31306C7583
:1004300020252D31306C75200A007478206C656E93
:1004400020202020207268206D69737320202020D6
:100450007268207374616C652020207268206D6959
:1004600073630A002563004F4B0A00256300256370
:1004700000256300256300445F434F4D50415353B3
:100480003D307825780A00445F414343454C3D3078
:100490007825780A00445F505245533D30782578DE
:1004A0000A00445F5057525F313D307825780A008A
:1004B000445F4145533D307825780A00445F503110
:1004C0005F4C45443D307825780A00445F50305FEA
:1004D0004C45443D307825780A00445F4556454EEA
:1004E000543D307825780A00445F504F5745523DBF
:1004F000307825780A00445F4C45443D30782578B3
:100500000A00445F4F573D307825780A00445F5019
:100510004B543D6E307825780A00445F54583D3086
:100520007825780A00445F52583D307825780A00D3
:10053000445F4F5045523D307825780A004375722C
:1005400072656E742064656275673D307825580A5F
:10055000004E65772064656275673D307825580ADE
:100560000025730A0025372E33662025372E336683
:100570000025352E326620004572726F72203020C1
:10058000566F6C74004E6F7420737570706F727458
:1005900065640A004572726F72203020566F6C7469
:1005A000004572726F72203020566F6C7400257394
:1005B0000A00545820506F7765723D25640A004345
:1005C00068616E3D25640A005465737420362025E9
:1005D000730A005465737420352025730A0054652E
:1005E000737420342025730A0054657374203320FB
:1005F00025730A005465737420322025730A005451
:1006000065737420312025730A0025730A00257351
:100610000A0025730A0025730A00646565700A00E4
:10062000666F7263655F69646C650A006E6F6E6504
:100630000A00707772733D005854414C5F54524920
:100640004D3D25640025730A00525F50413D090964
:100650003078256C7800525F503D09093078256C60
:100660007800525F41333D09093078257800525FA8
:1006700041323D09093078257800525F41313D090A
:10068000093078257800525F565F494E3D090930A0
:1006900078257800525F52483D0909307825780066
:1006A000525F555054494D453D09307825780052E8
:1006B0005F50315F543D09093078257800525F5012
:1006C000313D09093078257800525F50305F543D44
:1006D00009093078257800525F50303D090930789B
:1006E000257800525F565F4D43553D093078257897
:1006F00000525F545F4D43553D09307825780052D4
:100700005F54313D09093078257800525F543D0926
:10071000093078257800525F4536343D0909307834
:10072000257800525F49443D090930782578005208
:100730005F50412000525F502000525F4133200043
:10074000525F41322000525F41312000525F565FBC
:10075000494E2000525F52482000525F5550544984
:100760004D452000525F50315F542000525F5031A0
:100770002000525F50305F542000525F5030200004
:10078000525F565F4D43552000525F545F4D4355B5
:100790002000525F54312000525F542000525F45C8
:1007A00036342000525F494420002530327800253D
:1007B000372E33662025372E33662025352E3066BA
:1007C0000025352E32662000204E657665722D7527
:1007D00073656420737461636B203E20256420621E
:1007E000797465730A00557074696D6520256420FD
:1007F000646179732C20253032643A253032643AB2
:10080000253032640A0074657374205B6F66667C01
:10081000317C327C337C347C355D202020202020CC
:1008200020202D2074657374206D6F6465730A0D2C
:1008300000776474205B6F6E7C6F66667C74657392
:10084000745D20202020202020202020202D2077B3
:1008500061746368646F670A0D00757067722020A9
:100860002020202020202020202020202020202088
:100870002020202020202D207265626F6F7420764A
:10088000696120626F6F746C6F616465720A0D003C
:10089000626F6F7420202020202020202020202024
:1008A0002020202020202020202020202D207265A4
:1008B000626F6F740A0D0070777273205B646565F8
:1008C000707C666F7263655F69646C657C6E6F6E69
:1008D000655D202D206D637520736C656570206DDE
:1008E0006F64650A0D007265737420656570726FC0
:1008F0006D202020202020202020202020202020AB
:1009000020202D20726573746F726520656570728A
:100910006F6D0A0D007031205B6F6E7C6F66665DD7
:1009200020202020202020202020202020202020C7
:10093000202D2064697361626C652070756C73652D
:1009400020703120746F207361766520706F776539
:10095000720A0D0070777231205B6F6E7C6F666675
:100960005D2020202020202020202020202020204A
:100970002D2070696E31207077720A0D00747870C6
:1009800077205B31352D305D202020202020202055
:100990002020202020202020202D20545820507757
:1009A000722E20486967686573742030202833648C
:1009B000426D290A0D007373202020202020202062
:1009C0002020202020202020202020202020202027
:1009D00020202D2073797374656D2073756D6D61A2
:1009E00072790A0D00727320202020202020202000
:1009F00020202020202020202020202020202020F7
:100A0000202D20726164696F2073746174730A0D04
:100A1000007269205B696E745D20202020202020F8
:100A2000202020202020202020202020202D207267
:100A300065706F727420696E74657276616C0A0DF0
:100A4000007265205B6D61736B5D2020202020208B
:100A5000202020202020202020202020202D206D3C
:100A60006F7465207265706F727420736574746939
:100A70006E670A0D006F7720202020202020202084
:100A80002020202020202020202020202020202066
:100A9000202D206F6E652D776972652073656E73EA
:100AA0006F72730A0D006C6F67205B6175746F7CE9
:100AB0006F6E7C6F66665D20202020202020202025
:100AC00020202D206D6F7465732064617461206F28
:100AD0006E205553420A0D006E65205B666C75737F
:100AE000685D202020202020202020202020202081
:100AF000202020202D206E65696768626F72207447
:100B000061626C650A0D0065727220202020202031
:100B100020202020202020202020202020202020D5
:100B20002020202D206572726F7220696E666F0A18
:100B30000D006D6375202020202020202020202003
:100B400020202020202020202020202020202D2098
:100B50006D637520696E666F0A0D006964205B72B3
:100B6000657365745D202020202020202020202017
:100B7000202020202020202D2069642068616E64C0
:100B80006C696E670A0D0068756D70205B6F6E7C16
:100B90006F66665D2020202020202020202020203D
:100BA0002020202D2068756D696469747920706536
:100BB000726D2073656E736F72207077720A0D000C
:100BC00068756D202020202020202020202020203B
:100BD0002020202020202020202020202D2068756B
:100BE0006D69646974792073656E736F720A0D00A4
:100BF0006465205B6D61736B5D20202020202020C8
:100C00002020202020202020202020202D2064654E
:100C10006275670A0D006368616E205B31312D32A9
:100C2000365D202020202020202020202020202071
:100C300020202D204368616E2031312D323620284E
:100C4000322E3430352D32343830204D687A290A2E
:100C50000D0063616C69205B5B765F696E7C61315E
:100C60007C61325D20766F6C747C72657365747C18
:100C70006E6F6E655D202D2063616C6962726174B8
:100C8000650A0D00616463202020202020202020A0
:100C90002020202020202020202020202020202054
:100CA0002D2073686F7720765F696E2C2061312C60
:100CB00020613220766F6C74616765730A0D006184
:100CC0006573205B6F6E7C6F66665D202020202040
:100CD00020202020202020202020202D20696E741C
:100CE0006567726574790A0D007520202020202028
:100CF00020202020202020202020202020202020F4
:100D000020202020202D20757074696D650A0D004B
:100D1000762020202020202020202020202020207D
:100D20002020202020202020202020202D2076651B
:100D30007273696F6E0A0D00682020202020202029
:100D400020202020202020202020202020202020A3
:100D5000202020202D2068656C700A0D002563007E
:100D6000756E6B6E6F776E20636D640A004E48443B
:100D7000433032313620004C334734323030442057
:100D800000484D433538383320004144584C333403
:100D9000352000424D503038352000484948363122
:100DA00033302000415432344D414320002025731C
:100DB000002025362E32662000253032780020258E
:100DC00073002025362E3266204F6E2D426F6172E1
:100DD000640025303278000A00452025642E256401
:100DE00020636C6F636B20256C7520637075202504
:100DF0006C75206C706D20256C75206972712025D2
:100E00006C7520676C656420256C7520796C656451
:100E100020256C7520726C656420256C75207478B3
:100E200020256C75206C697374656E20256C7520A7
:100E300073656E736F727320256C752073657269AC
:100E4000616C20256C750A00532025642E256420D2
:100E5000636C6F636B20256C7520747820256C752E
:100E600020727820256C752072747820256C75208E
:100E700072727820256C75207265786D69742025F2
:100E80006C752061636B747820256C75206E6F61C2
:100E9000636B747820256C752061636B72782025F4
:100EA0006C752074696D65646F757420256C752090
:100EB00062616461636B727820256C7520746F6F5A
:100EC0006C6F6E6720256C7520746F6F73686F721E
:100ED0007420256C752062616473796E63682025C7
:100EE0006C752062616463726320256C7520636F8A
:100EF0006E74656E74696F6E64726F7020256C75A8
:100F00002073656E64696E6764726F7020256C75FE
:100F1000206C6C747820256C75206C6C72782025A0
:100F20006C750A00257325730A004F6E6C696E6537
:100F30000A000A002C20636865636B207261746587
:100F400020257520487A0025732025732C2063689E
:100F5000616E6E656C20257520706F776572202537
:100F600075000A0025783A004D414320616464729F
:100F7000657373200052616E646F6D20455549366C
:100F80003420616464726573732067656E65726195
:100F90007465640A000A2A2A2A2A2A2A2A426F6FBA
:100FA00074696E672025732A2A2A2A2A2A2A0A00A7
:100FB000020000FFFE00000141544D45474131321F
:100FC0003872666131006C6F63616C686F737400B6
:100FD000454550524F4D20697320636F7272757092
:100FE000742C20726577726974696E6720776974F2
:100FF000682064656661756C74732E0A006E616E9C
:1010000000696E660000407A10F35A00A0724E1814
:10101000090010A5D4E80000E87648170000E40BAA
:1010200054020000CA9A3B000000E1F50500008070
:10103000969800000040420F000000A086010000CA
:1010400000102700000000E803000000006400001A
:101050000000000A00000000000100000000002C59
:1010600076D888DC674F0823DFC1DFAE59E1B1B71E
:1010700096E5E3E453C63AE651997696E8E6C284EB
:1010800026EB898C9B62ED407C6FFCEFBC9C9F4003
:10109000F2BAA56FA5F490055A2AF75C936B6CF928
:1010A000676DC11BFCE0E40D47FEF520E6B500D0FE
:1010B000ED902E0300943577050080841E08000013
:1010C000204E0A000000C80C333333330F986E12E1
:1010D000831141EF8D2114893BE65516CFFEE6DBE7
:1010E00018D1844B381BF77C1D901DA4BBE4242031
:1010F0003284725E228100C9F124ECA1E53D2749CA
:101100004E46494E4954594E414ECDCCCC3D0AD75E
:10111000233C17B7D13877CC2B329595E6241FB1F5
:101120004F0A000020410000C84200401C4620BC7D
:10113000BE4CCA1B0E5AAEC59D7411241FBECFEF04
:10114000D1E4DEBFCDBF16E0A0E0B2E0E8E2F2E01D
:1011500001E00BBF02C007900D92AC3DB107D9F77B
:101160001DE2ACEDB6E001C01D92A63AB107E1F771
:101170000E947C4F0C9412810C94000029E0FC0129
:1011800020935700C895802D089500D082E396E003
:10119000EDB7FEB7928381830E94FC7D8091C504E8
:1011A0009091C6040F900F9093FF04C000D08CE282
:1011B00096E009C092FF04C000D080E296E003C030
:1011C00000D08AE196E0EDB7FEB7928381830E945A
:1011D000FC7D0F900F900895E091CB17F0E0EF7138
:1011E000F070E05EF74E80838091CB178F5F809325
:1011F000CB178091E02488608093E0244CEE54E08B
:10120000CA0161E10E94C44080E090E008954F92DD
:101210005F926F927F928F929F92AF92BF92CF9286
:10122000DF92EF92FF920F931F93DF93CF93CDB78F
:10123000DEB760970FB6F894DEBF0FBECDBF3B019F
:101240000E94A155E82FF0E0EE0FFF1FEB56F84E7D
:10125000808191810196918380838091DC069091B9
:10126000DD0681FD74980E948C474C0181E097E077
:101270000E94BB410AC0C8010296B3010E94913E80
:10128000009701F5C8010E948142082F192F01150E
:10129000110589F721C1C8010296B3010E94883E59
:1012A000D4018C918150F801808780E091E0A0E02A
:1012B000B0E081879287A387B48781E097E0B80187
:1012C0000E944242C8010D9660E074E64EE85AE082
:1012D00098010E94804484E00E94C048D80115967D
:1012E0009C938E93149783E00E94C0482C01F801D0
:1012F00097838683D401AC908085A81ABB24CC2424
:10130000DD2486E0AA0CBB1CCC1CDD1C8A95D1F721
:10131000618572858385948520EC30E040E050E063
:101320000E94337A672F782F892F9927A60EB71E30
:10133000C81ED91EF801A186B286C386D486D40100
:101340008C9180878091DC069091DD0681FD08C03C
:101350008091C50480FD04C081FFB6C01D9BB4C050
:10136000EDB7FEB772970FB6F894FEBF0FBEEDBF94
:10137000EDB6FEB60894E11CF11C80E092E0928389
:101380008183C4010196D70113969C938E93129783
:10139000F301808114968C93149715961C921597DF
:1013A000818116968C93169717961C92D4018C9176
:1013B000F70180871186D80114968D919C9115971D
:1013C0009387828755864486BB27AD2D9C2D8B2D18
:1013D00097878687C601B50124E630E040E050E0FB
:1013E0000E94337A672F782F892F99270E94797A64
:1013F000F701718B608B0E94EA7D2091A8048DB764
:101400009EB742960FB6F8949EBF0FBE8DBF2223A3
:10141000A9F000D000D0EDB7FEB7319687EE91E08D
:10142000ADB7BEB712969C938E9311972283138209
:101430000E94FC7D0F900F900F900F908091691C7F
:1014400086FF42C00E94724DC40104960E94314D35
:10145000EDB7FEB73C970FB6F894FEBF0FBEEDBFD9
:1014600031967E010894E11CF11CADB7BEB712960F
:10147000FC92EE92119780E190E0938382838CE35B
:1014800092E095838483D80114968D919C91159751
:101490009783868316968D919C9117979187808765
:1014A000D4018C91828713860E945A7EEDB7FEB7D5
:1014B0003C960FB6F894FEBF0FBEEDBF82E00E94CF
:1014C0004E4DC7010E94314D8091DC069091DD06A2
:1014D00081FF0DC0749A0BC085E595E00E944F41D5
:1014E000082F192F0115110509F0D5CEEDCF609603
:1014F0000FB6F894DEBF0FBECDBFCF91DF911F9125
:101500000F91FF90EF90DF90CF90BF90AF909F90A2
:101510008F907F906F905F904F900895EF92FF9221
:10152000CF93DF93E82EE7017E01F92EE70180914A
:10153000DC069091DD0687FF2FC08DB79EB70C9714
:101540000FB6F8949EBF0FBE8DBFEDB7FEB73196B4
:101550008FE492E0ADB7BEB712969C938E9311972D
:101560008A81828313828B81848315828885868316
:1015700017828C819D81918780878E819F8193873F
:1015800082870E94EA7D2DB73EB7245F3F4F0FB69A
:10159000F8943EBF0FBE2DBF81E097E0BE010E94D0
:1015A000094285E595E0BE010E947541DF91CF912A
:1015B000FF90EF90089587EE93E08115910511F06B
:1015C0000197F1F708958823E9F052985A981DBAC7
:1015D00080916900806280936900EA9A8091C504D5
:1015E0009091C60494FF12C053985B98EB9A809137
:1015F00069008068809369008091680081608093B1
:1016000068000895109269005A9AEA9808951F9206
:101610000F920FB60F9211248F939F93AF93BF93A6
:101620008091680080FF20C08091C0249091C124E7
:10163000A091C224B091C3240196A11DB11D809335
:10164000C0249093C124A093C224B093C32480915A
:10165000DC069091DD0690FF07C0749882E090E070
:1016600090939B0480939A04BF91AF919F918F9127
:101670000F900FBE0F901F9018951F920F920FB6EC
:101680000F9211248F939F93AF93BF938091680023
:1016900080FF20C08091C4249091C524A091C624CD
:1016A000B091C7240196A11DB11D8093C4249093CD
:1016B000C524A093C624B093C7248091DC069091E2
:1016C000DD0691FF07C0739882E090E090939B0441
:1016D00080939A04BF91AF919F918F910F900FBE0D
:1016E0000F901F90189580937C0080917B00877FDE
:1016F00080937B0080917C00806C80937C0085E0EF
:1017000080937A0080917A00806880937A0080913B
:101710007B0087FFFCCF80917B0085FFFCCF809111
:101720007A00806480937A0080917A0086FDFCCFF5
:10173000109279001092780084E090E060E070E010
:1017400020917A00206420937A0020917A0026FD6F
:10175000FCCF2091780030917900620F731F0197C0
:1017600079F710927C0080917A008F7780937A00CD
:10177000769567957695679580E090E00E94B677BC
:10178000089580E00E94730B20919C0430919D0489
:1017900040919E0450919F040E94947821EE3AE774
:1017A00044E95EE30E948476089580E180935101CC
:1017B000809351019091510195FF03C08F5F8F314C
:1017C000B9F76BE4869FB0011124882777FD8095D7
:1017D000982F0E94B87720E030E64FE954E40E9449
:1017E000847620E030E04AE754E40E944E77089582
:1017F0008091BF0484FF4BC080917B008860809300
:101800007B0089EC80937C0085E080937A00809156
:101810007A00806880937A0080917B0087FFFCCFFC
:1018200080917B0085FFFCCF80917A00806480935B
:101830007A0080917A0086FDFCCF80917A008064E6
:1018400080937A0080917A0086FDFCCF60917800C9
:101850007091790080E090E00E94B67727ED33EA3E
:1018600040E95FE30E94947826E636E648E853E4D0
:101870000E9483766093A0177093A1178093A2179C
:101880009093A31780917A008F7780937A000895C0
:101890006F927F928F929F92AF92BF92CF92DF9280
:1018A000EF92FF920F931F93DF93CF93CDB7DEB7E5
:1018B0002A970FB6F894DEBF0FBECDBF3C01109241
:1018C000E4068FEF89836CEDC62E67E1D62E00E02B
:1018D00010E052E0E52EF12CEC0EFD1E4E010894B6
:1018E000811C911C4AE0A42EB12CAC0EBD1E3FC041
:1018F0000830110509F441C0C401B7012A870E94CC
:101900007E4A89812A858F3F11F08E3F19F480939A
:10191000E40634C06114710479F4C7010E94984A46
:101920008093DD24F701A5EDB4E281918D93EA1552
:10193000FB05D9F721E022C0C7010E94984AF601B1
:101940008083D701F80133E0EE0FFF1F3A95E1F7EE
:10195000E00FF11FEC52F84E8D918193AA15BB0553
:10196000D9F70F5F1F4F89E090E0C80ED91E202FD6
:101970008981882309F0BCCF01C028E0822F2A96F4
:101980000FB6F894DEBF0FBECDBFCF91DF911F9190
:101990000F91FF90EF90DF90CF90BF90AF909F900E
:1019A0008F907F906F90089500D087ED9DE0EDB708
:1019B000FEB7928381830E94FC7D0F900F90089563
:1019C0002F923F924F925F926F927F928F929F924F
:1019D000AF92BF92CF92DF92EF92FF920F931F933D
:1019E000DF93CF9300D000D0CDB7DEB78C01009746
:1019F00041F489E290E06BE270E04AE250E027E0D7
:101A00000AC08130910549F489E290E06BE270E010
:101A10004AE250E026E00E945A49C8010E94480C60
:101A2000F801EE51F94F808301151105A1F01CED6D
:101A3000C12E17E1D12E00E010E04F01B9EB6B2E63
:101A4000BDE07B2EA1EB4A2EADE05A2EFDEA2F2EF3
:101A5000FDE03F2EFAC085ED94E20E94CA4B9C0146
:101A6000B901882777FD8095982F0E94B877C82EF6
:101A7000E92EE5EDAE2EE4E2BE2E02ED1DE0D5012D
:101A80008D915D0100D000D0EDB7FEB73196ADB7B6
:101A9000BEB712961C930E931197828313826B83A9
:101AA0007C830E94FC7D0F900F900F900F906B81B4
:101AB0007C81BDEDAB16B4E2BB0609F700D000D0C7
:101AC00000D00DB71EB70F5F1F4F22EC3DE0EDB702
:101AD000FEB7328321838C2D9E2D20E030E048EC30
:101AE00052E40E944E77D80112966D937D938D93A8
:101AF0009C9315970E94FC7DEDB7FEB736960FB606
:101B0000F894FEBF0FBEEDBF8091DD24882319F04D
:101B10008EE792E002C087E892E000D000D02EEB82
:101B20003DE0ADB7BEB712963C932E931197149635
:101B30009C938E9313970E94FC7D0F900F900F90B3
:101B40000F900E94D40C88C0780173E0EE0CFF1C4B
:101B50007A95E1F7E00EF11EE4EDF7E1EE0EFF1EDF
:101B6000C7010E94CA4B9C01B901882777FD809567
:101B7000982F0E94B8775C0120E030E0D7018D916A
:101B80007D0100D000D0EDB7FEB73196ADB7BEB73E
:101B900012967C926E9211978283138229833A83E4
:101BA0006B837C830E94FC7D29813A812F5F3F4FAC
:101BB0000F900F900F900F906B817C812830310532
:101BC000E9F600D000D000D0EDB6FEB60894E11CD6
:101BD000F11CEDB7FEB7528241828A2D9B2D20E089
:101BE00030E048EC52E40E944E77D70112966D9394
:101BF0007D938D939C9315970E94FC7DEDB7FEB766
:101C000036960FB6F894FEBF0FBEEDBFD6018C918D
:101C1000882319F08EE792E002C087E892E000D0B6
:101C200000D0EDB7FEB732822182948383830E9475
:101C3000FC7D0F900F900F900F900E94D40C0F5FBF
:101C40001F4F29E030E0C20ED31ED4018C9190E0EA
:101C5000081719070CF478CF0F900F900F900F9082
:101C6000CF91DF911F910F91FF90EF90DF90CF9078
:101C7000BF90AF909F908F907F906F905F904F90AC
:101C80003F902F900895DF93CF9300D0CDB7DEB76C
:101C90008091D62489838091DC248A83CE010196A9
:101CA0000E94A33E0F900F90CF91DF910895CF93A4
:101CB000DF93EC018091D5248F3FB1F58091D6243C
:101CC0008F3F91F58091D7248F3F71F58091D82473
:101CD0008F3F51F58091D9248F3F31F58091DA24DF
:101CE0008F3F11F58091DB248F3FF1F48091DC244C
:101CF0008F3FD1F489E290E06BE270E04AE250E07D
:101D000027E00E945A4980E090E00E94480CCE51A2
:101D1000D94F888385ED94E268E170E049E050E0B6
:101D20000E944C7F0E94430EDF91CF9108951F9235
:101D30000F920FB60F920BB60F9211241F932F9391
:101D40003F934F935F936F937F938F939F93AF9343
:101D5000BF93EF93FF938091E02482608093E0240F
:101D60008091C50486FD2B9A8091C50487FD2B9A2E
:101D700080919A0490919B041816190614F4749A91
:101D8000739A8091DC069091DD0685FF02C07498FD
:101D9000739880915D0590915E05019790935E0523
:101DA00080935D05009709F07EC0809110079091A7
:101DB00011070196909311078093100720916B20D3
:101DC00030916C2040916D2050916E202F5F3F4FDD
:101DD0004F4F5F4F20936B2030936C2040936D20CA
:101DE00050936E2020E130E030935E0520935D0536
:101DF0002091C50420FD02C01D9B05C01092E00685
:101E00001092DF0606C021E030E03093E006209318
:101E1000DF066091C3047091C4046115710599F0E7
:101E200001960E94527A009771F477988091DC06AF
:101E30009091DD0693FF07C0749884E090E0909342
:101E40009B0480939A046091C3047091C40461154B
:101E5000710579F080911007909111070E94527AD4
:101E6000009739F488E095E062E140E050E00E949C
:101E7000C4408091C50486FD2B988091C504909143
:101E8000C60491FF10C00E94A1558A3119F0182F85
:101E90001F5F01C01BE00E94E553812F90E00E946C
:101EA000B9550E94835487E795E060E040E050E038
:101EB0000E94C440FF91EF91BF91AF919F918F918C
:101EC0007F916F915F914F913F912F911F910F9053
:101ED0000BBE0F900FBE0F901F9018958091CB17DF
:101EE00090917F20891B08950E946E0F882379F0BE
:101EF000E0917F20F0E0EF71F070E05EF74E20811E
:101F000030E080917F208F5F80937F2002C02FEF91
:101F10003FEFC9010895CF93DF93EC0110920407BE
:101F20001092030788819981009731F022E0863D65
:101F3000920709F0B9C009C00E946E0F882341F4CE
:101F400086ED92E099838883B3C0613109F0B0C017
:101F5000F89478940E94740F90E09093080780930F
:101F600007078D3009F47CC08F3F31F38231910532
:101F700069F18F37910521F08830910509F053C040
:101F800080910B0790910C07181619060CF060C091
:101F90006091A02D7091A12D88E090E00E94BE7DFF
:101FA0006091A02D7091A12D80E290E00E94BE7DF5
:101FB0006091A02D7091A12D88E090E00E94BE7DDF
:101FC00080910B0790910C0701973EC06091A02D66
:101FD0007091A12D8DE090E00E94BE7D10920A07C5
:101FE0001092090714C080589F4DFC0180816091B8
:101FF000A02D7091A12D90E00E94BE7D80910907D7
:1020000090910A07019690930A078093090780919F
:10201000090790910A0720910B0730910C0782174E
:1020200093070CF315C06091A02D7091A12D0E9413
:10203000BE7D80910B0790910C0720910707FC0152
:10204000E058FF4D2083019690930C0780930B0777
:1020500080910B0790910C078F33910509F06CCF9D
:1020600010927F2080917F208093CB1780910B0767
:1020700090910C07FC01E058FF4D108290930407EB
:102080008093030710920C0710920B078091DE24B7
:102090009091DF24009709F44FCF6091050740E04D
:1020A00050E00E94C44048CF1982188283E001C0EA
:1020B00081E0DF91CF91089578948091DF0690912F
:1020C000E0060097C9F08091C5049091C60493FD85
:1020D00013C092FF03C083B7817F03C083B7817FA2
:1020E000866083BFF89483B7816083BF78948895B6
:1020F00083B78E7F83BF78940895CF93DF93EC01ED
:1021000088819981009721F02AE0843C920799F414
:102110000E94D3520E945C108091960E9091970E6F
:1021200065E840E050E00E94C44084EC9AE0998366
:10213000888381E003C01982188283E0DF91CF9108
:102140000895CF93DF930E94D35280EB0E944A4CB4
:102150008823B1F40E94B04C8091691C90916A1C54
:10216000816090936A1C8093691C00D084EA9DE092
:10217000EDB7FEB7928381830E94FC7D0F900F9094
:102180008EB1C82FD0E0C470D070729A0E94D35222
:102190008EE40E944A4C8823B1F40E94B04C809196
:1021A000691C90916A1C826090936A1C8093691CE0
:1021B00000D08BE99DE0EDB7FEB7928381830E944A
:1021C000FC7D0F900F90209709F472980E94D352D3
:1021D0008EEE0E944A4C8823B1F40E94B04C80914C
:1021E000691C90916A1C846090936A1C8093691C9E
:1021F00000D083E99DE0EDB7FEB7928381830E9412
:10220000FC7D0F900F9086EA0E944A4C8823B1F41F
:102210000E94B04C8091691C90916A1C88609093D8
:102220006A1C8093691C00D08AE89DE0EDB7FEB778
:10223000928381830E94FC7D0F900F900E94D35265
:102240008CE30E944A4C8823B1F40E94B04C8091E8
:10225000691C90916A1C806190936A1C8093691C30
:1022600000D081E89DE0EDB7FEB7928381830E94A4
:10227000FC7D0F900F900E94D35282ED0E944A4C39
:102280008823B1F40E94B04C8091691C90916A1C23
:10229000806290936A1C8093691C00D087E79DE060
:1022A000EDB7FEB7928381830E94FC7D0F900F9063
:1022B000C7E0D0E00E94D3528CE70E944A4C8823AA
:1022C000B9F40E94B04C8091691C90916A1C8064A2
:1022D00090936A1C8093691C00D08DE69DE0EDB759
:1022E000FEB7928381830E94FC7D0F900F9002C005
:1022F000219701F70E94B04C0E94D40CDF91CF913E
:102300000895DF93CF9300D0CDB7DEB74A836983BA
:102310000E94864C6981862F0E94B84C4A81842F86
:102320000E94B84C0E94B04C0F900F90CF91DF915B
:102330000895AF92BF92DF92EF92FF920F931F9397
:10234000DF93CF9300D00F92CDB7DEB7082FD22EF8
:102350004A835B8369830E94864C6981862F0E9431
:10236000B84C802F81600E94AD4C4A815B81042F64
:10237000152FAA24BB24ED2CFF240894E108F108B2
:102380000FC0AE14BF0419F40E94D34C02C00E94C7
:10239000C94CF80180830894A11CB11C0F5F1F4F2A
:1023A000AD1478F30E94B04C0F900F900F90CF9126
:1023B000DF911F910F91FF90EF90DF90BF90AF9052
:1023C0000895AF92BF92CF92DF92EF92FF920F9358
:1023D0001F93DF93CF93CDB7DEB760970FB6F89416
:1023E000DEBF0FBECDBFB82EA42E662309F455C0A4
:1023F000AE014F5F5F4F80E1DA011D928A95E9F7E8
:1024000080EB68E928E00E949911BB2059F000D0C8
:1024100088E892E0EDB7FEB7928381830E94EA7D5F
:102420000F900F908E010F5F1F4F38E0E32EF12CBD
:10243000EC0EFD1E2FE8C22E22E0D22ED8018D9187
:102440008D0100D000D0EDB7FEB73196ADB7BEB765
:102450001296DC92CE921197828313820E94EA7DBB
:102460000F900F900F900F900E151F0539F700D0A9
:1024700000D0EDB7FEB7319684E992E0ADB7BEB7B4
:1024800012969C938E9311978885828313820E9463
:10249000EA7D0F900F900F900F90AA2009F457C07B
:1024A000AE014F5F5F4F80E1FA0111928A95E9F723
:1024B00080EB60E828E00E949911BB2069F000D011
:1024C0008AE992E0ADB7BEB712969C938E931197AE
:1024D0000E94EA7D0F900F908E010F5F1F4F90E1D9
:1024E000E92EF12CEC0EFD1E8FE8C82E82E0D82ECE
:1024F000F80181918F0100D000D0EDB7FEB7319681
:10250000ADB7BEB71296DC92CE921197828313823A
:102510000E94EA7D0F900F900F900F900E151F05EF
:1025200039F700D000D0EDB7FEB7319684E992E0DC
:10253000ADB7BEB712969C938E9311978885828310
:1025400013820E94EA7D0F900F900F900F9060967B
:102550000FB6F894DEBF0FBECDBFCF91DF911F91B4
:102560000F91FF90EF90DF90CF90BF90AF900895C4
:102570000F931F93DF93CF9300D0CDB7DEB71A82AE
:1025800019828EEE6AEA8E010F5F1F4FA80122E0CA
:102590000E949911398120E08A8190E0822B932B4F
:1025A00090934118809340188EEE6CEAA80122E0C7
:1025B0000E949911398120E08A8190E0822B932B2F
:1025C00090934318809342188EEE6EEAA80122E0A1
:1025D0000E949911398120E08A8190E0822B932B0F
:1025E00090934518809344188EEE60EBA80122E08A
:1025F0000E949911398120E08A8190E0822B932BEF
:1026000090935318809352188EEE62EBA80122E04B
:102610000E949911398120E08A8190E0822B932BCE
:1026200090935518809354188EEE64EBA80122E025
:102630000E949911398120E08A8190E0822B932BAE
:1026400090935718809356188EEE66EBA80122E0FF
:102650000E949911398120E08A8190E0822B932B8E
:1026600090934718809346188EEE68EBA80122E0FD
:102670000E949911398120E08A8190E0822B932B6E
:1026800090934918809348188EEE6AEBA80122E0D7
:102690000E949911398120E08A8190E0822B932B4E
:1026A00090934D1880934C188EEE6CEBA80122E0AD
:1026B0000E949911398120E08A8190E0822B932B2E
:1026C00090934F1880934E188EEE6EEBA80122E087
:1026D0000E949911398120E08A8190E0822B932B0E
:1026E00090935118809350180F900F90CF91DF91D5
:1026F0001F910F9108952F923F924F925F926F9288
:102700007F928F929F92AF92BF92CF92DF92EF9281
:10271000FF920F931F93DF93CF93CDB7DEB76C97E4
:102720000FB6F894DEBF0FBECDBFA82E4A8B2B8FFD
:10273000FE01319683E0DF011D928A95E9F78091D1
:102740006418882339F46C8F0E94B81281E080935A
:1027500064186C8D662309F475C08EEE64EF4EE24A
:102760000E94811169E07AE180E090E00E94374C9C
:102770008EEE66EFAE014F5F5F4F22E00E9499112F
:10278000698170E080E090E0982F872F762F662790
:102790002A8130E040E050E0622B732B842B952B94
:1027A000209156183091571840E050E0621B730B8F
:1027B000840B950B209154183091551840E050E04F
:1027C0000E94337A7B018C013FE015950795F794C1
:1027D000E7943A95D1F760914E1870914F18882779
:1027E00077FD8095982F2BE0660F771F881F991F24
:1027F0002A95D1F72091501830915118442737FD70
:102800004095542F2E0D3F1D401F511F0E949B7A53
:102810002E0D3F1D30934B1820934A18285F3F4FD1
:1028200014E0359527951A95E1F779010027F7FC13
:102830000095102FE0925818F092591800935A18EA
:1028400010935B18BA2DB295BB0FBB0FB07CBC5C6C
:10285000B9872A2D30E03E8B2D8B63E070E00A2C87
:1028600002C0660F771F0A94E2F7882777FD8095EC
:10287000982F25E335E040E050E00E94337ADC01F8
:10288000CB010296A11DB11D8A879B87AC87BD87AE
:1028900020E533EC40E050E004C05595479537956E
:1028A0002795AA94D2F72E873F87488B598B188695
:1028B0001C821D821E821F8248E050E08D899E8905
:1028C000481B590B5C8B4B8B69C18EEE64EF4985BD
:1028D0000E9481116A857B858C859D850E94374C7D
:1028E0008EEE66EFAE014F5F5F4F23E00E949911BD
:1028F00080914A1890914B18805A9F401C014424A3
:1029000037FC4094542CC201B101A20191010E94F4
:10291000337A6F8B788F898F9A8F209144183091FA
:102920004518442737FD4095542FC201B1010E943C
:10293000337A7B018C01BDE015950795F794E794F8
:10294000BA95D1F722E030E040E050E0E20EF31E0D
:10295000041F151F6F89788D898D9A8DACE0959530
:10296000879577956795AA95D1F72091461830916C
:102970004718442737FD4095542F0E94337ABC01F5
:10298000992777FD9095892FE60EF71E081F191FCE
:10299000E2E015950795F794E794EA95D1F780E082
:1029A00090E8A0E0B0E0E80EF91E0A1F1B1F20917E
:1029B00052183091531840E050E0C801B7010E940E
:1029C000337A3B014C017FE0969487947794679427
:1029D0007A95D1F7A980BB24CC24DD246501BB24E2
:1029E000AA248A8190E0A0E0B0E0BA2FA92F982F06
:1029F0008827A82AB92ACA2ADB2A8B8190E0A0E07E
:102A0000B0E0A82AB92ACA2ADB2A0B8804C0D594C8
:102A1000C794B794A7940A94D2F7209142183091A2
:102A20004318442737FD4095542FC201B1010E943D
:102A3000337A7B018C014BE015950795F794E79469
:102A40004A95D1F78091401890914118AA2797FD97
:102A5000A095BA2F32E0880F991FAA1FBB1F3A9585
:102A6000D1F7E80EF91E0A1F1B1F2091481830915C
:102A70004918442737FD4095542F6F89788D898DEB
:102A80009A8D0E94337A27E195958795779567957A
:102A90002A95D1F7E60EF71E081F191F0D8804C0EE
:102AA000EE0CFF1C001F111F0A94D2F722E030E049
:102AB00040E050E0E20EF31E041F151F82E0159562
:102AC0000795F794E7948A95D1F7AE18BF08C00A26
:102AD000D10AC601B5012E853F85488959890E94D2
:102AE000337A97FD0BC0660F771F881F991FA401CB
:102AF00093010E94797A79018A010AC0A4019301A5
:102B00000E94797A79018A01EE0CFF1C001F111FC7
:102B1000552717FD5A95412F302F2F2DCA01B90186
:102B20000E94337A2EED3BE040E050E00E94337A81
:102B30005B016C01C801B70123E433EE4FEF5FEF97
:102B40000E94337ABC01992777FD9095892F6153B4
:102B5000714F8F4F9F4F5601DD24B7FCD094CD2C81
:102B60006A0D7B1D8C1D9D1D44E09595879577957D
:102B700067954A95D1F76E0D7F1D801F911F2C819F
:102B80003D814E815F81260F371F481F591F2C83BF
:102B90003D834E835F8338853F5F388748855A89F8
:102BA000451708F492CE552391F0252F30E040E0F0
:102BB00050E06C817D818E819F810E94797A209383
:102BC0005C1830935D1840935E1850935F188B8D9E
:102BD0008823C9F160915C1870915D1880915E182E
:102BE00090915F18611571058105910561F10E9451
:102BF000B87720E836EE45EC57E40E944E7721E0A6
:102C00003EED42E45EE30E94F778562F472F382FBF
:102C1000292F60E070E080E89FE3DA01F9012B2FB3
:102C20003A2F4F2F5E2F0E9483762BE43AE34DEB31
:102C300057E30E944E7760936018709361188093F9
:102C40006218909363186C960FB6F894DEBF0FBEAF
:102C5000CDBFCF91DF911F910F91FF90EF90DF904B
:102C6000CF90BF90AF909F908F907F906F905F902C
:102C70004F903F902F900895DF93CF9300D000D0D6
:102C800000D0CDB7DEB7FE01319686E0DF011D92A0
:102C90008A95E9F78091AA17882399F486EA61E377
:102CA00040E00E94811186EA6CE24AE00E948111B4
:102CB00081E08093AA176CE77EE380E090E00E94B9
:102CC000374C86EA6DE248E00E9481116CE77EE3B2
:102CD00080E090E00E94374C86EA62E3AE014F5FED
:102CE0005F4F26E00E94991186EA6DE247E00E945C
:102CF00081119A8180E0498150E0482B592B5093F3
:102D0000A5174093A4179C8180E02B8130E0282BED
:102D1000392B3093A7172093A6177E8160E08D8111
:102D200090E0862B972B9093A9178093A8176DB7E7
:102D30007EB7685070400FB6F8947EBF0FBE6DBF6F
:102D4000EDB7FEB731966EE972E0ADB7BEB7129639
:102D50007C936E93119753834283358324839783A7
:102D600086830E94EA7D6DB77EB7685F7F4F0FB69E
:102D7000F8947EBF0FBE6DBF26960FB6F894DEBFE7
:102D80000FBECDBFCF91DF910895CF92DF92EF922A
:102D9000FF920F931F93DF93CF9300D000D000D00A
:102DA000CDB7DEB78E010F5F1F4F86E0F80111929D
:102DB0008A95E9F78CE362E041E00E9481118CE39F
:102DC00060E048E50E94811162E174E380E090E0F8
:102DD0000E94374C8CE363E0A80126E00E94991121
:102DE0008CE362E043E00E948111998180E00A81D6
:102DF00010E0082B192B10938B1700938A179B81D7
:102E000080E06C8170E0682B792B70938D17609354
:102E10008C173D8120E08E8190E0822B932B909344
:102E20008F1780938E17882777FD8095982F0E94A3
:102E3000B8776B017C01B801882777FD8095982FC2
:102E40000E94B8779B01AC01C701B6010E94F776DA
:102E50002DB73EB72C5030400FB6F8943EBF0FBE92
:102E60002DBF0DB71EB70F5F1F4F2CEA32E0EDB735
:102E7000FEB73283218320918A1730918B17F80196
:102E80003383228320918C1730918D1735832483CF
:102E900020918E1730918F173783268320EE3EE2E4
:102EA00045E652E40E94947820E030E044E353E4A5
:102EB0000E948476F80160877187828793870E94D9
:102EC000EA7D2DB73EB7245F3F4F0FB6F8943EBF63
:102ED0000FBE2DBF26960FB6F894DEBF0FBECDBF36
:102EE000CF91DF911F910F91FF90EF90DF90CF90E6
:102EF0000895CF93DF93EC0188819981009731F099
:102F00002AE08D3A920709F071C00BC085EE96E079
:102F100060E870E00E947A438DEA9AE099838883A2
:102F200069C085EE96E00E94A543009709F462C04F
:102F30008091DC069091DD0694FF3FC08091691C72
:102F400082FF3BC083E061E048E021E00E947B1308
:102F50008DB79EB70A970FB6F8949EBF0FBE8DBF70
:102F6000EDB7FEB731968FEC91E0ADB7BEB71296D4
:102F70009C938E93119780915C1890915D18A0910D
:102F80005E18B0915F1882839383A483B583809188
:102F9000601890916118A0916218B09163188683AF
:102FA0009783A087B1870E94FC7D8DB79EB70A9654
:102FB0000FB6F8949EBF0FBE8DBF8091DC06909136
:102FC000DD0695FF06C08091691C83FF02C00E9448
:102FD0003C168091DC069091DD0696FF97CF80919C
:102FE000691C84FF93CF0E94C51690CF1982188266
:102FF00083E001C081E0DF91CF910895CF92DF920D
:10300000FF920F931F93CF93DF93729A8091C50421
:1030100083FD06C0C0E5D0E00E94DB0A2197E1F7FE
:103020008EE40E944A4C8823B1F080916F209091E9
:103030007020A0917120B09172200196A11DB11D48
:1030400080936F2090937020A0937120B093722092
:1030500021E030E084C0C0E5D0E00E94DB0A219787
:10306000E1F78FE40E944A4C0E94C94CF82E8295E9
:103070008695869583708130A9F4209173203091D4
:10308000742040917520509176202F5F3F4F4F4F15
:103090005F4F20937320309374204093752050939A
:1030A000762016C08230A0F02091772030917820D1
:1030B0004091792050917A202F5F3F4F4F4F5F4FC3
:1030C00020937720309378204093792050937A2072
:1030D0000E94C94C1F2D1F7300E0080F111D0E9494
:1030E000C94C0E94D34C20E0E901C80FD11DD695F0
:1030F000C795D695C7950E94B04C8091C50483FFB3
:103100007298B80180E090E00E94B67720E134E048
:1031100048EC5BE30E94947860936518709366189E
:103120008093671890936818BE0180E090E00E9439
:10313000B67724EA3CEF44E25CE30E94947820E016
:1031400030E040E252E40E9483766093E124709381
:10315000E2248093E3249093E42420E030E0C9014A
:10316000DF91CF911F910F91FF90DF90CF90089545
:103170007298729A8EE40E944A4C80EA0E94B84C7F
:1031800080E00E94B84C80E00E94B84C8FE40E941E
:103190004A4C0E94C94C82958695869583708130F1
:1031A000A9F42091732030917420409175205091A2
:1031B00076202F5F3F4F4F4F5F4F20937320309308
:1031C0007420409375205093762016C08230A0F072
:1031D00020917720309178204091792050917A2069
:1031E0002F5F3F4F4F4F5F4F2093772030937820D2
:1031F0004093792050937A2000D000D0EDB7FEB7ED
:10320000319621EC32E0ADB7BEB712963C932E93C7
:103210001197828313820E94EA7D0F900F900F9086
:103220000F908EE40E944A4C80E80E94B84C80E0E7
:103230000E94B84C80E00E94B84C0E94B04C80E0E4
:1032400090E0089500D080E69DE0ADB7BEB712963D
:103250009C938E9311970E94FC7D2091A8040F905F
:103260000F902223A9F000D000D0EDB7FEB7319621
:103270008DE59DE0ADB7BEB712969C938E931197E6
:10328000228313820E94FC7D0F900F900F900F906D
:10329000089500D088E39DE0EDB7FEB79283818367
:1032A0000E94FC7D80E19DE0EDB7FEB792838183B3
:1032B0000E94FC7D89EE9CE0EDB7FEB7928381838E
:1032C0000E94FC7D8FEB9CE0EDB7FEB7928381837B
:1032D0000E94FC7D84E89CE0EDB7FEB79283818379
:1032E0000E94FC7D82E59CE0EDB7FEB7928381836E
:1032F0000E94FC7D86E19CE0EDB7FEB7928381835E
:103300000E94FC7D80EF9BE0EDB7FEB79283818346
:103310000E94FC7D80EC9BE0EDB7FEB79283818339
:103320000E94FC7D87E89BE0EDB7FEB79283818326
:103330000E94FC7D8BE59BE0EDB7FEB79283818315
:103340000E94FC7D82E39BE0EDB7FEB79283818310
:103350000E94FC7D87E09BE0EDB7FEB792838183FE
:103360000E94FC7D88ED9AE0EDB7FEB792838183E1
:103370000E94FC7D86EA9AE0EDB7FEB792838183D6
:103380000E94FC7D85E79AE0EDB7FEB792838183CA
:103390000E94FC7D81E49AE0EDB7FEB792838183C1
:1033A0000E94FC7D81E19AE0EDB7FEB792838183B4
:1033B0000E94FC7D85EE99E0EDB7FEB79283818394
:1033C0000E94FC7D86EB99E0EDB7FEB79283818386
:1033D0000E94FC7D8DE799E0EDB7FEB79283818373
:1033E0000E94FC7D84E599E0EDB7FEB7928381836E
:1033F0000E94FC7D85E199E0EDB7FEB79283818361
:103400000E94FC7D86EE98E0EDB7FEB79283818343
:103410000E94FC7D87EB98E0EDB7FEB79283818335
:103420000E94FC7D80E998E0EDB7FEB7928381832E
:103430000E94FC7D8AE598E0EDB7FEB79283818318
:103440000E94FC7D81E398E0EDB7FEB79283818313
:103450000E94FC7D86E098E0EDB7FEB79283818301
:103460000E94FC7D0F900F90089581ED92E00E94E4
:10347000237E08952F923F924F925F926F927F9298
:103480008F929F92AF92BF92CF92DF92EF92FF9274
:103490000F931F93CF93DF9360916B2070916C20FB
:1034A00080916D2090916E20A0906B20B0906C2048
:1034B000C0906D20D0906E2060906B2070906C203A
:1034C00080906D2090906E2020906B2030906C202A
:1034D00040906D2050906E202DB73EB72A5030405E
:1034E0000FB6F8943EBF0FBE2DBFCDB7DEB7219605
:1034F00026EE37E0EDB7FEB732832183A0E8EA2E4F
:10350000A1E5FA2EA1E00A2F112DA80197010E9432
:10351000797A3B832A83C601B501A80197010E94ED
:10352000797AF0E1EF2EFEE0FF2E012D112DA8019A
:1035300097010E94797A332727FD30953D832C83AC
:10354000C401B301A80197010E94797AECE3EE2E41
:10355000F12C012D112DA80197010E94797A3327B2
:1035600027FD30953F832E83C201B101A801970149
:103570000E94797A772767FD7095798768870E941E
:10358000FC7D2DB73EB7265F3F4F0FB6F8943EBF88
:103590000FBE2DBFDF91CF911F910F91FF90EF9044
:1035A000DF90CF90BF90AF909F908F907F906F9063
:1035B0005F904F903F902F900895E6EAFDE2808162
:1035C000918122E482349207B9F000D000D088ECD7
:1035D00097E0ADB7BEB712969C938E931197E65ABB
:1035E000FD421496FC93EE9313970E94FC7D0F907E
:1035F0000F900F900F9008953A96B1E4E53FFB07C6
:10360000F0F208958F929F92AF92BF92CF92DF9285
:10361000EF92FF920F931F938C9A0E94C10B00D0E0
:1036200000D000D021EC37E0ADB7BEB712963C9386
:103630002E931197EDB7FEB76383748385839683CA
:103640000E94FC7D8DB79EB706960FB6F8949EBF7C
:103650000FBE8DBF81E00E94730B2091A0043091BA
:10366000A1044091A2045091A3040E9494787B018C
:103670008C0182E00E94730B2091A4043091A50478
:103680004091A6045091A7040E949478B62EC72EAC
:10369000D82EA92E83E00E94730B9B01AC01ADB71D
:1036A000BEB71E970FB6F894BEBF0FBEADBFEDB745
:1036B000FEB731968FEA97E012969C938E931197FE
:1036C000C701A02FB12F82839383A483B5830B2DD1
:1036D0001C2DC801AD2DBA2D86839783A087B18795
:1036E00022873387448755870E94FC7D8C98EDB7ED
:1036F000FEB73E960FB6F894FEBF0FBEEDBF0E9418
:10370000D40C1F910F91FF90EF90DF90CF90BF905E
:10371000AF909F908F9008950F931F93CF93DF9357
:10372000882389F085ED94E26FEF70E049E050E086
:103730000E94747D85ED94E268E170E049E050E01C
:103740000E944C7F1CC0C5EDD4E20AEA17E08991C3
:1037500000D000D0EDB7FEB73196ADB7BEB7129628
:103760001C930E931197828313820E94FC7D0F900D
:103770000F900F900F90B4E2CD3DDB0741F70E9410
:10378000D40CDF91CF911F910F910895EF92FF928A
:103790000F931F936091AD047091AE0480E090E0B0
:1037A0000E94667D65EF72E00E947B7D009709F0C4
:1037B00096C086E294E9A0E0B0E08093BF049093C5
:1037C000C004A093C104B093C2048FEB94E06EE0F8
:1037D00070E044E050E00E944C7F8CE390E09093D6
:1037E000C4048093C30483EC94E062E170E042E09F
:1037F00050E00E944C7F8AE090E09093C604809352
:10380000C50485EC94E064E170E042E050E00E9481
:103810004C7F1092DD061092DC068CED96E060E0A5
:1038200070E042E050E00E944C7F0F2EF2E2EF2E5B
:10383000FFEFFF2EFCEC0F2FFBE31F2FF02DE0928C
:10384000A004F092A1040093A2041093A30480EAC0
:1038500094E066E070E044E050E00E944C7FE0922B
:10386000A404F092A5040093A6041093A70484EA8C
:1038700094E06AE070E044E050E00E944C7F87ED05
:1038800094E3AFEEBCE380939C0490939D04A093DB
:103890009E04B0939F048CE994E062E070E044E001
:1038A00050E00E944C7F1092E10681EE96E066E1C6
:1038B00070E041E050E00E944C7F8AE18093E10695
:1038C00087EC94E067E170E041E050E00E944C7FBB
:1038D00081E00E948C1B80E090E00E94570E1F91B7
:1038E0000F91FF90EF900895882309F44BC18091C8
:1038F000BF0480FF0BC000D084EA97E0EDB7FEB7AD
:10390000928381830E94FC7D0F900F908091BF0471
:1039100081FF0BC000D08DE997E0EDB7FEB7928331
:1039200081830E94FC7D0F900F908091BF0482FFE5
:103930000BC000D088E997E0EDB7FEB79283818392
:103940000E94FC7D0F900F908091BF0483FF0BC0FD
:1039500000D082E997E0EDB7FEB7928381830E94A1
:10396000FC7D0F900F908091BF0484FF0BC000D0AE
:1039700089E897E0EDB7FEB7928381830E94FC7DD2
:103980000F900F908091BF0485FF0BC000D080E89E
:1039900097E0EDB7FEB7928381830E94FC7D0F9084
:1039A0000F908091BF0486FF0BC000D08AE797E09C
:1039B000EDB7FEB7928381830E94FC7D0F900F903C
:1039C0008091BF0487FF0BC000D082E797E0EDB77E
:1039D000FEB7928381830E94FC7D0F900F908091AF
:1039E000BF049091C004A091C104B091C20490FFA3
:1039F0000BC000D08CE697E0EDB7FEB792838183D1
:103A00000E94FC7D0F900F908091BF049091C004A4
:103A1000A091C104B091C20491FF0BC000D084E614
:103A200097E0EDB7FEB7928381830E94FC7D0F90F3
:103A30000F908091BF049091C004A091C104B091F7
:103A4000C20492FF0BC000D08AE597E0EDB7FEB745
:103A5000928381830E94FC7D0F900F908091BF0420
:103A60009091C004A091C104B091C20493FF0BC017
:103A700000D084E597E0EDB7FEB7928381830E9482
:103A8000FC7D0F900F908091BF049091C004A09195
:103A9000C104B091C20494FF0BC000D08CE497E045
:103AA000EDB7FEB7928381830E94FC7D0F900F904B
:103AB0008091BF049091C004A091C104B091C20450
:103AC00095FF0BC000D086E497E0EDB7FEB7928378
:103AD00081830E94FC7D0F900F908091BF04909194
:103AE000C004A091C104B091C20496FF0BC000D0E5
:103AF00080E497E0EDB7FEB7928381830E94FC7D5E
:103B00000F900F908091BF049091C004A091C104C8
:103B1000B091C20497FF0BC000D08AE397E0EDB7E5
:103B2000FEB7928381830E94FC7D0F900F9080915D
:103B3000BF049091C004A091C104B091C204A0FF41
:103B40000BC000D085E397E0EDB7FEB79283818389
:103B50000E94FC7D0F900F908091BF049091C00453
:103B6000A091C104B091C204A1FF14C200D08FE2A1
:103B700097E0EDB7FEB7928381830E94FC7D0F90A2
:103B80000F9008C200D000D000D083E297E0EDB7DC
:103B9000FEB79283818381E090E0A0E0B0E0838370
:103BA0009483A583B6830E94FC7D8DB79EB706964D
:103BB0000FB6F8949EBF0FBE8DBF0E94D40C00D0EC
:103BC00000D000D086E197E0EDB7FEB79283818305
:103BD00082E090E0A0E0B0E083839483A583B68385
:103BE0000E94FC7D8DB79EB706960FB6F8949EBFD7
:103BF0000FBE8DBF0E94D40C00D000D000D08BE04F
:103C000097E0EDB7FEB79283818384E090E0A0E077
:103C1000B0E083839483A583B6830E94FC7D8DB737
:103C20009EB706960FB6F8949EBF0FBE8DBF0E943A
:103C3000D40C00D000D000D08FEF96E0EDB7FEB7E7
:103C40009283818388E090E0A0E0B0E08383948356
:103C5000A583B6830E94FC7D8DB79EB706960FB6EE
:103C6000F8949EBF0FBE8DBF0E94D40C00D000D030
:103C700000D081EF96E0EDB7FEB79283818380E1BB
:103C800090E0A0E0B0E083839483A583B6830E9494
:103C9000FC7D8DB79EB706960FB6F8949EBF0FBEFB
:103CA0008DBF0E94D40C00D000D000D083EE96E0EF
:103CB000EDB7FEB79283818380E290E0A0E0B0E0B0
:103CC00083839483A583B6830E94FC7D8DB79EB7C2
:103CD00006960FB6F8949EBF0FBE8DBF0E94D40CFF
:103CE00000D000D000D087ED96E0EDB7FEB792830C
:103CF000818380E490E0A0E0B0E083839483A58397
:103D0000B6830E94FC7D8DB79EB706960FB6F894D9
:103D10009EBF0FBE8DBF0E94D40C00D000D000D03B
:103D200089EC96E0EDB7FEB79283818380E890E05E
:103D3000A0E0B0E083839483A583B6830E94FC7DDA
:103D40008DB79EB706960FB6F8949EBF0FBE8DBF77
:103D50000E94D40C00D000D000D08DEB96E0EDB7DF
:103D6000FEB79283818380E091E0A0E0B0E083839E
:103D70009483A583B6830E94FC7D8DB79EB706967B
:103D80000FB6F8949EBF0FBE8DBF0E94D40C00D01A
:103D900000D000D08FEA96E0EDB7FEB79283818322
:103DA00080E092E0A0E0B0E083839483A583B683B3
:103DB0000E94FC7D8DB79EB706960FB6F8949EBF05
:103DC0000FBE8DBF0E94D40C00D000D000D080EA7E
:103DD00096E0EDB7FEB79283818380E094E0A0E0A7
:103DE000B0E083839483A583B6830E94FC7D8DB766
:103DF0009EB706960FB6F8949EBF0FBE8DBF0E9469
:103E0000D40C00D000D000D084E996E0EDB7FEB726
:103E10009283818380E098E0A0E0B0E08383948384
:103E2000A583B6830E94FC7D8DB79EB706960FB61C
:103E3000F8949EBF0FBE8DBF0E94D40C00D000D05E
:103E400000D086E896E0EDB7FEB79283818380E0EC
:103E500090E1A0E0B0E083839483A583B6830E94C1
:103E6000FC7D8DB79EB706960FB6F8949EBF0FBE29
:103E70008DBF0E94D40C00D000D000D08AE796E01D
:103E8000EDB7FEB79283818380E090E2A0E0B0E0DE
:103E900083839483A583B6830E94FC7D8DB79EB7F0
:103EA00006960FB6F8949EBF0FBE8DBF0E94D40C2D
:103EB00000D000D000D08EE696E0EDB7FEB792833A
:103EC000818380E090E4A0E0B0E083839483A583C5
:103ED000B6830E94FC7D8DB79EB706960FB6F89408
:103EE0009EBF0FBE8DBF0E94D40C00D000D000D06A
:103EF00082E696E0EDB7FEB79283818380E090E89A
:103F0000A0E0B0E083839483A583B6830E94FC7D08
:103F10008DB79EB706960FB6F8949EBF0FBE8DBFA5
:103F20000E94D40C00D000D000D086E596E0EDB71A
:103F3000FEB79283818380E090E0A1E0B0E08383CC
:103F40009483A583B6830E94FC7D8DB79EB70696A9
:103F50000FB6F8949EBF0FBE8DBF0E94D40C00D048
:103F600000D000D089E496E0EDB7FEB7928381835C
:103F700080E090E0A2E0B0E083839483A583B683E1
:103F80000E94FC7D8DB79EB706960FB6F8949EBF33
:103F90000FBE8DBF0E94D40C08952F923F924F9276
:103FA0005F926F927F928F929F92AF92BF92CF92C9
:103FB000DF92EF92FF920F931F93DF93CF9300D086
:103FC000CDB7DEB79A838983DC018D919C911197DF
:103FD000009711F00C94A9336091AD047091AE0478
:103FE00080E890E20E94667D80E890E260E470E004
:103FF0000E94847D009759F46091A02D7091A12DAD
:104000008AE090E00E94BE7D81E00C94AE33813066
:10401000910549F4209080203324442455246624BB
:1040200077244301BFC18230910599F430918020FB
:1040300020918120932F80E0820F911D1C01892FF8
:10404000880F880B482E582E682E782E882E982E92
:10405000A9C18330910509F09CC020918020A090D7
:1040600081208090822030E040E050E060E070E00D
:1040700080E090E000E10E942072F22E132FE42EE7
:10408000D52EC62EB72E282E992E2A2D30E040E0B0
:1040900050E060E070E080E090E008E00E94207274
:1040A0002F0DB1E02F1508F0B0E0310FE1E031172E
:1040B00008F0E0E0B30FF1E0B31708F0F0E0EF2B09
:1040C0004E0D31E04E1508F030E0E40FF1E0E4175A
:1040D00008F0F0E03F2B5D0D41E05D1508F040E099
:1040E000A32FA50F31E0A51708F030E0432B6C0D8E
:1040F00031E06C1508F030E0F42FF60F41E0F617D0
:1041000008F040E0342B7B0D41E07B1508F040E0E7
:10411000532F570F31E0571708F030E0432B820D33
:1041200031E0821508F030E0480F61E0481708F0F0
:1041300060E0362B990D930F022F080D11E0021746
:1041400008F010E01B0F81E01B1708F080E0B82F8B
:10415000BE0F71E0BE1708F070E07A0F61E07A17C9
:1041600008F060E06F0F31E06F1708F030E0350FB6
:1041700021E0351708F020E0240F81E0241708F033
:1041800080E018014B2E572E662E732E822E982E0D
:10419000FEC0843091050CF4FCC020918020A090DA
:1041A0008120709082208090832030E040E050E0B9
:1041B00060E070E080E090E008E10E942072F22E62
:1041C000132FE42ED52EC62EB72E282E992E2A2D4B
:1041D00030E040E050E060E070E080E090E000E13E
:1041E0000E9420722F0DF1E02F1508F0F0E0310F42
:1041F000E1E0311708F0E0E0F30FA1E0F31708F079
:10420000A0E0EA2B4E0D31E04E1508F030E0E40F4F
:10421000A1E0E41708F0A0E03A2B5D0D41E05D1548
:1042200008F040E0B32FB50F31E0B51708F030E0EB
:10423000432B6C0D31E06C1508F030E0A42FA60F75
:1042400041E0A61708F040E0342B7B0D41E07B15E0
:1042500008F040E0532F570F31E0571708F030E0D7
:10426000432B820D31E0821508F030E0480F61E009
:10427000481708F060E0362B990E930E122F180D98
:1042800081E0121708F080E0282E2F0E81E02F1613
:1042900008F080E0F82EFE0E81E0FE1608F080E0C7
:1042A000E82EEB0E81E0EB1608F080E0D82EDA0E57
:1042B00081E0DA1608F080E0C82EC50E81E0C51650
:1042C00008F080E0B82EB40E81E0B41608F080E06B
:1042D000980E272D30E040E050E060E070E080E094
:1042E00090E008E00E942072210FE1E0211708F021
:1042F000E0E0320DF1E0321508F0F0E0E30FA1E06C
:10430000E31708F0A0E0FA2B4F0D31E04F1508F04D
:1043100030E0F40FA1E0F41708F0A0E03A2B5E0DB6
:1043200041E05E1508F040E0A32FA50F31E0A5178E
:1043300008F030E0432B6D0D31E06D1508F030E0F2
:10434000542F560F41E0561708F040E0342B7C0DF7
:1043500041E07C1508F040E0632F670F31E06717FC
:1043600008F030E0432B8B0D31E08B1508F030E086
:10437000480F71E0481708F070E0372B990D222E96
:104380003E2E4F2E5A2E652E762E842E932E990E6B
:1043900009C0AAE02A2E3324442455246624772415
:1043A000882499240E94D40CB22DB33689F4E32DCD
:1043B000E23371F4F42DF93659F4552049F46620AE
:1043C00039F4772029F4882019F4992009F46AC572
:1043D0009101A201B301C401F3E6AF2EE2E3BE2EC8
:1043E00009E6C02EDD24EE24FF2400E010E00E9448
:1043F0009172823008F074C2822D853689F4932D33
:10440000923771F4442061F4552051F4662041F450
:10441000772031F4882021F4992011F40C94792F1D
:104420009101A201B301C40115E6A12EB2E7BB2E92
:10443000CC24DD24EE24FF2400E010E00E949172E1
:10444000823008F009C1A22DA53681F4B32DB4360F
:1044500069F4442059F4552049F4662039F4772052
:1044600029F4882019F4992009F4E9C69101A201E0
:10447000B301C401A5E6AA2EF4E6BF2ECC24DD24A8
:10448000EE24FF2400E010E00E949172823008F0D8
:1044900063C0E22DE53781F4332071F4442061F4E8
:1044A000552051F4662041F4772031F4882021F41E
:1044B000992011F40C94822A9101A201B301C40144
:1044C000E5E7AE2EBB24CC24DD24EE24FF2400E05F
:1044D00010E00E949172823010F5F22DF83611F042
:1044E0000C94A733332011F00C94A733442011F01F
:1044F0000C94A733552011F00C94A733662011F0CB
:104500000C94A733772011F00C94A733882011F076
:104510000C94A733992011F00C94A733AEC7822DC9
:10452000863779F4332069F4442059F4552049F44E
:10453000662039F4772029F4882019F4992009F4A9
:10454000F1C7922D943611F00C94A733A32DA13608
:1045500011F00C94A7337BC0B22DB73789F4E32D4B
:10456000EF3671F4442061F4552051F4662041F493
:10457000772031F4882021F4992011F40C940D2E29
:104580009101A201B301C40107E7A02E1FE6B12EDD
:10459000CC24DD24EE24FF2400E010E00E94917280
:1045A0008230B8F5F22DF43681F4832D893669F422
:1045B000442059F4552049F4662039F4772029F431
:1045C000882019F4992009F473C7922D953611F0BB
:1045D0000C94A733A32DAE3611F00C94A7334420CE
:1045E00011F00C94A733552011F00C94A7336620DA
:1045F00011F00C94A733772011F00C94A733882086
:1046000011F00C94A733992011F00C94A7330C945B
:10461000692EB22DB13389F4E32DE03771F44420D3
:1046200061F4552051F4662041F4772031F488205C
:1046300021F4992011F40C94FA2EF22DF33311F099
:104640000C94A733832D813711F00C94A7334420A9
:1046500011F00C94A73395C0922D983789F4A32DAF
:10466000A43671F4B42DB13659F4552049F46620BE
:1046700039F4772029F4882019F4992009F40EC41C
:104680009101A201B301C401B8E7AB2EA4E6BA2E92
:10469000F1E6CF2EDD24EE24FF2400E010E00E949E
:1046A0009172823008F083C0E22DE33789F4F32D54
:1046B000F23771F4442061F4552051F4662041F43E
:1046C000772031F4882021F4992011F40C9445309E
:1046D0009101A201B301C401E3E7AE2E02E7B02EBF
:1046E000CC24DD24EE24FF2400E010E00E9491722F
:1046F000823020F5822D893611F00C94A733932D4A
:10470000923711F00C94A733442011F00C94A73386
:10471000552011F00C94A733662011F00C94A733A8
:10472000772011F00C94A733882011F00C94A73354
:10473000992011F00C94A7330C94F22FA22DA337DB
:1047400089F4B32DB33771F4442061F4552051F44A
:10475000662041F4772031F4882021F4992011F467
:104760000C945430E22DE33611F00C94A733F32D62
:10477000F43611F00C94A733842D813611F00C948B
:10478000A733552011F00C94A733662011F00C9438
:10479000A733772011F00C94A733882011F00C94E4
:1047A000A733992011F00C94A7330C944C32922D1E
:1047B000923791F4A32DA23779F4B42DB53661F474
:1047C000552051F4662041F4772031F4882021F4FB
:1047D000992011F40C94302D9101A201B301C40170
:1047E00012E7A12EB2E7BB2EA5E6CA2EDD24EE24E9
:1047F000FF2400E010E00E9491728230C0F5E22DAB
:10480000E33789F4F32DF53671F4842D813659F4AC
:10481000552049F4662039F4772029F4882019F4CA
:10482000992009F48FC6922D923611F00C94A7337B
:10483000A32DA53611F00C94A733B42DB43611F086
:104840000C94A733552011F00C94A733662011F077
:104850000C94A733772011F00C94A733882011F023
:104860000C94A733992011F00C94A733E8C4E22DDF
:10487000E33689F4F32DFD3671F4842D883659F42E
:10488000552049F4662039F4772029F4882019F45A
:10489000992009F40BC3922D9D3611F00C94A73387
:1048A000A32DA53711F00C94A733B42DB83611F011
:1048B0000C94A733552011F00C94A733662011F007
:1048C0000C94A733772011F00C94A733882011F0B3
:1048D0000C94A733992011F00C94A7330C945B32FD
:1048E000E22DE63391F4F32DF93679F4842D8537F2
:1048F00061F4952D953649F4662039F4772029F432
:10490000882019F4992009F4BCC59101A201B301D2
:10491000C401F6E3AF2EE9E6BE2E05E7C02E15E68C
:10492000D12EEE24FF2400E010E00E94917282302C
:1049300008F04BC1A22DA13391F4B32DB13379F41A
:10494000E42DE13761F4552051F4662041F47720DD
:1049500031F4882021F4992011F40C94932D9101C5
:10496000A201B301C401B1E3AB2EA1E3BA2EF1E77A
:10497000CF2EDD24EE24FF2400E010E00E9491728F
:10498000823008F085C0F22DF73691F4832D8F36F2
:1049900079F4942D9C3661F4552051F4662041F44D
:1049A000772031F4882021F4992011F40C94DD2C27
:1049B0009101A201B301C401E7E6AE2E0FE6B02ECD
:1049C0001CE6C12EDD24EE24FF2400E010E00E944E
:1049D0009172823020F5A22DA43611F00C94A733E9
:1049E000B32DB33611F00C94A733E42DEC3611F04F
:1049F0000C94A733552011F00C94A733662011F0C6
:104A00000C94A733772011F00C94A733882011F071
:104A10000C94A733992011F00C94A733CBC7F22D37
:104A2000F53791F4832D833679F4942D9D3661F416
:104A3000552051F4662041F4772031F4882021F488
:104A4000992011F40C94932DA22DA03311F00C9405
:104A5000A733B32DB13311F00C94A733E42DE13714
:104A600011F00C94A733552011F00C94A733662055
:104A700011F00C94A733772011F00C94A733882001
:104A800011F00C94A733992011F00C94A733E8C7C8
:104A9000F22DF43791F4832D8F3679F4942D9F36CF
:104AA00061F4A52DA23649F4662039F4772029F463
:104AB000882019F4992009F4D3C59101A201B3010A
:104AC000C401B4E7AB2EAFE6BA2EFFE6CF2EE2E686
:104AD000DE2EEE24FF2400E010E00E94917282306E
:104AE000D0F5B22DB03791F4E32DE53679F4F42DFD
:104AF000F23761F4552051F4662041F4772031F407
:104B0000882021F4992011F40C94792F822D843778
:104B100011F00C94A733932D943611F00C94A73315
:104B2000A42DA73711F00C94A733552011F00C9445
:104B3000A733662011F00C94A733772011F00C9462
:104B4000A733882011F00C94A733992011F00C940E
:104B5000A7330C943E33B22DB93691F4E32DEC36E5
:104B600079F4F42DF13661F4852D833649F466200D
:104B700039F4772029F4882019F4992009F4C3C165
:104B8000922D9E3611F00C94A733A32DA13611F06F
:104B90000C94A733B42DB83611F00C94A733E52D3F
:104BA000E33611F00C94A733662011F00C94A73370
:104BB000772011F00C94A733882011F00C94A733C0
:104BC000992011F00C94A73320C5F22DF33799F4F6
:104BD000832D823781F4942D973769F4A52DA03762
:104BE00051F4662041F4772031F4882021F4992093
:104BF00011F40C94452F9101A201B301C40103E704
:104C0000A02E12E7B12EB7E7CB2EA0E7DA2EEE24C6
:104C1000FF2400E010E00E949172823008F09FC0F3
:104C2000B22DB03799F4E32DED3681F4F42DF5373C
:104C300069F4852D883651F4662041F4772031F4EB
:104C4000882021F4992011F40C94332E9101A201B3
:104C5000B301C401F0E7AF2EEDE6BE2E05E7C02E8E
:104C600018E6D12EEE24FF2400E010E00E9491729D
:104C70008230D0F5922D903791F4A32DAC3679F493
:104C8000B42DB53661F4E52DE83649F4662039F4E3
:104C9000772029F4882019F4992009F4EEC3F22D25
:104CA000F13611F00C94A733832D8D3611F00C944E
:104CB000A733942D953711F00C94A733A52DA83662
:104CC00011F00C94A733662011F00C94A7337720D1
:104CD00011F00C94A733882011F00C94A73399207D
:104CE00011F00C94A733AEC7B22DB33799F4E32D6E
:104CF000E53681F4F42DF23769F4852D803751F4CF
:104D0000662041F4772031F4882021F4992011F4B1
:104D10000C94A632922D913311F00C94A733A32D4D
:104D2000A23711F00C94A733B42DB73711F00C94BF
:104D3000A733E52DE03711F00C94A733662011F06E
:104D40000C94A733772011F00C94A733882011F02E
:104D50000C94A733992011F00C94A733ABC0F22D1B
:104D6000F73791F4832D803779F4942D983761F4D7
:104D7000A52DA43749F4662039F4772029F488203A
:104D800019F4992009F41BC49101A201B301C401D3
:104D9000B7E7AB2EA0E7BA2EF8E7CF2EE4E7DE2E7A
:104DA000EE24FF2400E010E00E9491728230D8F5DA
:104DB000B22DB43799F4E32DE33781F4F42DF536B1
:104DC00069F4852D823751F4662041F4772031F45F
:104DD000882021F4992011F40C94F72E922D943709
:104DE00011F00C94A733A32DA33711F00C94A73323
:104DF000B42DB53611F00C94A733E52DE43711F03E
:104E00000C94A733662011F00C94A733772011F08F
:104E10000C94A733882011F00C94A733992011F03B
:104E20000C94A73321C4F22DF23791F4832D8736E9
:104E300079F4942D903761F4A52DA53749F46620B7
:104E400039F4772029F4882019F4992009F481C5D0
:104E5000B22DBC3611F00C94A733E32DE13611F0DE
:104E60000C94A733F42DF43711F00C94A733852D4F
:104E7000883711F00C94A733662011F00C94A733F7
:104E8000772011F00C94A733882011F00C94A733ED
:104E9000992011F00C94A7330C9402330E943C1615
:104EA0000C94A9330E94A1100C94A9330E94C5163A
:104EB0000C94A9336091AD047091AE0480E090E051
:104EC0000E94667D8C016CEF72E00E947B7D0097F2
:104ED00019F477980C94A933C8016FEF72E00E941F
:104EE0007B7D009719F4779A0C94A933779903C0C6
:104EF0008CEF92E002C08FEF92E000D000D021E66C
:104F000035E00C9496336091AD047091AE0480E06E
:104F100090E00E94667D8C0166E073E00E947B7DDC
:104F2000009709F052C06091AD047091AE0480E02A
:104F300090E00E94667D8C01009711F40C94A933D7
:104F400069E073E00E947B7D009729F482E29FEF85
:104F5000ACECBBE30BC0C8016FE073E00E947B7D4B
:104F6000009789F482E29FEFACECBAE38093A0044F
:104F70009093A104A093A204B093A30480EA94E0C8
:104F800066E070E0DCC0C8010E94597C7B018C01A6
:104F900020E030E0A9010E944A77882391F081E067
:104FA0000E94730B9B01AC01C801B7010E944E77B0
:104FB0006093A0047093A1048093A2049093A3042F
:104FC000DDCF00D081EA95E08CC0C80164E173E0D8
:104FD0000E947B7D009709F052C06091AD047091F2
:104FE000AE0480E090E00E94667D8C01009711F491
:104FF0000C94A93369E073E00E947B7D009729F44B
:1050000082E29FEFACECBBE30BC0C8016FE073E042
:105010000E947B7D009769F482E29FEFACECBAE3DB
:105020008093A4049093A504A093A604B093A7042E
:105030001DC0C8010E94597C7B018C0120E030E03A
:10504000A9010E944A778823B1F082E00E94730B85
:105050009B01AC01C801B7010E944E776093A40484
:105060007093A5048093A6049093A70484EA94E027
:105070006AE070E064C000D084E995E066C0C801D1
:1050800067E173E00E947B7D009709F06AC0609140
:10509000AD047091AE0480E090E00E94667D8C01CA
:1050A000009711F40C94A93369E073E00E947B7DB2
:1050B000009769F487ED94E3AFEEBCE380939C0422
:1050C00090939D04A0939E04B0939F0434C0C801A4
:1050D0006FE073E00E947B7D009741F400D085E88B
:1050E00095E0EDB7FEB79283818335C0C8010E9479
:1050F000597C1B012C0120E030E0A9010E944A7775
:10510000882301F180E00E94730B7B018C01C201B6
:10511000B10121EE3AE744E95EE30E948376A801FB
:1051200097010E944E7760939C0470939D04809336
:105130009E0490939F048CE994E062E070E044E068
:1051400050E01EC200D088E795E0ADB7BEB712961A
:105150009C938E9311970E94FC7D0F900F900C945E
:10516000A9330E94C10B00D000D000D021E735E068
:10517000EDB7FEB732832183ADB7BEB713966D93FB
:105180007D938D939C9316970E94FC7DEDB7FEB79F
:1051900036960FB6F894FEBF0FBEEDBF81E00E94B9
:1051A000730B2091A0043091A1044091A20450916E
:1051B000A3040E9494787B018C0182E00E94730B0F
:1051C0009B01AC018DB79EB70A970FB6F8949EBFAE
:1051D0000FBE8DBFCDB6DEB60894C11CD11C85E6CE
:1051E00095E0ADB7BEB712969C938E9311978E2D16
:1051F0009F2DA02FB12FF60182839383A483B583C3
:10520000CA01B9012091A4043091A5044091A604DB
:105210005091A7040E949478D60116966D937D93C1
:105220008D939C9319970E94FC7DEDB7FEB73A963B
:105230000FB6F894FEBF0FBEEDBF0C943B336091E8
:10524000AD047091AE0480E090E00E94667D00970E
:1052500061F160E070E040E150E00E944B7B209102
:10526000DC063091DD062617370799F17093DD06CD
:105270006093DC068CED96E060E070E042E050E088
:105280000E944C7F8091DC069091DD0600D000D01A
:1052900021E535E0ADB7BEB712963C932E9311973A
:1052A00014969C938E9313970EC08091DC06909178
:1052B000DD0600D000D02DE335E0EDB7FEB7328338
:1052C0002183948383830E94FC7D0F900F900F9025
:1052D0000F900E94D40C00D000D080E395E0ADB7D1
:1052E000BEB712969C938E93119781E090E014962E
:1052F0009C938E9313970E94FC7D85E295E0EDB719
:10530000FEB79283818382E090E0948383830E943E
:10531000FC7D8AE195E0ADB7BEB712969C938E9363
:10532000119784E090E014969C938E9313970E94BB
:10533000FC7D8DE095E0EDB7FEB79283818388E038
:1053400090E0948383830E94FC7D82E095E0ADB77A
:10535000BEB712969C938E93119780E190E01496BD
:105360009C938E9313970E94FC7D86EF94E0EDB79B
:10537000FEB79283818380E290E0948383830E94CE
:10538000FC7D88EE94E0ADB7BEB712969C938E93E9
:10539000119780E490E014969C938E9313970E944B
:1053A000FC7D8AED94E0EDB7FEB79283818380E8BF
:1053B00090E0948383830E94FC7D8BEC94E0ADB7F6
:1053C000BEB712969C938E93119780E091E014964D
:1053D0009C938E9313970E94FC7D8CEB94E0EDB729
:1053E000FEB79283818380E092E0948383830E945E
:1053F000FC7D80EB94E0ADB7BEB712969C938E9384
:10540000119780E094E014969C938E9313970E94DA
:10541000FC7D82EA94E0EDB7FEB79283818380E061
:1054200098E0948383830E94FC7D85E994E0ADB786
:10543000BEB712969C938E93119780E090E11496DC
:105440009C938E9313970E94FC7D87E894E0EDB7C0
:10545000FEB79283818380E090E2948383830E94ED
:10546000FC7D87E794E0ADB7BEB712969C938E9310
:10547000119780E090E40C949C330E9449190C949D
:10548000A93380918420843329F480E061E040E0F6
:105490000E94E1112091A804222311F40C94A93355
:1054A00000D000D0EDB7FEB7319684E794E020C07D
:1054B0006091AD047091AE0480E090E00E94667D42
:1054C00069E073E00E947B7D009711F481E001C0E8
:1054D00080E00E948C1B2091A804222311F40C94DC
:1054E000A93300D000D0EDB7FEB7319681E794E044
:1054F000ADB7BEB712969C938E93119722831382F9
:105500000C94A0330E943A1A2091A804222311F48B
:105510000C94A93300D000D0EDB7FEB731968EE6DB
:1055200094E0E6CF0E94351A2091A804222311F4BA
:105530000C94A93300D000D0EDB7FEB731968BE6BE
:1055400094E0D6CF6091AD047091AE0480E090E01D
:105550000E94667D8C016CEF72E00E947B7D00975B
:1055600099F48091C5049091C60484609093C60418
:105570008093C50485EC94E064E170E042E050E083
:105580000E944C7F0C94A933C8016FEF72E00E9417
:105590007B7D9C018091C5049091C6042115310545
:1055A00011F48B7FE3CF82FF03C08CEF92E002C047
:1055B0008FEF92E000D000D02EEA35E083C36091F7
:1055C000AD047091AE0480E090E00E94667D0E9480
:1055D0005D7C803150F48093E10690E00E942C576E
:1055E00081EE96E066E170E027C000D000D0EDB714
:1055F000FEB7319682EB95E0ADB7BEB712969C939D
:105600008E9311978091E10629C06091AD0470914D
:10561000AE0480E090E00E94667D0E945D7C982F41
:105620009B50903160F48093C70490E00E94A45591
:1056300087EC94E067E170E041E050E0A1CF00D05A
:1056400000D0EDB7FEB731968FEB95E0ADB7BEB7A2
:1056500012969C938E9311978091C70482834FCFAB
:105660000C9400000C94A9336091AD047091AE04C9
:1056700080E090E00E94667D8C016CE173E00E9406
:105680007B7D009739F4219A8091C5049091C604DE
:1056900080616CCFC8016EE173E00E947B7D009752
:1056A00039F4229A8091C5049091C60480625ECF3D
:1056B000C80160E273E00E947B7D009739F4239A71
:1056C0008091C5049091C604806450CFC80162E205
:1056D00073E00E947B7D009739F4239A8091C50482
:1056E0009091C604806842CFC80164E273E00E94D2
:1056F0007B7D0097D1F48091C5049091C6049160A0
:105700009093C6048093C50485EC94E064E170E056
:1057100042E050E00E944C7F88E095E062E140E08A
:1057200050E00E94C4400C94A933C80166E273E0C3
:105730000E947B7D009771F4EBEAF7E111921192E0
:10574000B7E1EB3CFB07D1F78091C5049091C6040B
:1057500092600CCFC8016FEF72E00E947B7D9C01CC
:105760008091C5049091C60421153105A9F48F706C
:105770009C7F9093C6048093C5042B9A85EC94E09B
:1057800064E170E042E050E00E944C7F8091CC24C4
:1057900090E00E94B955DDC784FF03C08CEF92E012
:1057A00002C08FEF92E000D000D02FEF35E0EDB7D0
:1057B000FEB732832183948383830E94FC7D809192
:1057C000C5040F900F900F900F9085FF03C08CEFD2
:1057D00092E002C08FEF92E000D000D024EF35E0DD
:1057E000ADB7BEB712963C932E93119714969C9327
:1057F0008E9313970E94FC7D8091C5040F900F90AB
:105800000F900F9086FF03C08CEF92E002C08FEFE5
:1058100092E000D000D029EE35E0EDB7FEB732833C
:105820002183948383830E94FC7D8091C5040F9023
:105830000F900F900F9087FF03C08CEF92E002C093
:105840008FEF92E000D000D02EED35E0ADB7BEB7BF
:1058500012963C932E93119714969C938E931397C4
:105860000E94FC7D8091C5049091C6040F900F901A
:105870000F900F9090FF03C08CEF92E002C08FEF6B
:1058800092E000D000D023ED35E0EDB7FEB73283D3
:105890002183948383830E94FC7D8091C504909131
:1058A000C6040F900F900F900F9091FF03C08CEFE4
:1058B00092E002C08FEF92E000D000D028EC35E0FB
:1058C000ADB7BEB712963C932E93119714969C9346
:1058D0008E9313970E94FC7D8091C5049091C6041D
:1058E0000F900F900F900F9091FF33C788E293E0D5
:1058F0000E94237E0BEA17E18BE0C82ED12CB0E387
:10590000EB2EB3E0FB2EF801819191918F0100D035
:1059100000D000D0EDB7FEB73196ADB7BEB7129646
:10592000FC92EE921197D382C282958384830E9467
:10593000EA7D0894C11CD11CEDB7FEB736960FB6B0
:10594000F894FEBF0FBEEDBFFBE1CF16D104D9F630
:1059500000C700D087E694E0ADB7BEB712969C931F
:105960008E9311970E94FC7D2091A8040F900F90B8
:105970002223A9F000D000D0EDB7FEB7319684E61F
:1059800094E0ADB7BEB712969C938E931197228385
:1059900013820E94FC7D0F900F900F900F9088E172
:1059A0000FB6F89480936000109260000FBE0C94C4
:1059B000007CCFC60E94D64DCCC66091AD047091DC
:1059C000AE0480E090E00E94667D1C016CEF72E006
:1059D0000E947B7D009749F40E9483548091C50406
:1059E0009091C60481608D7FC1CDC1016FEF72E0DF
:1059F0000E947B7D009741F40E94E5538091C5048D
:105A00009091C6048C7FB2CD0BE313E0C101B801C5
:105A10000E947B7D009749F40E94E5538091C50464
:105A20009091C6048E7F8260A1CD8091C50481FFD4
:105A30000BC000D000D08EE096E0EDB7FEB79283A9
:105A40008183148303837CC680FF03C08CEF92E0C4
:105A500002C08FEF92E000D000D02AE036E066C6A8
:105A600000D08AE394E0EDB7FEB7928381830E9471
:105A7000FC7D8DB79EB740970FB6F8949EBF0FBEC2
:105A80008DBFEDB7FEB731968CE194E0ADB7BEB7F0
:105A900012969C938E93119780917B2090917C20FD
:105AA000A0917D20B0917E2082839383A483B583CF
:105AB00080916F2090917020A0917120B091722000
:105AC00086839783A087B1878091732090917420FB
:105AD000A0917520B091762082879387A487B5879F
:105AE0008091772090917820A0917920B0917A20B0
:105AF00086879787A08BB18B0E94FC7D2091A8049C
:105B0000EDB7FEB772960FB6F894FEBF0FBEEDBFAD
:105B1000222309F41EC600D000D0EDB7FEB731969F
:105B200089E194E0E5CCF89481E090E00E94BE0821
:105B3000182F80E090E00E94BE08082F7894F89417
:105B400083E090E00E94BE08F82E82E090E00E9480
:105B5000BE08E82E789400D000D000D02FE034E0CA
:105B6000EDB7FEB73283218320911C1830911D18A8
:105B700040911E1850911F18ADB7BEB713962D93C4
:105B80003D934D935C9316970E94FC7D00D000D00E
:105B9000EDB7FEB7319628EE33E0ADB7BEB712963B
:105BA0003C932E931197E2821382F482158206832E
:105BB0001782108711860E94FC7DEDB7FEB73A96DA
:105BC0000FB6F894FEBF0FBEEDBF0E94DD1A209104
:105BD000660000D000D0EDB7FEB731968CED93E0B3
:105BE000ADB7BEB712969C938E9311972283138202
:105BF0000E94FC7D0F900F900F900F900E94D40C8C
:105C00002091A804222309F4A4C500D000D0EDB748
:105C1000FEB7319689ED93E06BCC80E090E00E9476
:105C2000E00C81E090E00E94E00C2091A804222387
:105C300009F48FC500D000D0EDB7FEB7319686EDE0
:105C400093E056CC0E94B8180E94D40C2091A8046E
:105C5000222309F47EC500D000D0EDB7FEB73196FF
:105C600083ED93E045CC6091AD047091AE0480E08B
:105C700090E00E94667D8C016CEF72E00E947B7D5B
:105C8000009731F48091C5049091C60488606ECC71
:105C9000C8016FEF72E00E947B7D9C018091C5047A
:105CA0009091C6042115310511F4877F5FCC83FFE5
:105CB00003C08CEF92E002C08FEF92E000D000D0E2
:105CC00022E136E0EDB7FEB73283218394838383EC
:105CD00037C56091AD047091AE0480E090E00E9401
:105CE000667D60E473E00E947B7D009741F5F89447
:105CF00081E097E00E94BB410CC0C8010D960E9454
:105D0000074585E595E0B8010E947541C8010E94EC
:105D10008142082F192F0115110579F704C081E080
:105D200097E00E94FC4181E097E00E946142009769
:105D3000B1F781E097E00E94B74178944BC081E0D1
:105D400097E00E94BB41482F592F7A0106E413E0E7
:105D50003DC08DB79EB70C970FB6F8949EBF0FBE8F
:105D60008DBFEDB7FEB73196ADB7BEB712961C9397
:105D70000E931197D70112968C91129782831382FA
:105D800013968C9113978483158218968C9118978B
:105D90008683178214968D919C91159791878087A1
:105DA00016968D919C911797938782870E94EA7D22
:105DB000EDB7FEB73C960FB6F894FEBF0FBEEDBF31
:105DC000C7010E948142482F592F7A01E114F10442
:105DD00009F0BFCF2091A804222309F4BAC400D04F
:105DE00000D0EDB7FEB7319680ED93E081CB0E94F5
:105DF000C61BAFC46091AD047091AE0480E090E02A
:105E00000E94667D8C016CEF72E00E947B7D0097A2
:105E100031F48091C5049091C60490610EC0C80110
:105E20006FEF72E00E947B7D9C018091C504909190
:105E3000C6042115310571F49F7E9093C6048093AA
:105E4000C50485EC94E064E170E042E050E00E941B
:105E50004C7F17C094FF03C08CEF92E002C08FEF1D
:105E600092E000D000D026E136E0EDB7FEB73283F5
:105E70002183948383830E94FC7D0F900F900F9069
:105E80000F9081E00E94E30A64C46091AD047091B8
:105E9000AE0480E090E00E94667D8C016DE673E0C8
:105EA0000E947B7D009731F48091C5049091C604D7
:105EB000937F5CCBC8016FE073E00E947B7D00970D
:105EC00039F48091C5049091C604937F98604ECBBD
:105ED000C80162E773E00E947B7D009739F48091EE
:105EE000C5049091C604937F946040CB0E94C5087E
:105EF00030C46091AD047091AE0480E090E00E94E7
:105F0000667D0097A9F160E070E040E150E00E94FA
:105F10004B7B6093BF047093C0048093C104909343
:105F2000C20400D000D000D02DEB33E0ADB7BEB737
:105F300012963C932E931197EDB7FEB7638374834B
:105F4000858396830E94FC7D8DB79EB706960FB61B
:105F5000F8949EBF0FBE8DBF8FEB94E06EE070E0B3
:105F600044E050E00E944C7F81E00E94741CF1C329
:105F700080E00E94741C0E94D40C00D000D000D09D
:105F800088EA93E0ADB7BEB712969C938E931197B3
:105F90008091BF049091C004A091C104B091C2044B
:105FA000EDB7FEB783839483A583B6830E94FC7DFF
:105FB0008DB79EB706960FB6F8949EBF0FBE8DBFE5
:105FC00081E00E94741C0E94D40C2091A80422231A
:105FD00009F4BFC300D000D0EDB7FEB7319685EA13
:105FE00093E086CA6091AD047091AE0480E090E0C9
:105FF0000E94667D009741F160E070E04AE050E069
:106000000E944B7B7093C4046093C30400D000D003
:10601000EDB7FEB7319628E833E0ADB7BEB71296BC
:106020003C932E931197738362830E94FC7D0F90A3
:106030000F900F900F9083EC94E062E170E042E0EB
:1060400050E00E944C7F14C000D000D087E693E05F
:10605000EDB7FEB7928381838091C3049091C4040D
:10606000948383830E94FC7D0F900F900F900F907C
:106070002091A804222309F46CC300D000D0EDB70E
:10608000FEB7319684E693E033CA0E9444452091DE
:10609000A804222309F45DC300D000D0EDB7FEB7F9
:1060A000319681E693E024CA00D081E593E0EDB714
:1060B000FEB7928381830E94FC7D0F900F900E9417
:1060C000351A00D08DE493E0ADB7BEB712969C931D
:1060D0008E9311970E94FC7D0F900F9080E00E949C
:1060E0008C1B00D087E493E0EDB7FEB792838183E9
:1060F0000E94FC7D0F900F900E94A1108091691C5E
:1061000080FF05C081E061E041E00E94E1110E9452
:106110003A1A00D000D0EDB7FEB731968EE393E087
:10612000ADB7BEB712969C938E9311978091C7041A
:10613000828313820E94FC7DEDB7FEB7319681E326
:1061400093E0ADB7BEB712969C938E931197809152
:10615000E106828313820E94FC7D89E193E0EDB722
:10616000FEB79283818380E490E0948383830E94CE
:10617000FC7D00D0EDB7FEB7319686E093E0ADB779
:10618000BEB712969C938E9311978091E5248283DB
:1061900013828091E624848315820E94FC7D0F90F7
:1061A0000F9081EF92E0EDB7FEB7928381838091EB
:1061B000C3049091C404948383830E94FC7D00D027
:1061C0008DED92E0ADB7BEB712969C938E9311976A
:1061D0008091BF049091C004A091C104B091C20409
:1061E000EDB7FEB783839483A583B6830E94FC7DBD
:1061F0008DB79EB706960FB6F8949EBF0FBE8DBFA3
:1062000081E00E94741C0E94C10B00D000D000D01D
:1062100020ED32E0ADB7BEB712963C932E931197A6
:10622000EDB7FEB763837483858396830E94FC7DFC
:106230008DB79EB706960FB6F8949EBF0FBE8DBF62
:106240000E94F80B0E94D50B00D000D000D022ECA9
:1062500032E0ADB7BEB712963C932E931197EDB7CF
:10626000FEB763837483858396830E94FC7D8DB71C
:106270009EB706960FB6F8949EBF0FBE8DBF1D9BAE
:1062800003C083E093E002C08FEF92E000D000D023
:1062900026EB32E0ADB7BEB712963C932E93119722
:1062A00014969C938E9313970E94FC7D2091C0249A
:1062B0003091C1244091C2245091C3248091C424C0
:1062C0009091C524A091C624B091C72400D000D0DD
:1062D00000D00DB71EB70F5F1F4F68E972E0EDB732
:1062E000FEB772836183F80122833383448355832D
:1062F00086839783A087B1870E94FC7DEDB7FEB7A8
:10630000319686E792E0ADB7BEB712969C938E9316
:1063100011978091CD249091CE24A091CF24B0915B
:10632000D02482839383A483B5838091D1249091D8
:10633000D224A091D324B091D42486839783A087BC
:10634000B1870E94FC7DEDB7FEB738960FB6F89482
:10635000FEBF0FBEEDBF8CE692E0928381830E9468
:10636000FC7D8091C5040F900F9081FF0EC000D07E
:1063700086E692E0ADB7BEB712969C938E931197C6
:106380000E94FC7D0F900F9017C080FF03C08CEF20
:1063900092E002C08FEF92E000D000D022E632E01F
:1063A000EDB7FEB732832183948383830E94FC7D03
:1063B0000F900F900F900F908091C50483FF03C042
:1063C0008CEF92E002C08FEF92E000D000D02FE47B
:1063D00032E0ADB7BEB712963C932E931197149648
:1063E0009C938E9313970E94FC7D8091C50490919D
:1063F000C6040F900F900F900F9094FF03C08CEF86
:1064000092E002C08FEF92E000D000D022E432E0B0
:10641000EDB7FEB732832183948383830E94FC7D92
:106420008091DC069091DD0625E332E0ADB7BEB782
:1064300012963C932E93119714969C938E931397D8
:106440000E94FC7D0F900F900F900F90779903C0E2
:106450008CEF92E002C08FEF92E000D000D02CE2EF
:1064600032E0EDB7FEB732832183948383830E94A9
:10647000FC7D0F900F900F900F900E94C508209107
:10648000A804222309F465C100D000D0EDB7FEB7FF
:10649000319689E292E02CC80E94021B2091A80448
:1064A000222309F456C100D000D0EDB7FEB73196D3
:1064B00086E292E01DC80E94FE170097B9F500D051
:1064C00000D000D08BE192E0EDB7FEB792838183DC
:1064D0008091651890916618A0916718B09168181E
:1064E00083839483A583B6830E94FC7D8EE092E033
:1064F000ADB7BEB712969C938E9311978091E1240D
:106500009091E224A091E324B091E424EDB7FEB78A
:1065100083839483A583B6830E94FC7D8DB79EB749
:1065200006960FB6F8949EBF0FBE8DBF0E94D40C86
:106530002091A804222309F40CC100D000D0EDB7AB
:10654000FEB731968BE092E00C94782A83E061E00C
:1065500048E021E00E947B1300D000D000D084E00E
:1065600092E0EDB7FEB792838183809158189091A5
:106570005918A0915A18B0915B1883839483A5830E
:10658000B6830E94FC7D00D000D0EDB7FEB73196F7
:1065900083EF91E0ADB7BEB712969C938E9311979F
:1065A00080915C1890915D18A0915E18B0915F1871
:1065B00082839383A483B58380916018909161183E
:1065C000A0916218B091631886839783A087B187E2
:1065D0000E94FC7DEDB7FEB73A960FB6F894FEBF69
:1065E0000FBEEDBF0E94D40C2091A804222309F411
:1065F000B0C000D000D0EDB7FEB7319680EF91E08B
:106600000C94782A6091AD047091AE0480E090E023
:106610000E94667D6DE773E00E947B7D0097B1F478
:106620006091AD047091AE0480E090E00E94667DC0
:10663000009709F48EC00E945D7C803108F089C00B
:1066400090915201982B9093520183C080915201F6
:1066500000D000D028E336E0EDB7FEB732832183C7
:1066600090E08F709070948383830E94FC7D0F90E4
:106670000F900F900F900E94D40C6BC06091AD04EE
:106680007091AE0480E090E00E94667D8C016CEF1A
:1066900072E00E947B7D009749F40E94C75280916E
:1066A000C5049091C60490620C94B62AC8016FEF9D
:1066B00072E00E947B7D0097E9F4F8940E94D55225
:1066C00088E10FB6F89480936000109260000FBECE
:1066D00084B7877F84BF8091600088618093600069
:1066E0001092600078948091C5049091C6049F7DBB
:1066F0000C94B62AC80162E873E00E947B7D9C017D
:106700008091C5049091C6042115310521F495FFAF
:1067100020C0F894FFCF95FF03C08CEF92E002C039
:106720008FEF92E000D000D025E436E0ADB7BEB7E1
:1067300012963C932E93119714969C938E931397D5
:106740000E94FC7D0F900F900F900F9002C00E944E
:106750002219E981FA811182108283E00F900F9053
:10676000CF91DF911F910F91FF90EF90DF90CF902D
:10677000BF90AF909F908F907F906F905F904F9061
:106780003F902F900895F89491E2E0E0F0E090932C
:1067900057008491E2E0F0E0909357002491E4E008
:1067A000F0E090935700E49190E0A0E0B0E0DC01CD
:1067B0009927882730E040E050E0542F432F322FB4
:1067C0002227820F931FA41FB51F8E0F911DA11D9D
:1067D000B11D80931C1890931D18A0931E18B093A0
:1067E0001F1878940895DF93CF93CDB7DEB727971E
:1067F0000FB6F894DEBF0FBECDBFCE0104966EE09B
:1068000070E044E050E00E942E7F8C819D81AE813B
:10681000BF818F3F2FEF92072FEFA2072FEFB20715
:1068200049F48FEB94E06EE070E044E050E00E94A9
:106830004C7F08C08093BF049093C004A093C10410
:10684000B093C204CE01029662E170E042E050E0F3
:106850000E942E7F8A819B812FEF8F3F920779F4D0
:106860008CE390E09093C4048093C30483EC94E0A1
:1068700062E170E042E050E00E944C7F04C09093DF
:10688000C4048093C304CE01029664E170E042E048
:1068900050E00E942E7F8A819B812FEF8F3F9207CD
:1068A00079F48AE090E09093C6048093C50485EC67
:1068B00094E064E170E042E050E00E944C7F04C04C
:1068C0009093C6048093C504CE01029660E070E008
:1068D00042E050E00E942E7F8A819B812FEF8F3F04
:1068E000920769F41092DD061092DC068CED96E0BA
:1068F00060E070E042E050E00E944C7F04C0909362
:10690000DD068093DC0685ED94E268E170E049E005
:1069100050E00E942E7F0E94430ECE01049666E056
:1069200070E044E050E00E942E7F8C819D81AE811A
:10693000BF818F3F2FEF92072FEFA2072FEFB207F4
:1069400049F480EA94E066E070E044E050E00E94A0
:106950004C7F08C080EA94E066E070E044E050E0DC
:106960000E942E7FCE0104966AE070E044E050E081
:106970000E942E7F8C819D81AE81BF818F3F2FEF42
:1069800092072FEFA2072FEFB20749F484EA94E0B1
:106990006AE070E044E050E00E944C7F08C084EA66
:1069A00094E06AE070E044E050E00E942E7FCE0167
:1069B000049662E070E044E050E00E942E7F8C81FB
:1069C0009D81AE81BF818F3F2FEF92072FEFA207EE
:1069D0002FEFB20749F48CE994E062E070E044E004
:1069E00050E00E944C7F08C08CE994E062E070E0C7
:1069F00044E050E00E942E7FCE01019666E170E0F7
:106A000041E050E00E942E7F89818F3F49F481EE62
:106A100096E066E170E041E050E00E944C7F08C0E3
:106A200081EE96E066E170E041E050E00E942E7F4A
:106A3000CE01019667E170E041E050E00E942E7FB8
:106A400089818F3F49F487EC94E067E170E041E091
:106A500050E00E944C7F08C087EC94E067E170E052
:106A600041E050E00E942E7F27960FB6F894DEBFDB
:106A70000FBECDBFCF91DF9108950E94BB526C9A9B
:106A80006B9A6A9A6F9A729A749A739A779A8098A4
:106A900080B3897F80BB8398849887E080937E0051
:106AA000549A0E94C3330E94F33381E00E94E30AA8
:106AB00080E090E00E94570E0E94444C8091C504F3
:106AC00086FD239A0895CF93DF93EC018881998105
:106AD000009731F02AE08E39920709F099C08FC0F3
:106AE0000E943D358091C50480FD06C081FF02C033
:106AF0001D9902C00E94E553809170008C7F8093A5
:106B000070008091B60080628093B6001092B2004F
:106B100082E08093B1008091B60090E08770907021
:106B20000097C9F78091700081608093700080E0C9
:106B300090E06CEE78E00E949E520E94351A80E050
:106B40000E948C1B00D08AEE91E0ADB7BEB71296C2
:106B50009C938E9311970E94FC7D0F900F900E9442
:106B6000A1108091691C86FF02C00E94814D809116
:106B7000E10690E00E942C578091C70490E00E94AB
:106B8000A4550E94A15580930F078091C70490E0FF
:106B90000E94A45500D000D000D0EDB7FEB73196CA
:106BA00087E893E0ADB7BEB712969C938E9311978A
:106BB00080910F07828313828091E106848315827E
:106BC0000E94EA7D10920E0710920D07EDB7FEB7F6
:106BD00036960FB6F894FEBF0FBEEDBF84ED94E07D
:106BE0009093DF248093DE2483E290E09093060765
:106BF000809305078EE99AE0998388830DC06332FC
:106C000059F48DE097E060E070E00E94CD1FE6CF80
:106C10001982188283E001C081E0DF91CF9108954D
:106C20008536910564F12091DC063091DD0620FF68
:106C300010C000D000D029E933E0EDB7FEB73283B1
:106C40002183948383830E94EA7D0F900F900F909D
:106C50000F9080917B2090917C20A0917D20B0911D
:106C60007E200196A11DB11D80937B2090937C20F6
:106C7000A0937D20B0937E2021E030E002C020E090
:106C800030E0C90108954F925F926F927F928F9288
:106C90009F92AF92BF92CF92DF92EF92FF920F93AB
:106CA0001F93DF93CF93CDB7DEB7CB58D0400FB64D
:106CB000F894DEBF0FBECDBF2C01633871F48DEEAA
:106CC00096E0C557DF4F6883CB58D0400E94FB3E0B
:106CD000C557DF4F6881CB58D040D2012D913C91F0
:106CE0001197BAE021353B0709F4A6C7EAE022353F
:106CF0003E0748F42115310589F0F9E021353F07B9
:106D000009F0E6C716C04AE02236340709F4BAC7CC
:106D10005AE02936350709F0DBC7CCC78DEE96E07F
:106D200061E870E041E555E00E94E03E81E599E0D0
:106D30007EC7623109F0D2C78091C5049091C60424
:106D400091FDF4CF8091BF049091C004A091C10443
:106D5000B091C20497FD8C9A0E94F80B8091BF04F9
:106D60009091C004A091C104B091C20493FF02C0ED
:106D70000E94FE178091BF049091C004A091C104AD
:106D8000B091C20494FF0AC00E94C10B6093C82452
:106D90007093C9248093CA249093CB248091BF041C
:106DA00080FF5DC062E1C62ED12CCC0EDD1E00D06E
:106DB00000D000D0EDB7FEB73196ADB7BEB7129692
:106DC000DC92CE92119788E790E0938382838DEADC
:106DD00093E0958384830E945A7E082F192F55EDE6
:106DE000E52E54E2F52EEDB7FEB736960FB6F894C1
:106DF000FEBF0FBEEDBF48E7A42EB12C3FE8832EA7
:106E000032E0932ED7012D917D01EDB7FEB7389773
:106E10000FB6F894FEBF0FBEEDBF3196C601800FCE
:106E2000911FADB7BEB712969C938E931197B38204
:106E3000A28295828482268317820E945A7E080F3E
:106E4000191FEDB7FEB738960FB6F894FEBF0FBE08
:106E5000EDBFFDEDEF16F4E2FF06A1F602C000E083
:106E600010E08091BF0481FF6EC022E1C22ED12CC0
:106E7000CC0EDD1E00D000D000D0EDB7FEB73196AD
:106E8000C601800F911FADB7BEB712969C938E932B
:106E9000119788E790E09383828381EB93E0958359
:106EA00084830E945A7E080F191F7E010894E11CFA
:106EB000F11C80E1F70111928A95E9F72DB73EB7F1
:106EC0002A5F3F4F0FB6F8943EBF0FBE2DBF80EB39
:106ED00068E9A70128E00E94991199E0A92EB12C38
:106EE000AC0EBD1E88E7882E912CBFE86B2EB2E059
:106EF0007B2ED7012D917D01EDB7FEB738970FB6E8
:106F0000F894FEBF0FBEEDBF3196C601800F911FF2
:106F1000ADB7BEB712969C938E93119793828282DF
:106F200075826482268317820E945A7E080F191F79
:106F3000EDB7FEB738960FB6F894FEBF0FBEEDBFA3
:106F4000EA14FB04B1F68091BF049091C004A091B3
:106F5000C104B091C2040097A105B10581F12DB71C
:106F60003EB7285030400FB6F8943EBF0FBE2DBF3D
:106F7000EDB7FEB73196CE014296800F911FADB7A7
:106F8000BEB712969C938E93119788E790E09383F7
:106F9000828386EB93E0958384838091DF069091D2
:106FA000E006978386830E945A7E080F191FEDB76B
:106FB000FEB738960FB6F894FEBF0FBEEDBF8091B6
:106FC000BF0482FF50C089E290E06BE270E04AE2C9
:106FD00050E027E00E945A4985ED94E20E94CA4B96
:106FE0002DB73EB72A5030400FB6F8943EBF0FBEC3
:106FF0002DBFEDB6FEB60894E11CF11C9E012E5E7D
:107000003F4F200F311FADB7BEB712963C932E9362
:10701000119728E730E0F701338322832DEB33E02B
:10702000358324839C01B901882777FD8095982FAB
:107030000E94B87720E030E048EC52E40E944E779E
:10704000D70116966D937D938D939C9319970E940B
:107050005A7E080F191FEDB7FEB73A960FB6F8948F
:10706000FEBF0FBEEDBF8091BF0483FF56C089E213
:1070700090E06BE270E04AE250E026E00E945A495C
:1070800081E090E00E94480C8093E30684ED97E154
:107090000E94CA4B2DB73EB72A5030400FB6F89425
:1070A0003EBF0FBE2DBFEDB6FEB60894E11CF11C2D
:1070B0009E012E5E3F4F200F311FADB7BEB7129617
:1070C0003C932E93119728E730E0F7013383228316
:1070D00027EC33E0358324839C01B901882777FDB1
:1070E0008095982F0E94B87720E030E048EC52E479
:1070F0000E944E77D70116966D937D938D939C9346
:1071000019970E945A7E080F191FEDB7FEB73A96DD
:107110000FB6F894FEBF0FBEEDBF8091BF0484FF91
:1071200036C02DB73EB72A5030400FB6F8943EBF58
:107130000FBE2DBFEDB7FEB73196CE014296800F40
:10714000911FADB7BEB712969C938E93119788E7A7
:1071500090E09383828382ED93E095838483809192
:10716000A0179091A117A091A217B091A3178683A1
:107170009783A087B1870E945A7E080F191FEDB729
:10718000FEB73A960FB6F894FEBF0FBEEDBF8091E2
:10719000BF0485FF31C00E94D50B2DB73EB72A50E2
:1071A00030400FB6F8943EBF0FBE2DBFEDB7FEB70F
:1071B00031969E012E5E3F4F200F311FADB7BEB7F7
:1071C00012963C932E93119728E730E03383228365
:1071D00020EE33E03583248366837783808791872D
:1071E0000E945A7E080F191FEDB7FEB73A960FB6E8
:1071F000F894FEBF0FBEEDBF8091BF0486FF3AC07A
:10720000F8948091C0249091C124A091C224B0919F
:10721000C32478942DB73EB72A5030400FB6F89467
:107220003EBF0FBE2DBF4DB75EB74F5F5F4F9E0194
:107230002E5E3F4F200F311FEDB7FEB73283218303
:1072400028E730E0FA01338322832EEE33E03583E2
:10725000248386839783A087B1870E945A7E080F74
:10726000191F2DB73EB7265F3F4F0FB6F8943EBFAC
:107270000FBE2DBF8091BF0487FF92C08091C304D1
:107280009091C404009709F48BC0F894C090C02476
:10729000D090C124E090C224F090C32478948091CF
:1072A000CC179091CD17A091CE17B091CF17A70111
:1072B0009601281B390B4A0B5B0BCA01B9010E94CE
:1072C000B677862EA72E682EB92E6091C3047091D2
:1072D000C40480E090E00E94B6779B01AC01682D69
:1072E0007A2D862D9B2D0E944E775C014DB75EB79F
:1072F0004A5050400FB6F8945EBF0FBE4DBFEDB779
:10730000FEB73196CE014296800F911FADB7BEB742
:1073100012969C938E93119788E790E093838283D3
:1073200087EF93E095838483262F372F4A2D5B2D9B
:107330002683378340875187C557DF4F6883CB58F3
:10734000D040C657DF4F7883CA58D0400E945A7E3B
:10735000080F191FC557DF4F6881CB58D040C6575B
:10736000DF4F7881CA58D040862F972FAA2DBB2D8A
:107370008093CD249093CE24A093CF24B093D02497
:10738000C092CC17D092CD17E092CE17F092CF17C3
:10739000EDB7FEB73A960FB6F894FEBF0FBEEDBF3D
:1073A0008091BF049091C004A091C104B091C20427
:1073B00090FF40C0F8948091C4249091C524A0917E
:1073C000C624B091C72478942DB73EB72A503040D8
:1073D0000FB6F8943EBF0FBE2DBF4DB75EB74F5FDF
:1073E0005F4F9E012E5E3F4F200F311FEDB7FEB75E
:1073F0003283218328E730E0FA013383228324E0BB
:1074000034E03583248386839783A087B1870E94E5
:107410005A7E080F191F2DB73EB7265F3F4F0FB694
:10742000F8943EBF0FBE2DBFC8010E9410360097D2
:1074300009F07CCC8091BF049091C004A091C1045C
:10744000B091C20491FF92C08091C3049091C40492
:10745000009709F48BC0F894C090C424D090C52440
:10746000E090C624F090C72478948091D017909132
:10747000D117A091D217B091D317A7019601281B5D
:10748000390B4A0B5B0BCA01B9010E94B677862EF5
:10749000A72E682EB92E6091C3047091C40480E0B9
:1074A00090E00E94B6779B01AC01682D7A2D862D65
:1074B0009B2D0E944E775C014DB75EB74A505040FD
:1074C0000FB6F8945EBF0FBE4DBFEDB7FEB7319655
:1074D000CE014296800F911FADB7BEB712969C9316
:1074E0008E93119788E790E0938382838DE094E0F8
:1074F00095838483262F372F4A2D5B2D2683378350
:1075000040875187C557DF4F6883CB58D040C65757
:10751000DF4F7883CA58D0400E945A7E080F191F47
:10752000C557DF4F6881CB58D040C657DF4F7881B1
:10753000CA58D040862F972FAA2DBB2D8093D124D7
:107540009093D224A093D324B093D424C092D01784
:10755000D092D117E092D217F092D317EDB7FEB7C1
:107560003A960FB6F894FEBF0FBEEDBF8091BF04F0
:107570009091C004A091C104B091C20492FF3EC09A
:1075800080916B2090916C20A0916D20B0916E2025
:107590002DB73EB72A5030400FB6F8943EBF0FBE0D
:1075A0002DBF4DB75EB74F5F5F4F9E012E5E3F4FC1
:1075B000200F311FEDB7FEB73283218328E730E07B
:1075C000FA01338322832AE134E0358324838683DE
:1075D0009783A087B1870E945A7E080F191F2DB785
:1075E0003EB7265F3F4F0FB6F8943EBF0FBE2DBF8C
:1075F000C8010E941036009709F098CB8091BF0413
:107600009091C004A091C104B091C20493FF3CC00A
:107610004DB75EB74A5050400FB6F8945EBF0FBEEC
:107620004DBFEDB7FEB73196CE014296800F911F48
:10763000ADB7BEB712969C938E93119788E790E0F2
:107640009383828383E294E0958384838091651899
:1076500090916618A0916718B091681886839783F7
:10766000A087B1870E945A7E080F191FEDB7FEB799
:107670003A960FB6F894FEBF0FBEEDBFC8010E9448
:107680001036009709F052CB8091BF049091C0044E
:10769000A091C104B091C20494FF3CC02DB73EB785
:1076A0002A5030400FB6F8943EBF0FBE2DBFEDB745
:1076B000FEB73196CE014296800F911FADB7BEB78F
:1076C00012969C938E93119788E790E09383828320
:1076D0008EE294E0958384838091C8249091C9249C
:1076E000A091CA24B091CB2486839783A087B187C9
:1076F0000E945A7E080F191FEDB7FEB73A960FB6D3
:10770000F894FEBF0FBEEDBFC8010E94103600976F
:1077100009F00CCB8091BF049091C004A091C104EA
:10772000B091C20495FF48C081E00E94730B2DB751
:107730003EB72A5030400FB6F8943EBF0FBE2DBF63
:10774000EDB6FEB60894E11CF11C9E012E5E3F4F83
:10775000200F311FADB7BEB712963C932E931197F1
:1077600028E730E0F701338322832BE334E03583CD
:1077700024832091A0043091A1044091A20450914F
:10778000A3040E949478D70116966D937D938D93F0
:107790009C9319970E945A7E080F191FEDB7FEB7E8
:1077A0003A960FB6F894FEBF0FBEEDBFC8010E9417
:1077B0001036009709F0BACA8091BF049091C004B6
:1077C000A091C104B091C20496FF48C082E00E941B
:1077D000730B2DB73EB72A5030400FB6F8943EBF1A
:1077E0000FBE2DBFEDB6FEB60894E11CF11C9E0144
:1077F0002E5E3F4F200F311FADB7BEB712963C93A0
:107800002E93119728E730E0F7013383228328E491
:1078100034E0358324832091A4043091A504409161
:10782000A6045091A7040E949478D70116966D93F0
:107830007D938D939C9319970E945A7E080F191F70
:10784000EDB7FEB73A960FB6F894FEBF0FBEEDBF88
:10785000C8010E941036009709F068CA8091BF04E1
:107860009091C004A091C104B091C20497FF39C0A7
:1078700083E00E94730B2DB73EB72A5030400FB6FD
:10788000F8943EBF0FBE2DBFEDB7FEB731969E01F7
:107890002E5E3F4F200F311FADB7BEB712963C93FF
:1078A0002E93119728E730E03383228325E534E0D7
:1078B0003583248366837783808791870E945A7EED
:1078C000080F191F8C98EDB7FEB73A960FB6F894CB
:1078D000FEBF0FBEEDBFC8010E941036009709F031
:1078E00025CA8091BF049091C004A091C104B091B9
:1078F000C204A0FF06C083E061E046E020E00E94F1
:107900007B138091BF049091C004A091C104B091F9
:10791000C204A1FF06C083E061E046E021E00E94CE
:107920007B138091BF049091C004A091C104B091D9
:10793000C204A0FF3CC02DB73EB72A5030400FB65E
:10794000F8943EBF0FBE2DBFEDB7FEB73196CE0106
:107950004296800F911FADB7BEB712969C938E933F
:10796000119788E790E09383828382E694E0958381
:10797000848380915C1890915D18A0915E18B091FD
:107980005F1886839783A087B1870E945A7E080F6D
:10799000191FEDB7FEB73A960FB6F894FEBF0FBEAB
:1079A000EDBFC8010E941036009709F0BFC9809151
:1079B000BF049091C004A091C104B091C204A1FF82
:1079C0003CC02DB73EB72A5030400FB6F8943EBFAA
:1079D0000FBE2DBFEDB7FEB73196CE014296800F98
:1079E000911FADB7BEB712969C938E93119788E7FF
:1079F00090E0938382838AE694E0958384838091E8
:107A0000601890916118A0916218B09163188683F4
:107A10009783A087B1870E945A7E080F191FEDB780
:107A2000FEB73A960FB6F894FEBF0FBEEDBFC80181
:107A30000E941036009709F079C9779A8091DC0688
:107A40009091DD0693FD749A8091DC069091DD069D
:107A500082FD08C08091C50480FD04C081FF31C053
:107A60001D9B2FC000D000D085E794E0ADB7BEB716
:107A700012969C938E931197CE01429614969C93E6
:107A80008E9313970E94EA7D2091A8040F900F9087
:107A90000F900F902223A9F000D000D0EDB7FEB7D1
:107AA000319684EE91E0ADB7BEB712969C938E935B
:107AB0001197228313820E94FC7D0F900F900F90EC
:107AC0000F9080910007898BFE01E00FF11F128A51
:107AD0000F5F1F4F8091DC069091DD0680FF12C082
:107AE00000D000D08CE794E0EDB7FEB7928381839D
:107AF000C8010196948383830E94EA7D0F900F90C2
:107B00000F900F9068010894C11CD11CA1E1EA2ECE
:107B1000F12CEC0EFD1EC701B6010E945848809161
:107B2000C50482FF45C08FEA94E0B701A60120ECAE
:107B300030E20E94DD4C8091DC069091DD0692FFE0
:107B400037C0F0ECEF2EF0E2FF2EEDE8AE2EE4E0D1
:107B5000BE2ED7018D917D0100D000D0EDB7FEB7CC
:107B60003196ADB7BEB71296BC92AE921197828392
:107B700013820E94EA7D0F900F900F900F90B0ED4E
:107B8000EB16B0E2FB0629F78AE090E00E941C7E2B
:107B900000D000D082E994E0EDB7FEB792838183F4
:107BA000D482C3820E94EA7D0F900F900F900F90B5
:107BB0008091DC069091DD0682FD73980E948354CB
:107BC0008DEE96E00E94FE3E8091C5049091C60421
:107BD00090FF43C0E090C304F090C4040E94A155FC
:107BE000C82E1092C4041092C30489E190E00E9450
:107BF000B95524C07398809100078F5F8093000768
:107C0000898BB8016F5F7F4FCE0141960E94584823
:107C10008DEE96E00E94FE3E8091960E9091970E1A
:107C200065E840E050E00E94C44081E59AE0D2015E
:107C300011969C938E9352C000E010E02091C504F1
:107C40003091C60430FDD6CF8C2D90E00E94B955FE
:107C5000F092C404E092C304739A8091DF0690917D
:107C6000E006009711F00E94E553809100078F5FB6
:107C7000809300078091DC069091DD0682FF56C854
:107C8000739A54C888EF96E00E94A543009731F19B
:107C90000E9483548091C50487FD2B9888EF96E05D
:107CA00060E470E00E947A4389E69AE0F2019183F1
:107CB000808314C088EF96E00E94A543009771F07E
:107CC0000E94E5538091C50487FF30C82B9A2EC8C7
:107CD000D20111961C921E9283E001C081E0C5572B
:107CE000DF4F0FB6F894DEBF0FBECDBFCF91DF914F
:107CF0001F910F91FF90EF90DF90CF90BF90AF90CA
:107D00009F908F907F906F905F904F90089508950F
:107D1000FC01DB018C91808311968C9111978183FA
:107D20000895FC01DB0190818C91981741F421E0CA
:107D300030E0918111968C911197981711F020E005
:107D400030E0C9010895FC0180818093E5248181A0
:107D50008093E6240895DC011996ED91FC911A9721
:107D60000280F381E02D309709F009950895EF9294
:107D7000FF920F931F93DF93CF9300D0CDB7DEB761
:107D80008C0188E10E94D348BC017E010894E11C6B
:107D9000F11CC7010E94883ED8011996ED91FC9113
:107DA0001A970190F081E02DC801B70109950F9055
:107DB0000F90CF91DF911F910F91FF90EF90089559
:107DC000EF92FF920F931F93CF93DF93EC018B0100
:107DD0007A0141E655E00E940C3FFA86E986C80127
:107DE00065E675E00E946B3FDF91CF911F910F9187
:107DF000FF90EF9008950E94253F0895CF93DF9361
:107E0000EC0188E165EE74E20E94C948CE010E944F
:107E1000283FDF91CF910895EF92FF920F931F9328
:107E2000CF93DF93EC018B017A010E94443FF886E7
:107E3000EF82C80169E675E00E946B3FDF91CF9148
:107E40001F910F91FF90EF9008950E944D3F08956C
:107E50000E945A5A0895FC01A781B0852D913C914A
:107E6000F90109950895DC011796ED91FC91189799
:107E70000280F381E02D309709F00995089582E999
:107E80009EE00E94B7410895FC017383628382E9FA
:107E90009EE0BF010E9442420895BC0182E99EE03B
:107EA0000E9409420895CF93DF93EC0182E99EE09E
:107EB0000E94BB4108C0828193818C179D0739F0D5
:107EC000CF010E948142E82FF92F3097A1F7CF010F
:107ED000DF91CF9108950F931F93CF93DF938B0181
:107EE0000E94533FEC01009731F01D830C83C801C1
:107EF0000E94B25C8E83DF91CF911F910F91089504
:107F00001F93CF93DF93EC01162F888580FF1DC050
:107F1000EC81FD813097C9F0D093970EC093960EF7
:107F200082E08887CE0106960995992787FD90956E
:107F300002978230910510F0133829F4CE01BE016A
:107F40000E94A93F02C081E08887DF91CF911F91F5
:107F50000895CF92DF92EF92FF920F931F93CF93EA
:107F6000DF93EC017B01C090960ED090970E0091AC
:107F7000940E1091950EF80103C00190F081E02D50
:107F8000EC17FD0719F03097C1F746C0209709F4A8
:107F900043C08885882309F118860BC0C017D10714
:107FA00029F0C80167E8AE010E94803FF801008116
:107FB00011810115110591F7EC81FD81309769F070
:107FC000CE15DF0551F0D093970EC093960ECE01DB
:107FD000069663E840E050E00995E091940EF09138
:107FE000950ECE17DF0791F4888199819093950EB5
:107FF0008093940E0DC0808191818C179D0729F488
:10800000888199819183808303C0FC01309799F71F
:10801000D092970EC092960EDF91CF911F910F9143
:10802000FF90EF90DF90CF9008951F93CF93DF9351
:108030001092980EC091940ED091950E11E00EC042
:108040008985882341F018871986CE0162E840E0CF
:1080500050E00E94803F0990D881C02D209781F781
:10806000DF91CF911F9108958091430F982F9F5FCB
:108070009093430F08956091960E7091970E0E9411
:10808000A93F08958AE88093430F10929A0E1092A8
:10809000990E1092950E1092940E1092970E1092C7
:1080A000960E08958091980E882311F00E94154035
:1080B0007091990E772309F455C020919A0E30E003
:1080C000F901EE0FFF1FEE0FFF1FE20FF31FE55642
:1080D000F14F60816093420F418152815093410F73
:1080E0004093400F8381948190933F0F80933E0F84
:1080F0002F5F3F4F2F71307020939A0E7150709305
:10810000990E009741F58091940E9091950E18C0AC
:108110008091980E882311F00E9415404091400FE5
:108120005091410F80913C0F90913D0F6091420F13
:108130000E94803FE0913C0FF0913D0F8081918142
:1081400090933D0F80933C0F80913C0F90913D0F99
:108150000097F1F607C0613819F421E0FC0120878F
:108160000E94803F8091980E2091990E30E0280F58
:10817000311DC90108958091980E2091990E30E02B
:10818000280F311DC90108957091990E7032D9F0F0
:1081900020919A0E270F2F7120933B0F30E0F901A9
:1081A000EE0FFF1FEE0FFF1FE20FF31FE556F14F1B
:1081B000608352834183948383837F5F7093990E9E
:1081C00020E030E002C021E030E0C9010895CF9303
:1081D000DF93C091960ED091970E0E94803FD0936E
:1081E000970EC093960EDF91CF910895FC01AB01DD
:1081F0009091940E8091950E9C01A32FB22F03C0F5
:108200000D90BC91A02DAE17BF0791F01097C1F74C
:10821000309771F090838183F093950EE093940EE4
:1082200081E0808717821682CF0161E80E94E740D3
:108230000895FC01009741F080858150823020F440
:1082400081E081878093980E089521E030E0FC0161
:108250008085882311F420E030E0C9010895CF9390
:10826000DF93EC014A815B818C819D8160E070E04D
:108270000E94747D4A815B8188819981489F900129
:10828000499F300D589F300D11248E819F8160E0F1
:1082900070E0A9010E94747DDF91CF910895FC01E7
:1082A0008281938120E030E019C0A481B581A20FC2
:1082B000B31F4C91442381F481E08C934081518120
:1082C000249FC001259F900D349F900D112426817D
:1082D0003781280F391F07C02F5F3F4F28173907F5
:1082E00020F320E030E0C9010895FC0126813781A8
:1082F0004281538180E090E018C02617370781F44F
:10830000A481B581A80FB91F2C91121614F4215025
:108310002C930480F581E02DE80FF91F80810895EA
:10832000A081B1812A0F3B1F01968417950728F37E
:108330008FEF0895FC01CB01268137816217730707
:1083400090F0A081B18162817381A69FA001A79F57
:10835000500DB69F500D1124420F531F21E030E005
:108360008417950710F020E030E0C9010895FC0162
:10837000118210820895FC01808191810895FB0192
:1083800020813181FC01318320830895FC0120810B
:1083900031812115310511F407C09C01F90180815B
:1083A00091810097D1F702C020E030E0C901089523
:1083B000CF93DF93DC012D913C911197211531056D
:1083C000A9F0F90180819181009729F411961C92FE
:1083D0001E920EC0F90120813181D9018D919C91AD
:1083E00011970097B9F71182108202C020E030E0A7
:1083F000C901DF91CF910895DC01ED91FC911197B6
:10840000309729F08081918111969C938E93CF01B2
:108410000895CF93DF93FC01A081B1811097D9F02B
:10842000C0E0D0E016C0A617B70771F48D919C91FB
:108430001197209719F49183808302C099838883D0
:1084400011961C921E9207C0ED0198818981A92F77
:10845000B82F109741F7DF91CF9108950F931F9395
:10846000CF93DF938C01EB010E940942F8018081D8
:10847000918199838883D183C083DF91CF911F91AC
:108480000F910895EF92FF920F931F93CF93DF9375
:10849000EC017B010E940942F70111821082CE019A
:1084A0000E94C641FC01009719F4E882F98202C0DB
:1084B000F182E082DF91CF911F910F91FF90EF90B9
:1084C0000895DC01ED91FC91119720E030E005C0AA
:1084D0002F5F3F4F0190F081E02D3097C9F7C90120
:1084E0000895FB01309721F4BA010E942E420895AD
:1084F000DA018081918111969C938E935183408300
:108500000895009721F0FC012081318102C020E014
:1085100030E0C90108958091440F9091450F009774
:1085200029F41092470F1092460F08950E94475168
:10853000E091440FF091450F2281338140815181B8
:10854000240F351F281B390B0CC0428153816081D9
:108550007181460F571F481B590B4217530708F4E8
:108560009A010480F581E02D309779F7280F391FA3
:108570003093470F2093460F089587E795E00E94B8
:1085800019410895CF92DF92EF92FF920F931F93BC
:10859000CF93DF937C01FC0180819181009729F0CA
:1085A0008A35910509F06EC00BC01092450F1092EC
:1085B000440F8AE590E0F7019183808381E066C0F3
:1085C000673849F5CA01E091440FF091450F03C0A7
:1085D0000480F581E02D309741F3268137812817FB
:1085E0003907B1F3E093440FF093450F0FC016968F
:1085F0002D913C9117972817390739F414962D912E
:108600003C91159735832483DF01FD01A481B58159
:10861000109769F7CECF623861F6C091440FD091C0
:10862000450F00E010E02BC0CE010E94AA60009729
:10863000F1F08E819F8168E8AE010E94C4400097EE
:10864000A1F41F821E828C819D810115110521F0EC
:10865000F8019583848304C09093450F8093440F61
:108660001D821C820E948B42D8CF0E94BD428E0187
:108670009C818D81C92EE6016E01D82EE6012097DE
:1086800099F697CFF7011182108283E0DF91CF91A5
:108690001F910F91FF90EF90DF90CF900895CF93AF
:1086A000DF93EC010E94BD428E819F81009769F0AB
:1086B000E091440FF091450F06C0EC17FD07A9F0BB
:1086C0000480F581E02D3097C1F78091960E90914E
:1086D000970E9F838E838091440F9091450F9D83C9
:1086E0008C83D093450FC093440F0E948B42DF913F
:1086F000CF910895CF93DF93EC010E948A60CE0161
:108700000E944F43DF91CF910895CF93DF93EC0107
:108710000E949660CE010E944F43DF91CF91089551
:10872000CF93DF93EC010E94A060CE010E944F43E3
:10873000DF91CF910895FC0180819181860F971F71
:10874000918380830E948B42089521E030E0FC01F8
:1087500086819781009711F020E030E0C9010895EB
:10876000FC012281338180819181280F391FC90149
:108770000895FC0180819181089521E030E080918D
:10878000440F9091450F009711F420E030E0C901AB
:1087900008958091440F9091450F009729F0209102
:1087A000460F3091470F02C020E030E0C901089524
:1087B000CF93DF93EC01E091440FF091450F8E17BA
:1087C0009F0741F48C819D819093450F8093440FC6
:1087D00014C0FC01309731F0848195818C179D077E
:1087E000C1F707C01D821C821F821E82DF91CF91BC
:1087F00008958C819D81958384830E948B42F2CF62
:10880000CF92DF92EF92FF920F931F93CF93DF935C
:108810008C017A01FC0180819181009729F08B34D1
:10882000910509F051C01EC089E49FE00E94BB4140
:10883000C82EE6017E01F92EE70109C06C817D8119
:10884000CE0102960E947A430990D881C02D2097CC
:10885000A9F781E08093480F8BE490E0F8019183C1
:10886000808337C06838A9F589E49FE00E94BB4146
:10887000C82EE6016E01D92EE60123C0CE01029674
:10888000E816F906D9F489E49FE0BE010E94094286
:10889000E090960EF090970E8A859B859093970EA8
:1088A0008093960EEC85FD85309719F08E859F8517
:1088B0000995F092970EE092960ECECF0990D8814E
:1088C000C02D2097D9F6C8CFF8011182108283E01D
:1088D00001C081E0DF91CF911F910F91FF90EF9048
:1088E000DF90CF9008951092480F89E49FE00E9496
:1088F000B74180E995E060E070E00E94F64008959D
:108900000F931F93CF93DF93EC010091960E10917C
:10891000970E1B870A875D874C873F872E8780913C
:10892000480F882379F080E995E09093970E809323
:10893000960ECE0102960E947A431093970E0093F2
:10894000960E02C07D836C8389E49FE0BE010E9485
:10895000094289E49FE0BE010E944242DF91CF912B
:108960001F910F9108950F931F93CF93DF93EC0105
:108970008091480F882391F00091960E1091970EE8
:1089800080E995E09093970E8093960ECE01029623
:108990000E9485431093970E0093960E89E49FE002
:1089A000BE010E94094289E49FE0BE010E9442424A
:1089B000DF91CF911F910F9108950F931F93CF9344
:1089C000DF93EC018091480F882391F00091960E7F
:1089D0001091970E80E995E09093970E8093960EF4
:1089E000CE0102960E9490431093970E0093960E2C
:1089F00089E49FE0BE010E94094289E49FE0BE0134
:108A00000E944242DF91CF911F910F910895CF9321
:108A1000DF93EC018091480F882329F0CE01029664
:108A20000E94D84304C01F821E821986188689E4DA
:108A30009FE0BE010E940942DF91CF910895CF933C
:108A4000DF93EC018091480F882331F0CE0102962C
:108A50000E94A5439C0114C089E49FE00E94BB4191
:108A6000E82FF92F06C0EC17FD0741F00190F081C7
:108A7000E02D3097C1F721E030E002C020E030E087
:108A8000C901DF91CF9108950F931F930091E524C1
:108A90001091E6240E9474512DB73EB72255304004
:108AA0000FB6F8943EBF0FBE2DBFEDB7FEB731969F
:108AB00028E43EE0ADB7BEB712963C932E931197D3
:108AC000028313821483158266837783808791875C
:108AD0008091D8269091D926A091DA26B091DB26F4
:108AE00082879387A487B5878091DC269091DD26C5
:108AF000A091DE26B091DF2686879787A08BB18B69
:108B00008091E0269091E126A091E226B091E326A3
:108B1000828B938BA48BB58B8091E4269091E52674
:108B2000A091E626B091E726868B978BA08FB18F18
:108B30008091E8269091E926A091EA26B091EB2653
:108B4000828F938FA48FB58F8091EC269091ED2624
:108B5000A091EE26B091EF26868F978FA0A3B1A3A8
:108B60008091F0269091F126A091F226B091F32603
:108B700082A393A3A4A3B5A38091F4269091F52694
:108B8000A091F626B091F72686A397A3A0A7B1A738
:108B90008091F8269091F926A091FA26B091FB26B3
:108BA00082A793A7A4A7B5A78091FC269091FD2644
:108BB000A091FE26B091FF2686A797A7A0ABB1ABE8
:108BC0008091002790910127A0910227B09103275F
:108BD00082AB93ABA4ABB5AB8091042790910527F2
:108BE000A0910627B091072786AB97ABA0AFB1AF96
:108BF0008091082790910927A0910A27B0910B270F
:108C000082AF93AFA4AFB5AFEDB7FEB7FF9680913B
:108C10000C2790910D27A0910E27B0910F278083EC
:108C20009183A283B383EDB7FEB7ED5BFF4F8091D5
:108C3000102790911127A0911227B09113278083BC
:108C40009183A283B383EDB7FEB7E95BFF4F8091B9
:108C5000142790911527A0911627B091172780838C
:108C60009183A283B383EDB7FEB7E55BFF4F80919D
:108C7000182790911927A0911A27B0911B2780835C
:108C80009183A283B383EDB7FEB7E15BFF4F809181
:108C90001C2790911D27A0911E27B0911F2780832C
:108CA0009183A283B3830E94FC7D0091E5241091FF
:108CB000E6242DB73EB72E5A3F4F0FB6F8943EBF6D
:108CC0000FBE2DBF0E947451ADB7BEB7D2970FB67D
:108CD000F894BEBF0FBEADBFEDB7FEB7319629ED1C
:108CE0003DE012963C932E931197028313821483D6
:108CF0001582668377838087918780912027909162
:108D00002127A0912227B091232782879387A487C8
:108D1000B5878091242790912527A0912627B0918F
:108D2000272786879787A08BB18B809128279091E2
:108D30002927A0912A27B0912B27828B938BA48B74
:108D4000B58B80912C2790912D27A0912E27B09143
:108D50002F27868B978BA08FB18F80913027909192
:108D60003127A0913227B0913327828F938FA48F20
:108D7000B58F8091342790913527A0913627B091F7
:108D80003727868F978FA0A3B1A380913827909122
:108D90003927A0913A27B0913B2782A393A3A4A39C
:108DA000B5A380913C2790913D27A0913E27B0919B
:108DB0003F2786A397A3A0A7B1A7809148279091AA
:108DC0004927A0914A27B0914B2782A793A7A4A730
:108DD000B5A780914C2790914D27A0914E27B09137
:108DE0004F2786A797A7A0ABB1AB0E94FC7D2DB7FC
:108DF0003EB72E5C3F4F0FB6F8943EBF0FBE2DBF5F
:108E00001F910F91089580E380934B0F0895EF9287
:108E1000FF92CF93DF9320914B0F30E0C0E3D0E07F
:108E2000C21BD30B205B304FB901AE010E946B7D9A
:108E3000CE01DF91CF91FF90EF900895AF92BF9256
:108E4000CF92DF92EF92FF920F931F93CF93DF9316
:108E50007C01C0904C0FD0904D0F20914B0F30E013
:108E60008601005D1F4F021B130B01381105E0F452
:108E7000C0E3D0E0C21BD30B205B304FB901AE0181
:108E80000E946B7DCE0DDF1D20914E0F30914F0F54
:108E90008091021090910310280F391FCE01B90163
:108EA000A6010E946B7D02C000E010E0C801DF91C6
:108EB000CF911F910F91FF90EF90DF90CF90BF90D7
:108EC000AF90089590914B0F980F90934B0F08958A
:108ED00040914C0F50914D0F9C014817590798F045
:108EE0008091021090910310820F931F90930310B2
:108EF00080930210421B530B50934D0F40934C0F25
:108F000021E030E002C020E030E0C90108959093F4
:108F10004D0F80934C0F0895209102103091031053
:108F20002058304FC901089520914B0F30E0205B4D
:108F3000304FC901089521E030E080914E0F9091AB
:108F40004F0F4FE08038940711F420E030E0C90162
:108F500008950E949B47009771F020E83FE06091E0
:108F60004E0F70914F0F40914C0F50914D0FC90112
:108F70000E946B7D0895A0910210B091031010978C
:108F8000B9F020914C0F30914D0F205D3F4FA0580C
:108F9000B04FE0E8FFE080E390E003C04D914193E3
:108FA000019682179307D4F31092031010920210C7
:108FB000089580914E0F90914F0F089580914C0F1E
:108FC00090914D0F089590914B0F80E3891B089568
:108FD00080E390914B0F891B20914C0F30914D0FE6
:108FE000280F311DC90108951F93CF93DF93EC0122
:108FF00010914B0F812F90E08C179D076CF00E9411
:10900000E8478C0F9D1F8138910530F41C1B10938D
:109010004B0F21E030E002C020E030E0C901DF91D9
:10902000CF911F910895CF93DF93EFEEF4E2119269
:10903000119285E2EF31F807D1F7C0E0D0E0CE0120
:10904000880F991F89519B4D6FE575E00E94883EFE
:109050002196C430D10599F7DF91CF9108951092F0
:1090600003101092021010924D0F10924C0F80E3DB
:1090700080934B0F80E89FE090934F0F80934E0FAB
:109080000E94134808950F931F93CF93DF93EC0131
:109090008B010E942F48D0934F0FC0934E0F109317
:1090A0004D0F00934C0FDF91CF911F910F910895B9
:1090B000CF92DF92EF92FF920F931F93DF93CF93A4
:1090C00000D0CDB7DEB78C0169837A830E942F4828
:1090D00069817A81C62ED72E21E8C216D10418F0F4
:1090E00030E8C32ED12C80914E0F90914F0FB801D4
:1090F000A6010E946B7DD0924D0FC0924C0FC6010D
:109100000F900F90CF91DF911F910F91FF90EF90F3
:10911000DF90CF900895282F392FD901EFEEF4E298
:1091200080E301900D928150E1F7862F972FDC01AB
:10913000E7EEF4E288E001900D928150E1F70895A6
:10914000EFEEF4E2282F392FD90180E30D90019240
:109150008150E1F7A7EEB4E2862F972FFC0188E05B
:1091600001900D928150E1F70895E82FF0E0EE0FA5
:10917000FF1FE151FB4D7183608381E090E0089512
:10918000E82FF0E0EE0FFF1FE151FB4D8081918150
:10919000089590E0880F991F89549B4D0E94883E46
:1091A00081E090E00895282F30E0220F331F2954EA
:1091B0003B4DC90108958115910511F00197F1F713
:1091C0000895E0912225F091232590818091212519
:1091D00089230895E0911F25F091202580819091A9
:1091E0002125892B8083E0912425F09125258081FC
:1091F00090912125892B80830895E0911F25F0917E
:109200002025908180912125809589238083E0917C
:109210002425F09125259081809121258095892311
:1092200080830895FF920F931F93E0911F25F09183
:109230002025908180912125809589238083E0914C
:109240002425F0912525808190912125892B8083EB
:109250008FEB93E00E94DB48FFB6F894E091242561
:10926000F091252590818091212580958923808307
:1092700083E890E00E94DB48E0912225F0912325CD
:10928000008110912125FFBE78948BE393E00E942A
:10929000DB48E0912225F0912325808190912125C2
:1092A000892319F0802F812301C081E01F910F9144
:1092B000FF900895509325254093242570932025F1
:1092C00060931F25909323258093222581E090E0D1
:1092D00002C0880F991F2A95E2F7809321250E94EA
:1092E000124908950F931F93182F0FB7F894E09128
:1092F0002425F0912525808190912125892B80833B
:1093000083E090E00E94DB48112351F0E091242596
:10931000F091252590818091212580958923808356
:1093200087E190E00E94DB48E0912225F09123251F
:10933000808190912125892309F410E089E590E04E
:109340000E94DB48E0912425F091252590818091B1
:1093500021258095892380830FBF8BE390E00E94B5
:10936000DB48812F1F910F9108950F931F93182FA2
:1093700008E0812F81700E94724916958111106852
:109380000150B9F7812F1F910F9108958FEF0E941F
:10939000B5490895DF92EF92FF920F931F93CF93F9
:1093A000DF93182FEB010E941249882389F580EF83
:1093B0000E94B549EE2400E498EFD92ED00E81E04A
:1093C0000E947249F82E81E00E947249882319F0A8
:1093D000FF2069F020C0FF2051F4011728F0888198
:1093E00080FF05C0101719F0E02EFF24F3948F2D95
:1093F0000E947249888186958883FF2011F08068D9
:10940000888301500D15D9F6002339F02196D4CF69
:10941000EE24EA9402C08EEFE82E8E2DDF91CF91DC
:109420001F910F91FF90EF90DF9008950F931F937E
:10943000CF93DF93182FEB010E941249209751F030
:1094400085E50E94B54908E089910E94B54901501F
:10945000D9F703C08CEC0E94B549812F0E94B54911
:10946000DF91CF911F910F9108950F931F93CF9389
:10947000DF93FB01DA01E801408150E0718160E097
:10948000462B572B803171F4BA016E7F13E0660FC3
:10949000771F1A95E1F796814CE050E0491B51097E
:1094A000460F571F57FF06C091E09C93509541957A
:1094B0005F4F01C01C92883289F4848190E0BC0126
:1094C000607670706036710549F086FF02C04E7F8D
:1094D00005C085FF02C04C7F01C0487FCA0154E02F
:1094E000969587955A95E1F7F90180834F704883E7
:1094F00080E0DF91CF911F910F9108950F931F93FB
:10950000CF93DF938C01EB01F8018081BE010E94B3
:10951000CA49F801808381508D3F28F488818832C0
:1095200011F0803189F7DF91CF911F910F9108954C
:109530001F93CF93DF93EC010E94124984EBBE018D
:109540000E94164A81E00E947249182F0E94124917
:1095500081E0112309F480E0DF91CF911F910895FC
:109560001F93CF93DF93182FEB010E9412490E94A3
:10957000E148882349F084E4BE010E94164A113074
:1095800029F00E94EA4802C082E001C080E0DF9139
:10959000CF911F9108956F927F928F929F92AF9279
:1095A000BF92CF92DF92EF92FF920F931F93DF93C0
:1095B000CF93CDB7DEB729970FB6F894DEBF0FBEB5
:1095C000CDBF7C014B013A0159010E9412498EEB3B
:1095D000B7010E94164A8E010F5F1F4F8AE0C82E06
:1095E000D12CCC0EDD1E0E94C649F80181938F015B
:1095F000EC15FD05C1F78E010F5F1F4FC80169E033
:1096000070E00E945B65882351F4F7018081B80106
:10961000A401930185010E94354A80E001C083E0E6
:1096200029960FB6F894DEBF0FBECDBFCF91DF9164
:109630001F910F91FF90EF90DF90CF90BF90AF9070
:109640009F908F907F906F9008957F928F929F92BE
:10965000AF92BF92CF92DF92EF92FF920F931F9340
:10966000DF93CF93CDB7DEB729970FB6F894DEBF5F
:109670000FBECDBF782E5B014A0179018EEB60E011
:1096800070E00E94164A8E010F5F1F4F9AE0C92EAC
:10969000D12CCC0EDD1E0E94C649F80181938F01AA
:1096A000EC15FD05C1F78E010F5F1F4FC80169E082
:1096B00070E00E945B65882349F4872DB801A501FD
:1096C000940187010E94354A80E001C083E0299619
:1096D0000FB6F894DEBF0FBECDBFCF91DF911F91C3
:1096E0000F91FF90EF90DF90CF90BF90AF909F9041
:1096F0008F907F9008950F931F93DF93CF93CDB7F3
:10970000DEB728970FB6F894DEBF0FBECDBF182F77
:10971000062FDE011196E2EAF5E088E001900D9255
:109720008150E1F7242F332727FD309541E752E0A0
:10973000249FC001259F900D349F900D112464E655
:1097400070E00E94667AAB0164E6069FB0011124C6
:10975000460F571FFE013196CE010996619170E0C8
:109760002617370719F44F5F5F4F03C0E817F90753
:10977000A9F7112319F0509541955F4FCA0128961A
:109780000FB6F894DEBF0FBECDBFCF91DF911F9112
:109790000F9108950F931F93DF93CF93CDB7DEB74B
:1097A0002B970FB6F894DEBF0FBECDBF182F092F31
:1097B000885F612F792F0E94B04A882309F049C041
:1097C00066E471E48FE090E00E94374C812F902F87
:1097D000BE016F5F7F4FAE014E5F5F4F9E012D5FF9
:1097E0003F4F0E94CB4A8823A1F5DE011496EAE997
:1097F000F5E088E001900D928150E1F74B81642FF4
:1098000070E021E732E0629FC001639F900D729F7C
:10981000900D112464E670E00E94667A9A8184E6D5
:10982000989FC0011124680F791FFE013496CE0164
:109830000C962191421719F46F5F7F4F03C0E81710
:10984000F907B9F78981882331F0709561957F4FC9
:1098500002C064E371E2CB012B960FB6F894DEBF31
:109860000FBECDBFCF91DF911F910F910895DC0105
:10987000CB0181159105A105B10529F081509040DA
:10988000A040B040D9F708951092B90080E28093CB
:10989000B800089594EA9093BC0020EA36E841E0CD
:1098A00050E005C02150304040405040F1F09091D0
:1098B000BC0097FFF7CF1DC09031B9F48093BB0077
:1098C00084E88093BC0080EA96E8A1E0B0E004C0A0
:1098D0000197A109B10959F02091BC0027FFF8CFE9
:1098E0000EC081E0903421F40FC081E0089581E042
:1098F00008959091B900987F9830F1F6DFCF90915C
:10990000B900987F983169F780E0089544EA34E817
:1099100024E94093BC009091BC0097FFFCCF90914C
:10992000B900987F983011F0903199F78093BB007F
:109930003093BC009091BC0097FFFCCF9091B90090
:10994000987F903211F0983539F42093BC009091B3
:10995000BC0094FDFCCFDDCF08950E944A4C0895D1
:1099600084E98093BC008091BC0084FDFCCF089505
:109970008093BB0084E88093BC008091BC0087FF8B
:10998000FCCF9091B900987F81E0983209F480E093
:10999000089584EC8093BC008091BC0087FFFCCFCD
:1099A0008091BB00089584E88093BC008091BC0046
:1099B00087FFFCCF8091BB000895E82FF92F80E14D
:1099C000919190933F018150D9F780913C018F7D17
:1099D00080933C0180913C01877F80933C01862FDE
:1099E000972FFC0180E1919190933E018150D9F72E
:1099F00080913C01806880933C0180913D0180FF13
:109A0000FCCF4051504080913C01806280933C01EA
:109A100080913C01877F80933C0114C0862F972F53
:109A2000FC0180E1919190933E018150D9F78091A2
:109A30003C01806880933C0180913D0180FFFCCF18
:109A400040515040141615064CF3822F932FFC0101
:109A500080E190913E0191938150D9F781E090E0AF
:109A600008950F931F93CF93DF938C018CE70E948F
:109A7000864C8CE70E94B84CC0E0D0E0F8018191A0
:109A80008F010E94B84C2196C031D105B9F70E94D0
:109A9000B04CDF91CF911F910F910895813039F42F
:109AA0008CE790E060E070E040E050E006C08CE7BA
:109AB00090E060E070E040EC50E00E948111089579
:109AC000813039F48CE790E060E070E04EE050E0E7
:109AD00006C08CE790E060E070E048E050E00E9453
:109AE000811108958CE790E060E070E041E050E083
:109AF0000E9481116AE67AE080E090E00E94374C93
:109B000008958CE790E060E070E048E350E00E9448
:109B100081118CE790E060E070E049E350E00E9442
:109B200081118CE790E060E070E044E150E00E9439
:109B300081118CE790E060E070E048E750E00E941F
:109B400081118CE790E060E070E04EE550E00E940B
:109B500081118CE790E060E070E04DE650E00E94FB
:109B600081116CE17AE186E090E00E94374C8CE74D
:109B700090E060E070E04CE050E00E9481118CE7E2
:109B800090E060E070E041E050E00E9481118CE7DD
:109B900090E060E070E046E050E00E9481116AE6EB
:109BA0007AE080E090E00E94374C0895DF93CF93F5
:109BB000CDB7DEB7A2970FB6F894DEBF0FBECDBF0C
:109BC000DE011196EAEAF5E081E101900D92815003
:109BD000E1F7DE015296EBEBF5E081E101900D92A9
:109BE0008150E1F70E94814DCE0101960E94314DD6
:109BF00082E00E944E4D6AE67AE080E090E00E94AA
:109C0000374CCE0142960E94314D60E17EEA88E2F7
:109C100090E00E94374C80E00E94604D60E17EEA57
:109C200088E290E00E94374C81E00E94604DA2964D
:109C30000FB6F894DEBF0FBECDBFCF91DF91089570
:109C4000E6E4F1E0808120819081308182958695E3
:109C50008695837022952F70822B832B92959F700F
:109C6000892B0895DF92EF92FF920F931F93DF935A
:109C7000CF9300D0CDB7DEB780E06CE046E00E9425
:109C8000085289E18093C4001092C50082E080935D
:109C9000C00080E00E94B2520E94375184B784B75E
:109CA00084B784B784B7E6EAFDE222E432E4318384
:109CB00020833A968DB79EB70A97E817F907B8F34D
:109CC00000D000D085E99FE0ADB7BEB712969C9357
:109CD0008E9311978CEC95E014969C938E9313972A
:109CE0000E94FC7D0F900F900F900F900E94746166
:109CF0000E94424087E795E060E070E00E94F640F5
:109D00000E947344E0911706F091180609950E948D
:109D1000204E90E00E94B261CE0101960E946550F3
:109D2000882359F000D085E79FE0EDB7FEB7928316
:109D300081830E94FC7D0F900F908E010F5F1F4F5B
:109D4000C8010E94A33E0E946F507C010E94745083
:109D5000BC01C701A8010E94BF550E94CD4F0E94BF
:109D6000A4550E9479500E942C5700D088E69FE0AD
:109D7000ADB7BEB712969C938E9311970E94FC7D4F
:109D800000D0EDB7FEB7319604E61FE0ADB7BEB721
:109D900012961C930E9311978A81828313820E94DC
:109DA000FC7DEDB7FEB73196ADB7BEB712961C93EA
:109DB0000E9311978981828313820E94FC7D0F90FC
:109DC0000F9082E69FE0EDB7FEB7928381830E94F9
:109DD000FC7D0F900F900E94B861E0919A06F0917F
:109DE0009B060995E0918106F09182060995E09124
:109DF0004306F09144060995E0907F06F0908006B6
:109E000000919806109199060E94A155D82E0E94A3
:109E100034572DB73EB72A5030400FB6F8943EBFA6
:109E20000FBE2DBFEDB7FEB7319627E43FE0ADB7CB
:109E3000BEB712963C932E931197F382E28215835C
:109E40000483D6821782808711860E94FC7DE09170
:109E5000A406F091A5062DB73EB7265F3F4F0FB67B
:109E6000F8943EBF0FBE2DBF3097D1F00995BC01CD
:109E700000D000D084E39FE0ADB7BEB712969C93AC
:109E80008E93119780E890E00E94527AEDB7FEB76A
:109E9000748363830E94FC7D0F900F900F900F904E
:109EA00000D082E39FE0ADB7BEB712969C938E932D
:109EB00011970E94FC7D0F900F9083EC96E060E07C
:109EC00070E00E94F64085E495E00E945E6000D05C
:109ED0008AE29FE0EDB7FEB7928381830E94FC7D0A
:109EE0000F900F900F900F90CF91DF911F910F91D6
:109EF000FF90EF90DF900895EF92FF920F931F93E2
:109F000080E880936100109261000E94324E0E94AE
:109F100052400E94D3528091262590912725009788
:109F200029F001979093272580932625E0902825F6
:109F3000F090292500912A2510912B250E9474511B
:109F4000E616F7060807190711F30E94745160938B
:109F500028257093292580932A2590932B25D7CFE8
:109F600000D000D000D0EDB7FEB7319624E23FE03C
:109F7000ADB7BEB712963C932E931197938382830D
:109F8000758364830E94FC7D8DB79EB706960FB6DD
:109F9000F8949EBF0FBE8DBF08950F931F93DF935C
:109FA000CF93CDB7DEB7A2970FB6F894DEBF0FBE42
:109FB000CDBF83E490E00E94467F89839A83982FE7
:109FC0009B50903108F08A839A819095891709F403
:109FD00070C000D080ED9FE0ADB7BEB712969C93E5
:109FE0008E9311970E94FC7D8E010D5F1F4F0F9085
:109FF0000F90D80180E090E0FC01E055F04FE49133
:10A00000ED93019688309105B9F7F894CE01039647
:10A0100061E270E048E050E00E944C7FD80180E0AF
:10A0200090E0FC01E854F04FE491ED9301968E30FE
:10A030009105B9F7CE01039669E270E04EE050E079
:10A040000E944C7F80E090E0FC01EA53F04FE491E5
:10A05000D801ED938D0101968A309105A9F7CE01C3
:10A06000039667E370E04AE050E00E944C7F85E48D
:10A0700090E06DEC7BEA0E94647F87E490E060E012
:10A0800070E00E94647F89E490E060E00E94567F67
:10A0900081E490E060E070E00E94647F8AE189835F
:10A0A00085EE8A8369817A8183E490E00E94647FEF
:10A0B00078948981A2960FB6F894DEBF0FBECDBF0B
:10A0C000CF91DF911F910F910895F89461E270E0B4
:10A0D00042E050E00E942E7F789480E0089585E46D
:10A0E00090E00E94467F089587E490E00E94467FBA
:10A0F000089589E490E00E943E7F089520913425E0
:10A1000030913525409136255091372590E0A0E0DB
:10A11000B0E0280F391F4A1F5B1F2093342530936E
:10A1200035254093362550933725209130253091A1
:10A1300031254091322550913325280F391F4A1F70
:10A140005B1F209330253093312540933225509367
:10A1500033252091D4262223A1F020912C25309163
:10A160002D2540912E2550912F25280F391F4A1F4C
:10A170005B1F20932C2530932D2540932E25509343
:10A180002F2508951F920F920FB60F920BB60F92C4
:10A1900011242F933F934F935F936F937F938F93EC
:10A1A0009F93AF93BF93EF93FF938091041090918F
:10A1B000051001969093051080930410809106106D
:10A1C0008F5F80930610809106108038A9F410925A
:10A1D00006108091342590913525A0913625B091B7
:10A1E00037250196A11DB11D809334259093352507
:10A1F000A0933625B09337258091D4268823F1F09B
:10A20000809107108F5F809307108091071080382E
:10A21000A9F41092071080912C2590912D25A091E2
:10A220002E25B0912F250196A11DB11D80932C25BF
:10A2300090932D25A0932E25B0932F250E94BD43EA
:10A24000009711F00E94BD42FF91EF91BF91AF9135
:10A250009F918F917F916F915F914F913F912F913E
:10A260000F900BBE0F900FBE0F901F901895F89493
:10A270001092B60016BC83EF87BD82E084BD94E0E7
:10A2800095BD95B395BB80936E0078940895209109
:10A29000041030910510809104109091051028173A
:10A2A0003907A9F7C901089507C022E330E000008B
:10A2B00021503040E1F701970097B9F708950F93C7
:10A2C0001F93CF93DF938C010E944751EC010E94B2
:10A2D00047518C1B9D0B80179107C8F3DF91CF91DD
:10A2E0001F910F91089508952091342530913525BF
:10A2F0004091362550913725809134259091352510
:10A30000A0913625B0913725281739074A075B07F2
:10A3100059F7B901CA0108951F920F920FB60F9213
:10A3200011241092F0050F900FBE0F901F901895FA
:10A330001F920F920FB60F920BB60F9211242F930C
:10A340003F934F935F936F937F938F939F93AF93BD
:10A35000BF93EF93FF93E091E605F091E7058081CD
:10A36000E091F105F091F205309709F00995FF9120
:10A37000EF91BF91AF919F918F917F916F915F917D
:10A380004F913F912F910F900BBE0F900FBE0F90EA
:10A390001F9018951F920F920FB60F9211241092D2
:10A3A000FD050F900FBE0F901F9018951F920F92F2
:10A3B0000FB60F920BB60F9211242F933F934F932A
:10A3C0005F936F937F938F939F93AF93BF93EF931D
:10A3D000FF93E091F305F091F4058081E091FE0593
:10A3E000F091FF05309709F00995FF91EF91BF912A
:10A3F000AF919F918F917F916F915F914F913F911D
:10A400002F910F900BBE0F900FBE0F901F901895BD
:10A4100090E02DE030E0829FF001839FF00D929F4D
:10A42000F00D1124EA51FA4FA281B3811C92A4814C
:10A43000B5816C93A681B78188ED8C93A085B18599
:10A440004C93128614861386089590E02DE030E038
:10A45000829FF001839FF00D929FF00D1124EA512D
:10A46000FA4F81E08287A081B1816C933A96808116
:10A470008823E9F708951F93182F8A3031F48091CB
:10A4800008106DE00E94255202C08D3029F08091A5
:10A490000810612F0E94255280E090E01F910895DE
:10A4A000EF92FF921F93CF93DF93182FE62EE701D1
:10A4B0007E01F72EE7010CC08A3021F4812F6DE078
:10A4C0000E94255269916D3019F0812F0E9425520A
:10A4D0008881882389F7DF91CF911F91FF90EF90BA
:10A4E00008950F931F93DF93CF93CDB7DEB7FE018F
:10A4F0003A9609E010E1C80160E470E048855985AA
:10A500009F010E94987E8F81B8010E945052CF9186
:10A51000DF911F910F9108951F93CF93DF93182F11
:10A52000EB0104C0812F0E9425522196FE01649107
:10A530006623C1F7DF91CF911F91089590E02DE040
:10A5400030E0829FF001839FF00D929FF00D112467
:10A55000EA51FA4F748763870895682F80E00E945C
:10A56000255208958093081088ED95E09093A12DD1
:10A570008093A02D089584B7877F84BF88E10FB6AC
:10A58000F89480936000109260000FBE08952FE051
:10A5900088E190E00FB6F894A895809360000FBE14
:10A5A000209360000895A895089588E10FB6F89467
:10A5B00080936000109260000FBE0895F89428E028
:10A5C00088E190E00FB6F894A895809360000FBEE4
:10A5D00020936000FFCF8091472590E0FC01EE0FB3
:10A5E000FF1F9695982F882797958795E80FF91F55
:10A5F000E85BFA4D1082089580913F2580913F25B8
:10A6000090E008958091390181FD0CC081E491E0D2
:10A610006FE140E00E94D558813039F021E030E010
:10A62000813129F020E030E002C021E030E0C901B2
:10A6300008958091390181FD12C081E491E06FE1BC
:10A6400040E00E94D558982F8151823050F09F31C0
:10A6500041F0913041F081E0923031F402C081E06C
:10A66000089580E0089580E008950E94195388239A
:10A67000E1F3089581E491E06FE140E00E94D55854
:10A680000895E9E3F1E0808180818D7F80838DE012
:10A6900090E00197F1F782E491E06FE140E023E080
:10A6A0000E94DF5883E090E00197F1F708950E943F
:10A6B00035531092D4260E94415380913901826013
:10A6C00080933901809157278823E9F18091940084
:10A6D0009091950020916827309169278217930700
:10A6E000A0F48091342790913527A0913627B0911E
:10A6F00037278C57914EAF4FBF4F8093342790939D
:10A700003527A0933627B0933727809194009091F6
:10A710009500821B930BA0E0B0E02091342730918C
:10A7200035274091362750913727820F931FA41F5A
:10A73000B51F8093342790933527A0933627B09385
:10A74000372710925727809159278823E9F1809164
:10A7500094009091950020916C2730916D2782177D
:10A760009307A0F480913C2790913D27A0913E272C
:10A77000B0913F278C57914EAF4FBF4F80933C27EE
:10A7800090933D27A0933E27B0933F27809194005C
:10A7900090919500821B930BA0E0B0E020913C27A4
:10A7A00030913D2740913E2750913F27820F931FC4
:10A7B000A41FB51F80933C2790933D27A0933E276D
:10A7C000B0933F271092592708958091D42688236B
:10A7D00081F080914910882321F40E941953882325
:10A7E00031F481E08093CC1021E030E004C00E947D
:10A7F000575320E030E0C90108950F931F93182F9D
:10A80000883049F0863039F0893029F0863119F0E6
:10A81000893109F041C08091390181FD40C00E9419
:10A8200035530E943A53082F181709F43BC01830CB
:10A8300019F40E94415329C0193141F48631A9F419
:10A8400082E491E06FE140E029E009C0163169F44B
:10A85000893159F482E491E06FE140E026E00E9402
:10A86000DF58E3E0F0E03197F1F782E491E06FE147
:10A8700040E0212F0E94DF58083019F4E9E6F1E0AA
:10A8800002C0E3E0F0E03197F1F70E943A538117FC
:10A8900049F023E430E008C022E430E005C024E4BD
:10A8A00030E002C020E430E0C9011F910F9108950B
:10A8B000809194009091950090936D2780936C27E0
:10A8C00021E0209359278091390181FF15C0209301
:10A8D000D32680919400909195009093692780935E
:10A8E000682720935727809139018D7F8093390104
:10A8F0008091D3268823E1F786E10E94FD5381E011
:10A900008093D42608958091D426882351F4809191
:10A910004910882321F081E08093CB1002C00E946F
:10A92000585481E090E008951F93DF93CF930F92E6
:10A93000CDB7DEB78FB7898380914910882331F571
:10A94000F8948091D426882351F08091390181FDBB
:10A950001BC00E9419538823B9F080E003C00E94F5
:10A96000835481E0909147019E3010F010E001C0C7
:10A970001FEF882311F00E94E55316FF05C089815F
:10A980008FBF21E030E004C089818FBF20E030E03C
:10A99000C9010F90CF91DF911F9108958091CB1045
:10A9A000882321F00E9458541092CB108091CC1033
:10A9B000882321F00E9457531092CC101092491016
:10A9C0000895EF92FF92CF93DF93B82FA92FF62F20
:10A9D000E72F81E0809349102091182730911927A3
:10A9E00040911A2750911B272F5F3F4F4F4F5F4FCA
:10A9F000209318273093192740931A2750931B2729
:10AA0000862F8E5F87FF0CC08091D1269091D22631
:10AA100001969093D2268093D126CFEFDFEF0BC023
:10AA20002AE430E1C9016B2F7A2F4F2F5E2F0E944D
:10AA30006B7DC0E0D0E00E94CE54CE01DF91CF917B
:10AA4000FF90EF9008959091390191FD0AC0282F51
:10AA5000803108F02FE085E491E06FE040E00E9453
:10AA6000DF5808958093CE1008950E943A53825083
:10AA7000813130F4E82FF0E0E55DF94F80810895F1
:10AA800081E0089508958FEF80934E018CE691E068
:10AA900060EF44E022E00E94DF588CE290E06EE03C
:10AAA00041E025E00E94DF5880E880936F018091AB
:10AAB000460180936D0184E491E060E245E021E08D
:10AAC0000E94DF580895CF93DF93CDEFD3E0CE01FE
:10AAD0000197F1F70E94CB58109248251092CA2591
:10AAE00010924C261092472510924625E9E3F1E09A
:10AAF00080818E7F808380818D7F80838DE090E058
:10AB00000197F1F780818160808382E491E06FE1B9
:10AB100040E023E00E94DF582197F1F780915D012A
:10AB200080915E010E9443558DE096E060E070E008
:10AB30000E94F6400E94585481E090E0DF91CF914E
:10AB400008958091CD100895DF93CF930F92CDB7E4
:10AB5000DEB789830E94355329812093CD1088E484
:10AB600091E06FE140E00E94DF580F90CF91DF91BC
:10AB700008950E94A45586E00E94FD530895809395
:10AB800062019093630160936001709361014115CC
:10AB9000510531F1FA01819180936B01DA0111962F
:10ABA0008C9180936A01DF01119681818093690104
:10ABB000FD01319611968C9180936801DF01119609
:10ABC000818180936701FD01319611968C911197D7
:10ABD0008093660181818093650182818093640105
:10ABE00008958DE096E00E94194181E080933F2511
:10ABF0008091402590914125019690934125809325
:10AC0000402581E090E00895EF92FF92CF93DF938B
:10AC100050914725252F30E0F901EE0FFF1F3695A3
:10AC2000322F222737952795E20FF31FE85BFA4D65
:10AC30004081442309F4CEC02091390121FDCAC0CE
:10AC40002091D426222309F4C5C047FF16C00E94D4
:10AC5000EB528091082790910927A0910A27B09183
:10AC60000B270196A11DB11D8093082790930927FA
:10AC7000A0930A27B0930B27ADC04330B0F40E94D5
:10AC8000EB528091042790910527A0910627B0915F
:10AC900007270196A11DB11D8093042790930527D6
:10ACA000A0930627B093072795C0C42FD0E0229722
:10ACB0006C177D07B0F40E94EB52809100279091B1
:10ACC0000127A0910227B09103270196A11DB11D74
:10ACD0008093002790930127A0930227B093032726
:10ACE00079C0652F70E09B01220F331F7695762F78
:10ACF000662777956795260F371F275B3A4DB90171
:10AD000050E00E946B7D20914725822F90E0FC014E
:10AD1000EE0FFF1F9695982F882797958795E80F38
:10AD2000F91FE853FA4D808180933825822F90E0F7
:10AD3000FC01EE0FFF1F9695982F88279795879512
:10AD4000E80FF91FE85BFA4D10822F5F209347252B
:10AD5000233010F0109247258091472590E0FC01A8
:10AD6000EE0FFF1F9695982F882797958795E80FE8
:10AD7000F91FE85BFA4D8081882311F00E94F1559C
:10AD8000609147016093392580913E25882311F019
:10AD9000681710F460933E2584E070E00E94B54887
:10ADA0006091382583E070E00E94B54880911C27AF
:10ADB00090911D27A0911E27B0911F270196A11DDC
:10ADC000B11D80931C2790931D27A0931E27B0933D
:10ADD0001F2702C0C0E0D0E0CE01DF91CF91FF90ED
:10ADE000EF900895CF93DF93EC01888199810097CC
:10ADF00029F024E08B3F920739F505C08BEF94E0F2
:10AE00009983888325C0623819F510923F250E94E6
:10AE10002F480E948C4760E870E00E940456181684
:10AE2000190644F40E948747E0919E06F0919F0620
:10AE30000995E4CF80913C2590913D250196909312
:10AE40003D2580933C25DACF1982188283E001C02A
:10AE500081E0DF91CF91089591E0909349100E9495
:10AE600023550E94CE5408958091390181FD07C079
:10AE700085E491E06FE040E00E94D558089580E1BC
:10AE80000895CF92DF92EF92FF920F931F93CF938B
:10AE9000DF93182F21E0209349100091D426809150
:10AEA000390181FF16C08091940090919500909394
:10AEB000692780936827209357272093D326809172
:10AEC00039018D7F809339018091D3268823E1F762
:10AED00000E00E9435538091D426882309F441C0B4
:10AEE000809159278823E9F12091940030919500B1
:10AEF00080916C2790916D2728173907A0F4209135
:10AF00003C2730913D2740913E2750913F272C57B9
:10AF1000314E4F4F5F4F20933C2730933D27409356
:10AF20003E2750933F272091940030919500281B95
:10AF3000390B40E050E0C0903C27D0903D27E09096
:10AF40003E27F0903F272C0D3D1D4E1D5F1D209389
:10AF50003C2730933D2740933E2750933F27109244
:10AF6000592789E10E94FD5386E00E94C04800975E
:10AF700051F00E943457C82F86E00E94C04881508B
:10AF80000E94235502C0C0E0D0E0809194009091CF
:10AF9000950090936B2780936A2781E080935827D0
:10AFA000F894809139018260809339018091390150
:10AFB0008D7F80933901612F6E5F8AE490E10E945A
:10AFC000105978948091CE269091CF260196909337
:10AFD000CF268093CE260E94355382E491E060EE26
:10AFE00045E00E94D558182F86E00E94C04800977F
:10AFF00019F08C2F0E942355002319F00E945854F9
:10B0000002C00E945753809158278823E9F180910C
:10B0100094009091950040916A2750916B27841776
:10B020009507A0F48091382790913927A0913A276D
:10B03000B0913B278C57914EAF4FBF4F809338272D
:10B0400090933927A0933A27B0933B2720919400FF
:10B0500030919500241B350B40E050E0809138275B
:10B0600090913927A0913A27B0913B27280F391F9B
:10B070004A1F5B1F209338273093392740933A2784
:10B0800050933B27109258278091D426882361F053
:10B09000809194009091950090936D2780936C27F8
:10B0A00081E08093592707C082E491E06FE140E09E
:10B0B00023E00E94DF580E94CE541130E1F013309B
:10B0C000A9F48091102790911127A0911227B09197
:10B0D00013270196A11DB11D80931027909311276E
:10B0E000A0931227B093132712E00AC0153029F05D
:10B0F000173031F404C010E003C013E001C011E0C8
:10B10000812F90E0DF91CF911F910F91FF90EF90F1
:10B11000DF90CF900895CF93DF93EB010E94E1542D
:10B120009C01009731F4CE010E9441579C01009789
:10B1300049F08091D1269091D22601969093D22603
:10B140008093D126C901DF91CF9108950F931F936A
:10B150008091D426882321F40E94835411E001C0F9
:10B1600010E00E943A53863111F0813119F40091B8
:10B17000470109C086E491E06FE140E00E94D558A4
:10B18000082F000F080F112311F00E94E553802FA4
:10B190001F910F9108951092D0101092CF10EFE6EA
:10B1A000F0E08081806280830895FC0180818623A5
:10B1B00090E002C0959587954A95E2F70895F89436
:10B1C000FC019081862F8095892330E002C0220FF8
:10B1D000331F4A95E2F72623282B2083789408957D
:10B1E000DC01119620917B01FC012083215030E08D
:10B1F000A9014F575E4FE0E8F1E061916D93E417CC
:10B20000F507D9F7FC01E058FF4F2F573E4FD90102
:10B210002C9120838F579F4F21E0FC0120830895BC
:10B22000FC016093800101966350860F911DA1E897
:10B23000B1E021912D93E817F907D9F708951F92EE
:10B240000F920FB60F920BB60F9211242F933F93CC
:10B250004F935F936F937F938F939F93AF93BF931E
:10B26000EF93FF93809147018093392520914625E4
:10B2700030E0C901880F991F3695322F2227379564
:10B280002795820F931F885B9A4D0E94F0588091FA
:10B2900046258F5F80934625833010F01092462517
:10B2A0000E94F155FF91EF91BF91AF919F918F91C6
:10B2B0007F916F915F914F913F912F910F900BBEB6
:10B2C0000F900FBE0F901F9018951F920F920FB600
:10B2D0000F9211240F900FBE0F901F9018951F9280
:10B2E0000F920FB60F9211240F900FBE0F901F9068
:10B2F00018951F920F920FB60F9211240F900FBE48
:10B300000F901F9018951F920F920FB60F92112455
:10B310001092D3260F900FBE0F901F9018951F927A
:10B320000F920FB60F9211241092D3260F900FBEDA
:10B330000F901F9018951F920F920FB60F92112425
:10B340008F9381E080933F258F910F900FBE0F90D8
:10B350001F9018951F920F920FB60F921124109202
:10B36000D3260F900FBE0F901F9018951F920F922B
:10B370000FB60F9211248F939F938091CF109091CD
:10B38000D01001969093D0108093CF109F918F9101
:10B390000F900FBE0F901F9018950F931F93CF9390
:10B3A000DF938091DC269091DD26A091DE26B0917E
:10B3B000DF260196A11DB11D8093DC269093DD262A
:10B3C000A093DE26B093DF260E947E5CEC0181ED27
:10B3D00090E10E94BB410BC0D8011296ED91FC9107
:10B3E0001397309709F00995C8010E948142082FF0
:10B3F000192F0115110581F7209719F0CE010E9430
:10B400002B3FDF91CF911F910F9108950E94B8615A
:10B410000E942F480E94885A8FE796E09093D72683
:10B420008093D6260E947B5C82E090E060E074E02E
:10B4300040E05EE12FEF31E00E943C5C0895CF9246
:10B44000DF92EF92FF920F931F93CF93DF936C01E4
:10B45000EB018A0181ED90E10E94BB410CC0D70154
:10B460001496ED91FC911597309711F0CE01099546
:10B47000C7010E948142E82EF92EE114F10479F708
:10B48000C601BE01A8010E94333FDF91CF911F91F9
:10B490000F91FF90EF90DF90CF900895BC0181ED68
:10B4A00090E10E9442420895BC0181ED90E10E942A
:10B4B00009420895CF93DF93EC018091D8269091B3
:10B4C000D926A091DA26B091DB260196A11DB11DE7
:10B4D0008093D8269093D926A093DA26B093DB26C2
:10B4E000CE010E94955C009769F00E94A947E09107
:10B4F0008306F09184068FE19AE5BE01099521E06B
:10B5000030E002C020E030E0C901DF91CF91089522
:10B5100083ED90E10E94B74108950F93CF93DF939D
:10B52000EC017B836A8318865F834E8383ED90E111
:10B53000BE010E944242E091D510F091D6103097A2
:10B5400049F04C815D818A819B81688520E030E0F3
:10B5500001E00995DF91CF910F910895BC0183ED32
:10B5600090E10E94094208950F93DC0118961C9205
:10B570001897E091D510F091D610309759F01296A7
:10B580008D919C91139760E040E050E020E030E026
:10B5900000E009950F9108950F93DC01AB0114961B
:10B5A0002D913C91159781E018968C9318971596DC
:10B5B0007C936E931497E091D510F091D61030974C
:10B5C00039F012968D919C91139761E000E00995F6
:10B5D0000F9108950F93DC01E091D510F091D610F2
:10B5E000309769F014962D913C91159712968D9194
:10B5F0009C91139718966C91A90101E009950F9100
:10B600000895E091D710F091D810309709F009957E
:10B6100008959093D8108093D71008959093D610E2
:10B620008093D510089583ED90E10E94BB41089569
:10B63000EF92FF920F931F93CF93DF938C01EB0157
:10B640007A0183ED90E10E94BB4115C0DC011296A6
:10B650002D913C9113972C173D0759F41696ED91B7
:10B66000FC911797309761F0B801AE0197010995E9
:10B6700007C00E948142282F392FC901009731F756
:10B68000DF91CF911F910F91FF90EF900895089552
:10B69000AF92BF92CF92DF92EF92FF920F931F93E0
:10B6A000DF93CF9300D0CDB7DEB75B010E948C470C
:10B6B000FC01008111811A8309830C30110518F4F3
:10B6C000EE24FF242EC000D000D087E496E0EDB732
:10B6D000FEB792838183148303830E94EA7D0F90D7
:10B6E0000F900F900F9020C00E948C47F701EE0F33
:10B6F000FF1FEE0FFF1FE80FF91FC280D3800E94CB
:10B700008C470894E11CF11CF701EE0FFF1FEE0FB0
:10B71000FF1FE80FF91F40815181C501B6010E944A
:10B72000185BE016F10600F30F900F90CF91DF91B8
:10B730001F910F91FF90EF90DF90CF90BF90AF904F
:10B740000895CF93DF93C4EFD0E160910A11709117
:10B750000B11CE0143ED5BE520E030E00E94804418
:10B760000E94B56160910A1170910B110E94527A8A
:10B77000BC01CE01409748EE5BE520E030E00E943E
:10B780008044DF91CF9108950F93013051F480915F
:10B7900004119091051190930B1180930A110E944E
:10B7A000A15B0F91089580910A1190910B11209146
:10B7B000081130910911880F991F2817390708F4CB
:10B7C000C90190930B1180930A110E94A15B089507
:10B7D000EF92FF92CF93DF930E942F480E948C47F5
:10B7E000E82EE7017E01F92EE701198218820E94F6
:10B7F000135B26C028813981F901EE0FFF1FEE0F80
:10B80000FF1FEC0FFD1FDC0112964D915C91139709
:10B81000538342832F5F3F4FF901EE0FFF1FEE0F5F
:10B82000FF1FEC0FFD1F14964D915C9115975183EE
:10B830004083398328830E948142282F392FC901F0
:10B84000009721F0FC0120852223A1F688819981AF
:10B85000880F991F880F991F02960E948747888139
:10B860009981009721F089ED90E10E94FE3EDF91E1
:10B87000CF91FF90EF900895EF92FF920F931F9357
:10B88000CF93DF93FC018B017A01E90189ED90E10F
:10B89000BF0144E656E00E94E03E1093051100937C
:10B8A0000411F0920711E0920611D0930911C09390
:10B8B000081184EC9BE50E940E5BDF91CF911F91F4
:10B8C0000F91FF90EF900895CF93DF93C4EFD0E1F5
:10B8D000CE010E940745CE0140970E940745CE0148
:10B8E0004B970E94FB3EDF91CF91089580910A1102
:10B8F00090910B1108950E943F3F0895EF92FF929F
:10B90000CF93DF93E0916806F09169060995EC0109
:10B91000009729F06A817B8181E00E94B548CE01C1
:10B92000DF91CF91FF90EF9008950F931F93CF93E6
:10B93000DF938C01E0916A06F0916B060995EC01AA
:10B94000F8016281738181E00E94B54821E030E016
:10B95000209711F420E030E0C901DF91CF911F91D1
:10B960000F910895E0916C06F0916D060995089588
:10B97000FC0120E030E004C08181280F311D3296A7
:10B9800080818823C9F7C9010895FC01818190E075
:10B99000308120E0822B932B02C0880F991F6A957B
:10B9A000E2F7892F9927FA01E259F94F208130E017
:10B9B0008223932328E030E0241B350B02C09695A8
:10B9C00087952A95E2F708956F927F928F929F92C2
:10B9D000AF92BF92CF92DF92EF92FF920F931F939D
:10B9E000CF93DF936C017B015A0189012830310527
:10B9F00044F4CB01BA01A9010E94C55CF601808321
:10BA000041C0390133E0759467943A95E1F74115E7
:10BA1000510521F04C01C0E0D0E016C0DB01FC0173
:10BA2000C0E0D0E08D9181932196C615D705D4F35F
:10BA3000A801477050704115510521F1C7018C0FC5
:10BA40009D1F60E070E019C0C7018C0F9D1FB501FC
:10BA500048E050E00E94C55CF40181934F012196BB
:10BA6000C615D7058CF3A8014770507041155105D4
:10BA700049F0C7018C0F9D1FB5010E94C55CCC0D1C
:10BA8000DD1D8883DF91CF911F910F91FF90EF9083
:10BA9000DF90CF90BF90AF909F908F907F906F90EE
:10BAA00008954F925F926F927F928F929F92AF9282
:10BAB000BF92CF92DF92EF92FF920F931F93DF938B
:10BAC000CF9300D000D0CDB7DEB70E948C47E82ED0
:10BAD000092F82E090E00E946847009709F464C053
:10BAE000EE2DF02F918180E02081820F911D0E9428
:10BAF000533F7C01009709F459C00E948C473C01D8
:10BB0000F7014681242F30E02770307081E090E00B
:10BB10002115310511F480E090E046954695469553
:10BB2000840F911D0E9468470097F1F1F70104818D
:10BB30001581CC24DD2453E0452E512C4C0E5D1E86
:10BB40004E010894811C911C2AC0F801A180BB24DD
:10BB5000B60143E0759567954A95E1F7660D771D47
:10BB6000A60147705070883150F0C40195010E94C1
:10BB7000E45CF8018081B4010E94C9480CC01C82B9
:10BB80001B82C20195010E94E45C6B817C81F801FB
:10BB900080810E94B548CA0CDB1C0E5F1F4FF80164
:10BBA0008081882391F602C0EE24FF24C7010F9004
:10BBB0000F900F900F90CF91DF911F910F91FF90F9
:10BBC000EF90DF90CF90BF90AF909F908F907F903D
:10BBD0006F905F904F900895FC0150E080E190E0FD
:10BBE000861B970B821B930B02C0440F551F8A952F
:10BBF000E2F78081852B80838181842B8183089566
:10BC00006F927F928F929F92AF92BF92CF92DF926C
:10BC1000EF92FF920F931F93CF93DF938C015B0101
:10BC20006A0179012830310524F4C801FA01408104
:10BC300056C0390163E0759467946A95E1F7A114E1
:10BC4000B10421F04A01C0E0D0E021C0DA01F801DE
:10BC500080E090E02D912193019686159705D4F30D
:10BC600097012770307021153105D9F1F601E80FE1
:10BC7000F91F408150E068E070E0621B730B02C066
:10BC8000559547956A95E2F7800F911F26C0F401FC
:10BC900041914F01C8018C0F9D1FB50128E030E094
:10BCA0000E94EC5D2196C615D7058CF3970127708D
:10BCB000307021153105A9F0F601EC0FFD1F408110
:10BCC00050E0C5010896821B930B02C0559547951D
:10BCD0008A95E2F7C8018C0F9D1F60E070E00E941A
:10BCE000EC5DDF91CF911F910F91FF90EF90DF906E
:10BCF000CF90BF90AF909F908F907F906F9008955E
:10BD00004F925F926F927F928F929F92AF92BF926B
:10BD1000CF92DF92EF92FF920F931F93DF93CF9317
:10BD200000D0CDB7DEB78C01DC0116964C9116978A
:10BD3000842F90E08770907021E030E0009711F43C
:10BD400020E030E04695469546957901E40EF11CD9
:10BD5000C70102960E94F447009709F453C00E945D
:10BD60009447FC01D80112968C9112978083139608
:10BD70008C9181830E949447F2E06F2E712C680EA3
:10BD8000791EC30160E070E0A7010E94747DF80194
:10BD9000C480D58000E010E02E010894411C511CA5
:10BDA0002AC0D60111968C90119799247801E3E06E
:10BDB000F594E794EA95E1F7E60CF71C77E0A72EF7
:10BDC000B12CA022B122883130F00E94D348AC01BE
:10BDD000C701B50107C00E94C0489A838983C70183
:10BDE000B501A20194010E94005E080D191DE2E058
:10BDF000F0E0CE0EDF1ED6018C91882391F621E073
:10BE000030E002C020E030E0C9010F900F90CF91E8
:10BE1000DF911F910F91FF90EF90DF90CF90BF9037
:10BE2000AF909F908F907F906F905F904F9008950C
:10BE3000E0919C06F0919D0609950895E0914506D4
:10BE4000F091460609950895E091A006F091A106AB
:10BE500009950895E091A206F091A3060995089529
:10BE600080E090E008950895E0912706F09128067B
:10BE700009950895009731F0E0912706F091280682
:10BE800009950895E0912906F0912A0609950895EB
:10BE900080E090E008950F931F93DF93CF93CDB789
:10BEA000DEB7E0970FB6F894DEBF0FBECDBF0E949D
:10BEB000DE478C010E948C47602FAE014F5F5F4FC1
:10BEC0000E947E67882309F445C088A99801281B31
:10BED0003109C9010E9468470097E1F12E812223B0
:10BEE00071F18A859B853BEA8D3C930721F03FEFFA
:10BEF0008F3F930779F5223041F088E090E007C04A
:10BF0000019722912F3F41F00BC082E090E0FE01AB
:10BF1000E80FF91F3C96F4CF181619068CF30FC0E2
:10BF200089E1BE01645F7F4F0E94C94889E10E9498
:10BF3000D34865EE74E20E94913E009759F088E183
:10BF4000BE016A5E7F4F0E94C948E0918506F0916C
:10BF500086060995E0960FB6F894DEBF0FBECDBFFA
:10BF6000CF91DF911F910F910895AF92BF92CF9221
:10BF7000DF92EF92FF920F931F93DF93CF93CDB792
:10BF8000DEB7E0970FB6F894DEBF0FBECDBF6C01F1
:10BF90008B01FE01319680E3DF011D928A95E9F75E
:10BFA00081E089838CE00E94C0488C831D821F82BF
:10BFB00080910E1189878F5F80930E1183E0E82EA8
:10BFC000E8868DEC9BEA9B878A8789E10E94D348AB
:10BFD0006FE575E00E94913E009731F082E08E831C
:10BFE0008FEF8C878D8709C089E10E94D348BC01FF
:10BFF000CE010C960E94883EEE828DEC9BEA9D8BD2
:10C000008C8BCE01469665EE74E20E94883E0E94BB
:10C010008C479FA78EA70E94DE4788AB7E010894BD
:10C02000E11CF11CC7010E947566A82E90E00E94D9
:10C03000F447009741F10E949447BC01C7014A2D83
:10C040000E949366A0901D06B0901E060E94944721
:10C050007C010E94E847BC01C701F5010995C114A4
:10C06000D10489F0009721F08130910561F404C07A
:10C07000C80160E070E003C0C80164E070E041E026
:10C0800050E0F6010995E0960FB6F894DEBF0FBEBA
:10C09000CDBFCF91DF911F910F91FF90EF90DF9077
:10C0A000CF90BF90AF9008950E94B56180930E111C
:10C0B000E0912706F091280609950895EF92FF92E6
:10C0C000CF93DF93E82EE7017E01F92EE70104C04C
:10C0D00060E070E00E94F640899199910097C1F765
:10C0E000DF91CF91FF90EF900895EF92FF92CF9361
:10C0F000DF93E82EE7017E01F92EE70102C00E94DE
:10C100003B40899199910097D1F7DF91CF91FF90B2
:10C11000EF900895CF93DF93EC017B836A830E94B5
:10C12000475199838883DF91CF910895FC018081E5
:10C13000918122813381820F931F9183808308959F
:10C14000CF93DF93EC010E94475199838883DF915D
:10C15000CF910895CF93DF93EC010E94475128813E
:10C160003981821B930B019621E030E04A815B818B
:10C170004817590710F020E030E0C901DF91CF9156
:10C180000895EF92FF92CF93DF93FC01C281D38198
:10C1900080819181C80FD91F0E944751C81BD90BBC
:10C1A000CE01DF91CF91FF90EF900895CF93DF9371
:10C1B000EEE5F7E2C0E2D7E2A2E5B7E21192119212
:10C1C00019921992199219921D9287E2E637F8078F
:10C1D000A9F7DF91CF9108950F931F93CF93DF932A
:10C1E000FC01DC01AE5AB84D8C91882339F10091E5
:10C1F000940010919500EF01CC0FDD1FCC0FDD1FD7
:10C20000C05ED84DDF01AA0FBB1FA25AB84D8D9159
:10C210009C9111979801281B390B40E050E06881F0
:10C2200079818A819B81260F371F481F591F2883D8
:10C2300039834A835B8311961C930E93EE0FFF1F85
:10C24000EE0FFF1FE05EF84D608171818281938166
:10C25000DF91CF911F910F91089560E070E0CB01C5
:10C260000895FC01EE0FFF1FEE0FFF1FE05EF84D7B
:10C2700040835183628373830895EF92FF920F93FB
:10C280001F93CF93DF9322E537E2C0E2D7E2EEE5DA
:10C29000F7E2D9018D919D018823C9F04091940066
:10C2A00050919500808191817A01E81AF90A00E0A5
:10C2B00010E088819981AA81BB818E0D9F1DA01FEE
:10C2C000B11F88839983AA83BB83518340832496BB
:10C2D0003296B7E22E353B07E1F6DF91CF911F9101
:10C2E0000F91FF90EF9008950E94F26508950F93CB
:10C2F0001F93FC01CB0140910F115091101133831A
:10C3000022831583048371836083F0931011E0937B
:10C310000F114115510511F40E940C6680E090E068
:10C320001F910F91089580910F1190911011009716
:10C33000C1F01092101110920F11DC0114966D9142
:10C340007C9115971296ED91FC9113970995E091C8
:10C350000F11F0911011309721F0808191810E948E
:10C360000C6608950E94407B08950E943B7B0895CF
:10C3700086EA96E00E942F418EEA96E00E942F41C5
:10C380000895EF92FF92CF93DF930E949B4700970F
:10C39000C9F08EEA96E00E944F41E82EE7017E0147
:10C3A000F92EE701209731F10E94DE4799838883B7
:10C3B0000E94D9479B838A83C70104960E9407473E
:10C3C0008CAB18C086EA96E00E944F41EC017E01DA
:10C3D000F92EE701209771F0C70102960E941E47CF
:10C3E00099838883B7016E547F4FC7018E579F4F43
:10C3F0000E948B48CE01DF91CF91FF90EF9008957E
:10C40000BC016E547F4F8E579F4F0E948B480895FA
:10C41000CF93DF93EC0186EA96E0BE010E949A4139
:10C42000009719F086EA96E009C08EEA96E0BE0110
:10C430000E949A41009729F08EEA96E0BE010E9480
:10C440007541DF91CF910895EF92FF92CF93DF93E3
:10C45000EC0186EA96E0BE010E949A41009779F0CD
:10C4600068817981CE0102960E945848BE016E54BF
:10C470007F4FCE018E579F4F0E94A0481BC08EEA6F
:10C4800096E0BE010E949A410097A1F00E942F48B9
:10C49000688179818A819B810E9458488CA990E0AB
:10C4A0000E94F4470E9494474CA92496BE0150E094
:10C4B0000E946B7DDF91CF91FF90EF900895EF92F6
:10C4C000FF92CF93DF93EC0186EA96E0BE010E94D3
:10C4D0009A41009711F022960DC08EEA96E0BE01B7
:10C4E0000E949A41009721F00A80DB81C02D02C092
:10C4F000C0E0D0E0CE01DF91CF91FF90EF900895A2
:10C50000FC0180819181089570E06F5B7F4F660F21
:10C51000771F680F791FCB010895E62FF0E0EF5BDE
:10C52000FF4FEE0FFF1FE80FF91F808191810895E3
:10C53000089587E697E10E94A543009721F087E6DA
:10C5400097E10E9490430895E0917417F091751758
:10C55000309711F00995089580E00895EF92FF92C9
:10C560000F931F93CF93DF93EC018A018881998108
:10C57000009731F023E08C30920709F006C12BC000
:10C5800080E00BC0E82FF0E0EE0FFF1FEE0FFF1F63
:10C59000EB5AF84E118210828F5F843098F38093AB
:10C5A0006F178091960E9091970E909366178093D7
:10C5B00065170E9434408093762787E697E160E410
:10C5C00070E00E947A430E940D698CE093E09983A9
:10C5D000888381E0DDC0623009F4B9C0633030F493
:10C5E000662309F489C0613081F79CC0673819F06F
:10C5F000683859F741C01092701745E5E42E47E1BD
:10C60000F42E18C0F701828193818017910749F4B5
:10C61000808191810E94546AF701118210821382F5
:10C62000128284E090E0E80EF91E809170178F5F0F
:10C630008093701780917017843020F3E6E8FCE255
:10C64000848D958D8017910719F4158E148E118E97
:10C65000B0969DE2E630F90799F7ECE1FDE28185BD
:10C6600092858017910711F4158214823D962DE270
:10C67000EE39F207A1F7A9CF87E14736580709F04D
:10C68000A4CFCA010E94A543009709F49ECF10923F
:10C6900070172DC0F0E035E0EE0FFF1F3A95E1F77F
:10C6A000EA57F34D818D8823E9F087E697E10E94F0
:10C6B00090438091701790E025E0880F991F2A958C
:10C6C000E1F78A57934D9093852C8093842C82E0D8
:10C6D0000E94886A8091772790917827009711F0BF
:10C6E0000E94A462809170178F5F80937017E09111
:10C6F0007017E43078F269CF4115510509F465CF20
:10C700005093852C4093842C83E00E94886A80910A
:10C71000772790917827009711F00E94A4620E94D9
:10C72000996253CF4115510509F44FCF5093812C95
:10C730004093802C85E00E94886A809177279091B1
:10C740007827009709F441CF0E94A4623ECF8091E0
:10C75000772790917827009709F437CF8091882721
:10C76000863031F48091A02781FF02C00E94996237
:10C7700081E00E94886A80917727909178270097BE
:10C7800009F423CF0E94D76420CF1982188283E056
:10C79000DF91CF911F910F91FF90EF9008959093AB
:10C7A00075178093741708952091960E3091970E07
:10C7B00060E0E5E5F7E113C0408151814817590772
:10C7C00061F4428153814217530739F46093731720
:10C7D000118210820E94546A089534966F5F64300B
:10C7E00058F360937317089540E0E5E5F7E116C04C
:10C7F000542F5F5F208131812115310569F4409309
:10C800007217918380832091960E3091970E338317
:10C8100022830E946E6A08953496452F443040F377
:10C82000409372170895FC018091960E9091970E97
:10C83000958F848F778F668F0895FC018091960E77
:10C840009091970E92878187748763870895CF931D
:10C85000DF93EA010E94D069FC01009741F08091CA
:10C86000960E9091970E92878187D487C387CF01C8
:10C87000DF91CF9108950F931F93DF93CF9300D053
:10C8800000D0CDB7DEB78C01AB018FEF89838A83EF
:10C890008B838C83CE010196B8010E942764FC0132
:10C8A000009711F015830483CF010F900F900F9024
:10C8B0000F90CF91DF911F910F91089583EC96E037
:10C8C00062E040E050E00E94E7401092782710922A
:10C8D00077270895AC0183EC96E061E00E94C440A4
:10C8E0000895AC0183EC96E060E00E94C440089596
:10C8F0000F931F93CF93DF93EA010E9446698C0147
:10C90000009761F08091960E9091970EF801958FA7
:10C91000848FD78FC68FC8010E947164C801DF91D0
:10C92000CF911F910F910895CF93DF93A091842C05
:10C93000B091852C109719F0ED016C9605C0C0914F
:10C94000802CD091812C299680917F2C86FF22C04B
:10C950001092711740E0E5E5F7E116C020813181C2
:10C9600014968D919C9115972817390759F4828157
:10C970009381009739F040937117998388831B82C4
:10C980001A8206C034964F5F443040F340937117CB
:10C990000E94996288819981009731F04A815B8178
:10C9A000609176270E94E740DF91CF9108950F9321
:10C9B0001F93CF93DF9380918827863009F074C04E
:10C9C000809177279091782725E08030920709F0B1
:10C9D0006BC0C4E9D2E0D0937827C093772702E0F8
:10C9E0000093812714E9109382271092A4271092B4
:10C9F000A3270E940569809590959093A427809322
:10CA0000A32710928A27109289270E94F4688095A4
:10CA1000909590938A27809389270E94A462D0934F
:10CA20007827C093772700938127109382279091CE
:10CA3000822C8091832CE92FF82FDF01A459BD4F60
:10CA40008CE692E00D9001920197E1F787E997E279
:10CA50006CE672E00E94986880917B27809397270C
:10CA600080917C278093982780917D2780939927B8
:10CA700080917E2780939A271092A4271092A32753
:10CA80000E940569809590959093A4278093A32791
:10CA900010928A27109289270E94F46880959095B9
:10CAA00090938A27809389270E94A462DF91CF9177
:10CAB0001F910F910895282F392FF90120E030E0C0
:10CAC00080E0A8E112C0419198E0542F5827B52F7B
:10CAD000B17050FD8A278695B13009F48068915075
:10CAE00011F04695F2CF2F5F3F4F2617370759F7C2
:10CAF00008951F920F920FB60F920BB60F9211244A
:10CB00002F933F934F935F936F937F938F939F9355
:10CB1000AF93BF93EF93FF93809194009091950012
:10CB2000909363278093622781E0809354278091BC
:10CB30007100807D809371000E94936180915427E1
:10CB40008823E9F1809194009091950020916227CB
:10CB50003091632782179307A0F480912827909142
:10CB60002927A0912A27B0912B278C57914EAF4FA0
:10CB7000BF4F8093282790932927A0932A27B0930B
:10CB80002B278091940090919500821B930BA0E03D
:10CB9000B0E0209128273091292740912A275091F1
:10CBA0002B27820F931FA41FB51F809328279093D4
:10CBB0002927A0932A27B0932B2710925427FF915F
:10CBC000EF91BF91AF919F918F917F916F915F9105
:10CBD0004F913F912F910F900BBE0F900FBE0F9072
:10CBE0001F9018959FB7F894E1E7F0E08081807D71
:10CBF000808388B38F6288BB10929000E1E9F0E0F7
:10CC000010821092920010929500109294008081F0
:10CC1000856080839FBF08952FB7F8949093990003
:10CC20008093980088B38F6288BBE1E7F0E0808151
:10CC3000826080832FBF0895EF92FF92CF93DF939E
:10CC4000FC01DB0185E0EB0119928A95E9F785810A
:10CC500090E083709070009711F082E08C93878150
:10CC600090E083709070009721F082E012968C9390
:10CC70001297858190E083709070009799F087817A
:10CC800090E083709070009769F0238934898185E2
:10CC900092852817390731F481E0848312961C921B
:10CCA000129701C01482858183708250823030F4E3
:10CCB000C82FD0E0C353D94F888101C080E01196BE
:10CCC0008C931197E781E370E250E23028F4F0E0B2
:10CCD000E353F94F808101C080E013968C93139742
:10CCE000DF91CF91FF90EF900895DF93CF9300D025
:10CCF00000D00F92CDB7DEB7BE016F5F7F4F0E94AD
:10CD00001C6689819A81890F8D5F9B81890F9C8127
:10CD1000890F9D81890F0F900F900F900F900F90AA
:10CD2000CF91DF910895AF92BF92CF92DF92EF92B1
:10CD3000FF920F931F93DF93CF9300D000D000D0CA
:10CD4000CDB7DEB78C017B01BE016F5F7F4F4E8395
:10CD50000E941C66C9809A81A92EBB24DB808C812D
:10CD6000682F70E095012C0D311D2D5F3F4F2D0D6B
:10CD7000311D260F371F5D81250F311D4E8150E07B
:10CD8000421753070CF4A8C0D80111964C91119783
:10CD900050E041705070E3E0440F551FEA95E1F711
:10CDA00012962C91129730E02170307054E0220FCF
:10CDB000331F5A95E1F7242B3C913770232B1396A0
:10CDC0003C911397E32FF0E0E170F07045E0EE0F37
:10CDD000FF1F4A95E1F72E2B14963C911497E32FF1
:10CDE000F0E0E170F07036E0EE0FFF1F3A95E1F7EA
:10CDF0002E2BF701208315964C91159750E0437028
:10CE00005070440F551F440F551F16962C911697BE
:10CE100030E02370307054E0220F331F5A95E1F751
:10CE2000242B17963C9117973295330F330F307C94
:10CE3000322B318318962C9118972283FC2DF230D7
:10CE400069F419962C91D70113962C931397F80136
:10CE5000228514962C93149745E001C043E0E92FF6
:10CE6000F0E03B96E00FF11F542F0AC09701250F09
:10CE7000311DC290D901CC925F5F0894A108B1081E
:10CE8000A114B10499F7940FBD2DB23089F4F701C4
:10CE9000E90FF11DD80153962C91539720839F5F82
:10CEA000F701E90FF11D54962C91549720839F5F51
:10CEB000E82FF0E07596E00FF11F292F08C0D70189
:10CEC000A20FB11D32913C932F5F615070406115EC
:10CED0007105A9F7890F01C080E026960FB6F89476
:10CEE000DEBF0FBECDBFCF91DF911F910F91FF909D
:10CEF000EF90DF90CF90BF90AF900895BF92CF9208
:10CF0000DF92EF92FF920F931F93CF93DF937C01F9
:10CF1000D62EEA01633008F4ADC0FC018081B82E42
:10CF2000B294B694B694B3E0BB22F1E0BF22F7010D
:10CF30009181292F269526952370C92EC294C694D7
:10CF4000C694A3E0CA22382F37703883382F36951D
:10CF50003695369531703983382F329531703A8352
:10CF60008295869581708B83BC822D83892F8295D3
:10CF700083708E83CF828281888787010D5F1F4FE8
:10CF8000222361F1F801918180E0F7013381830F61
:10CF9000911D9A87898787010B5F1F4F223081F48B
:10CFA000CA010B966FE575E00E94883EF801818109
:10CFB0008B87F70185818C878701095F1F4F16C01A
:10CFC0002330A1F4F7013D96DA011B9682918D93EF
:10CFD000E017F107D9F7085F1F4F08C0CA010B9689
:10CFE0006FE575E00E94883E1A861986CC2089F18B
:10CFF000BB2059F4F801918180E02081820F911DBE
:10D000009C8B8B8B0E5F1F4F04C089859A859C8BF0
:10D010008B8BFC2DF23071F4CE0145966FE575E0F7
:10D020000E94883EF80181818D8B80818E8B0E5FFE
:10D030001F4F17C0FC2DF330A1F4085F1F4FD8011C
:10D04000FE01759680E09E9191938F5F8830D9F7AD
:10D0500008C0CE0145966FE575E00E94883E1C8AA7
:10D060001B8A802F8E199D2D981B9FA71EA70DA789
:10D07000D81608F480E0DF91CF911F910F91FF90B7
:10D08000EF90DF90CF90BF9008959C0141505040A9
:10D09000460F571FDB0110C0FC91E0E011968C9108
:10D0A0001197BF01680F711D260F371F261737070D
:10D0B00010F42F5F3F4F1296A417B50768F3A4171B
:10D0C000B50749F49C9180E0280F391F28173907CC
:10D0D00010F42F5F3F4FC9010895CF93DF939091D4
:10D0E0008227C92FD0E064973091812720E0C20FBA
:10D0F000D31F9E01280F311DC9016BE877E248E07C
:10D1000050E00E94456863E977E2AE010E944568FD
:10D11000009719F0382F292F02C02FEF3FEFC901D8
:10D12000DF91CF9108959093851780938417089588
:10D13000FC014381460F40937E27872F9927228148
:10D14000280F20937D27A181A0937C2750815093A5
:10D150007B2730E02817390748F48A2F8F5F8093A8
:10D160007C27882319F45F5F50937B27842F90E0FE
:10D1700070708617970798F480917D278F5F809352
:10D180007D27882361F480917C278F5F80937C27A3
:10D19000882329F480917B278F5F80937B270895D4
:10D1A000BC018091842C9091852C08960E949868EF
:10D1B000E091842CF091852C80917B278087809151
:10D1C0007C27818780917D27828780917E27838736
:10D1D00008959C01AB0180E090E0B9010E94456890
:10D1E000382F292FC901089580E090E06FE777E29A
:10D1F00044E150E00E944568009719F0382F292F2C
:10D2000002C02FEF3FEFC901089586E00E946D68CC
:10D21000089581E10E946D68089580E009C0E82FBB
:10D22000F0E0EE0FFF1FEA5FF24D118210828F5F78
:10D230008430A8F380E00BC0E82FF0E095E0EE0F1B
:10D24000FF1F9A95E1F7EA57F34D118E8F5F8430F7
:10D2500098F380E094E0909387178093861740E0DE
:10D260008DE090E00EC0242F30E0289FF001299F30
:10D27000F00D389FF00D1124E45EF24D15821482FA
:10D280004F5F4A3080F340938217089520918617AC
:10D29000309187172F5F3F4F4DE72030340710F054
:10D2A00020E030E1522F432FA0E013C0EA2FF0E03E
:10D2B000B5E0EE0FFF1FBA95E1F7EA57F34DB18DD8
:10D2C000BB2331F00480F581E02DE417F50711F35D
:10D2D000AF5FA43059F730938717209386171092C9
:10D2E000821720E0E0E0F0E01EC0A22FB0E035E0C1
:10D2F000AA0FBB1F3A95E1F7AA57B34D59963C9137
:10D300005997332321F420938217FD0110C0373041
:10D3100049F4309731F05A964C915A97328D341720
:10D3200008F4FD012F5F243000F32093821730971B
:10D33000A9F122E0218F20917C17248720917D176D
:10D34000258720917E17268720917F17278728ED34
:10D3500034E0338B228B358B248B21E030E0318B12
:10D36000208B138E21E0228F23E0208F168A20E16C
:10D37000278B209186173091871732272327322752
:10D380003583248377836683DC012D913D914D9114
:10D390005C9113972083318342835383CF01089597
:10D3A0000F931F93CF93DF932091861730918717A8
:10D3B0004DE050E02F5F3F4FADE720303A0710F0CF
:10D3C00020E030E1B22FA32F10E012C0C12FD0E037
:10D3D000C49FF001C59FF00DD49FF00D1124E45EB1
:10D3E000F24D0480F581E02DEA17FB0719F31F5F6A
:10D3F0001A3061F7309387172093861710E02DE0DD
:10D4000030E01AC0012F0F5FC12FD0E0C29FF001A2
:10D41000C39FF00DD29FF00D1124E45EF24DDF01A9
:10D420001496448155814115510529F410938217B2
:10D43000309749F433C0102F1A3020F3109382171D
:10D44000E0E0F0E02BC0209186173091871732275B
:10D450002327322711963C932E9377836683009778
:10D4600029F4108211821282138209C0DC012D91ED
:10D470003D914D915C9120833183428353838DE0B4
:10D4800090E0C89FD001C99FB00DD89FB00D112466
:10D49000A45EB24D80E418968C931897CF01DF916B
:10D4A000CF911F910F91089540E013C0E42FF0E059
:10D4B000542F5F5FEE0FFF1FEA5FF24D2081318135
:10D4C0002817390729F44093821711821082089592
:10D4D000452F443058F340938217089540E013C01D
:10D4E000E42FF0E0542F5F5FEE0FFF1FEA5FF24D75
:10D4F000208131812115310529F4409382179183D0
:10D5000080830895452F443058F34093821708953F
:10D51000EF92FF920F931F93CF93DF93C091842CD0
:10D52000D091852C843009F4F7C107EA17E21093F3
:10D53000832C0093822C10937A27009379278330D1
:10D5400071F4898D90E08F7090708330910509F0AF
:10D5500074C088899989009709F02FC78DC08230DF
:10D5600009F08EC080917F178F5F80937F1788238B
:10D5700099F480917E178F5F80937E17882361F4E2
:10D5800080917D178F5F80937D17882329F4809188
:10D590007C178F5F80937C171092782710927727E3
:10D5A00010921B2D10921A2D898D873011F0853025
:10D5B00041F48A8D8F5F8A8F843109F0FEC6198EFF
:10D5C000FCC6882309F4F9C6288939892115310553
:10D5D00009F44EC09A8D292F21502A8F992309F0E2
:10D5E000ECC69B8D983031F0282F2150223048F422
:10D5F000953039F4198E80E880937F2C0E949464D2
:10D6000095C5953048F423E030E0092E02C0220F82
:10D61000331F0A94E2F701C020E32A8F9F5F9B8F9C
:10D6200090E08F70907083309105E1F08430910527
:10D630004CF48130910509F461C38230910509F001
:10D64000BCC60DC08630910509F40CC58830910523
:10D6500009F408C58430910509F0AFC603C51092DE
:10D66000A0274FC384E080937F2C0E94946490C5D0
:10D670008F70833009F0A1C688E080937F2C4BC562
:10D68000853019F5E091802CF091812C8481958171
:10D69000009709F492C61092852C1092842C0C509D
:10D6A00010401093832C0093822C10937A270093C0
:10D6B000792710921B2D10921A2D10927827109214
:10D6C000772788E080937F2C25C1085210408091F5
:10D6D0007F27853409F071C69091812780E02091E1
:10D6E00082277C01E20EF11C8091772790917827A8
:10D6F0008E159F0508F461C6F0927827E09277278F
:10D700008091852790E08F739070009709F055C63F
:10D7100080918627882309F050C68091162D90911C
:10D72000172DC091D306D091D4068C179D0759F4BC
:10D730004091182D5091192D2091D5063091D60683
:10D7400042175307A1F020918F2730919027281777
:10D75000390709F032C620919127309192278091A4
:10D76000182D9091192D2817390709F026C60E9407
:10D77000F4682FEF8F3F920709F01FC6809188272A
:10D78000863009F431C18131E9F1813009F015C6E3
:10D7900080919327883009F010C6109293278091CA
:10D7A0009527909196274FEF873F940710F00996A1
:10D7B00001C00896909396278093952780918B2798
:10D7C00090918C27A0918D27B0918E2780938F27E1
:10D7D00090939027A0939127B09392278091162D34
:10D7E0009091172DA091182DB091192D80938B2712
:10D7F00090938C27A0938D27B0938E2780E4F80117
:10D800008087B8C5C7014C97909378278093772776
:10D810008BE997E29093832C8093822C80919927B7
:10D8200090919A27009739F00E940969FFEF8F3F86
:10D830009F0709F0C2C520919527309196272115A1
:10D84000310509F4BAC58CE19DE29093812C809357
:10D85000802C6091D5067091D6064091CF065091EC
:10D86000D0060091D1061091D20639C084819581ED
:10D87000009781F12817390769F58681978100970C
:10D8800039F0A0919327B0919427A817B90711F503
:10D89000808191818C179D0729F4A281B381A617FD
:10D8A000B70739F18417950729F4A281B381A0172E
:10D8B000B107F9F0A0918B27B0918C27A817B90771
:10D8C00049F4A0918D27B0918E2782819381A8176A
:10D8D000B90779F03D96F093812CE093802CE0918C
:10D8E000802CF091812C8DE2EE39F80708F4BECF40
:10D8F00064C51092852C1092842C82E080937F2C3A
:10D900008BE997E290937A278093792710921B2DC9
:10D9100010921A2D0E94946480911A2D90911B2DC3
:10D92000009709F44AC59C01245E3F4F3093782745
:10D93000209377273093812720938227E091802CB2
:10D94000F091812C20852093872721E1209388273F
:10D950000896982789279827909398278093972748
:10D9600010929A27109299278481958190939427F9
:10D97000809393278681978190939627809395270C
:10D980008091162D9091172DA091182DB091192DE1
:10D9900080938B2790938C27A0938D27B0938E270D
:10D9A00080819181A281B38180938F27909390276A
:10D9B000A0939127B093922787EA97E29093832CC4
:10D9C0008093822C0E9409698095909590939A2764
:10D9D00080939927009709F0CDC48FEF9FEF909324
:10D9E0009A2780939927C6C40E940569EFEF8F3F5D
:10D9F0009E0709F0E2C480919527909196270097A1
:10DA000009F4DBC420919327309194272115310527
:10DA100009F4D3C4C6E8DCE2498D4423E9F06C8103
:10DA20007D8186179707C1F46E817F81261737079E
:10DA300099F4E0918B27F0918C2768817981E61722
:10DA4000F70751F4E0918D27F0918E276A817B8151
:10DA5000E617F70709F46DC1A096FDE2C630DF07AF
:10DA6000D9F62091A0272F732230B9F49093811713
:10DA70008093801740E00DC0E42FF0E0EE0FFF1F11
:10DA8000EA5FF24D208131814F5F8217930709F4DD
:10DA90006EC0443088F3409382178091A02782FDA6
:10DAA0008CC484E1F80181A388E290E09093782708
:10DAB0008093772780E580A380919A2790919E2775
:10DAC000938F3091992790919D27928F368F209137
:10DAD000982790919C27918F258F909197279093CD
:10DAE000821740919B27408F948F8F5F878F882369
:10DAF00061F4832F8F5F868F882339F4822F8F5FA5
:10DB0000858F882311F49F5F948F80919327909144
:10DB100094279093811780938017209195273091B7
:10DB20009627F801358B248B978B868B80918B27DA
:10DB300090918C27A0918D27B0918E2780938F276D
:10DB400090939027A0939127B09392278091162DC0
:10DB50009091172DA091182DB091192D80938B279E
:10DB600090938C27A0938D27B0938E27E8C31092B3
:10DB7000821780E0C0E0D0E022C0E82FF0E075E03E
:10DB8000EE0FFF1F7A95E1F7EA57F34D918D992338
:10DB900021F480938217EF0116C0973079F4209713
:10DBA00021F0228D9A8D921748F4C82FD0E065E0BD
:10DBB000CC0FDD1F6A95E1F7CA57D34D8F5F8430D4
:10DBC000E0F280938217209709F4F7C3D093852C55
:10DBD000C093842C83E08A8F888F1E8A84E08F8B89
:10DBE0001B8E80919527909196279D838C838091A1
:10DBF0009327909194279F838E8380918B27909178
:10DC00008C27A0918D27B0918E2788839983AA8332
:10DC1000BB8381E0898F80917C178C8780917D17F1
:10DC20008D8780917E178E8780917F178F8781E007
:10DC300090E0998B888B80919A278B878091992788
:10DC40008A8780919827898780919727888781E0A4
:10DC500090E00E94D06880919F27282F30E0207F9D
:10DC60003070213531050CF449C082958F7090E0F9
:10DC70000597880F991F880F991F5091831740E0CF
:10DC800034C0F901E158F84D50A5552329F44093CB
:10DC900082171092831732C0513011F44F5F25C0A4
:10DCA0005230E1F461A56430C9F440938217509377
:10DCB000831732A520E083A590E0822B932B9093CD
:10DCC000811780938017F4E0893D9F0710F088ED5D
:10DCD00094E09B8B8A8B9D8B8C8B10C02158384D88
:10DCE000F90121A5222331F0420F242F30E028171B
:10DCF00039073CF2409382175093831780E1809359
:10DD0000A0278091A02782608093A02782E0809343
:10DD1000A72784E08093A8278093A92788ED809384
:10DD2000AA278CE290E0909378278093772780E66B
:10DD3000B3C2D093852CC093842C10927F2C8091F9
:10DD4000A02790E082FF03C0198E80E24EC220918E
:10DD50009F2722952F70220F220F20938217B70141
:10DD6000621B71099B012451304030937827209326
:10DD7000772750E04F7050704230510539F4AC01B4
:10DD80004F7350704231510551F42AC04130510552
:10DD900031F4AC014F7350704230510509F1211537
:10DDA000310531F49C012370307021153105C1F02B
:10DDB000309197272885321709F064C2309198274F
:10DDC0002985321709F05EC2309199272A853217CA
:10DDD00009F058C230919A272B85321709F052C2A8
:10DDE00084FF4AC0688979896115710509F444C0C6
:10DDF000CE010C960E94986830919B2780917B27DA
:10DE00003817D1F520919C2780917C272817A1F500
:10DE100090919D2780917D27981771F580919E277D
:10DE200040917E27841741F53C872D879E878F87F9
:10DE30008B8D8823D1F42E89888D9A8D891B922F02
:10DE4000969596959695891B280F2E8B87FD819523
:10DE50009F89392F36953695931B980F9F8B822F6C
:10DE6000869586958695890F888F81E080937F2C93
:10DE7000888D8A8F198A188A298D30E0C9018F70A0
:10DE800090708430910509F4B5C18530910564F432
:10DE900082309105C9F1833091050CF0B9C0813011
:10DEA000910509F08AC211C08630910509F4E2C1DA
:10DEB000863091050CF4BEC18730910509F4E2C1AA
:10DEC0008830910509F079C28AC180917F2C80FF4A
:10DED00014C083E0898F80E480937F2C198A188A8C
:10DEE0008091772790917827009709F410C122E458
:10DEF00020937F2C0E94D0680AC18091A0278F7345
:10DF0000823009F05AC2FACE80917F2C80FF75C012
:10DF10008091A0278F73823109F06FC080919F2775
:10DF2000282F30E0207F3070213531050CF449C0B6
:10DF300082958F7090E00597880F991F880F991F21
:10DF40005091831740E034C0F901E158F84D50A5D5
:10DF5000552329F4409382171092831732C0513011
:10DF600011F44F5F25C05230E1F461A56430C9F46B
:10DF7000409382175093831732A520E083A590E049
:10DF8000822B932B909381178093801774E0893DA7
:10DF9000970710F088ED94E09B8B8A8B9D8B8C8B80
:10DFA00010C02158384DF90121A5222331F0420F2C
:10DFB000242F30E0281739073CF240938217509302
:10DFC000831783E0898F809197278887809198278E
:10DFD0008987809199278A8780919A278B8781E00A
:10DFE00090E00E94D06882E480937F2C198A188A7E
:10DFF00010927827109277278AC080E280937F2C36
:10E000000E949464E091842CF091852C118E45CD72
:10E010008091A02780FF2AC024FD28C08889998983
:10E02000009709F0CAC180917727909178270196CF
:10E030000E94D06820917F2C822F806180937F2C5A
:10E040008091772790917827009719F0226120938B
:10E050007F2C0E94946481E090E0998B888B88E00B
:10E06000898F1B8E81E18093A0270FC185FF1CC083
:10E070005091A52740E08091A62790E0842B952B16
:10E080004091822C5091832C480F591F5093832C20
:10E090004093822C4091772750917827481B590B49
:10E0A000509378274093772780917727909178270E
:10E0B000009749F024FD07C020917F2C2260209317
:10E0C0007F2C0E94D0689091A12780E02091A22708
:10E0D000820F911D90938117809380172C893D8921
:10E0E0002817390710F0009721F4309381172093F7
:10E0F000801780918017909181179B8B8A8B8091DC
:10E100007F2C90E083709070009709F456C11092B4
:10E110001B2D10921A2D0E94946480917F2C85FFF4
:10E1200007C010921B2D10921A2D198E84E19BCFDF
:10E1300084FF0AC010921B2D10921A2D81E090E0EE
:10E14000998B888B84E08CCF20911A2D30911B2DD8
:10E1500021153105E1F080FF02C0198A188A8889EB
:10E160009989009781F48A899B898217930720F403
:10E1700090931B2D80931A2D80911A2D90911B2D19
:10E18000998B888B04C090931B2D80931A2D1B8E26
:10E190008091792790917A279093832C8093822C79
:10E1A00080911A2D90911B2D009759F0888999899B
:10E1B000009739F08896909378278093772788E1A5
:10E1C0000BC080917F2C81FFF8C088E290E0909393
:10E1D00078278093772780E18093A0275CC0809187
:10E1E0007F2C80FFEAC0198E80E180937F2C0E94F3
:10E1F0009464E3C08091772790917827009711F07D
:10E200000E94D0689091A02780917F2C90FF0BC036
:10E2100080FF06C087E0898F1A8E198A188A19C074
:10E2200086E0898F16C080FF1EC085E0898F198A1D
:10E23000188AC3C08091772790917827009711F0B2
:10E240000E94D0688091A02780FF0DC087E0898F51
:10E250001A8E81E090E00E94D06880E180937F2C4C
:10E260000E9494640FC0809177279091782700973F
:10E2700049F4A3C080917F2C80FF9FC087E0898FE5
:10E280001A8E9BC080E1F80181A388E290E0909310
:10E2900078278093772780E580939F2788858093D0
:10E2A0009B27898580939C278A8580939D278B85D2
:10E2B00080939E278C85809397278D8580939827C0
:10E2C0008E85809399278F8580939A2786E0809307
:10E2D00088278C819D8190939427809393278E81AA
:10E2E0009F8190939627809395278091162D9091EA
:10E2F000172DA091182DB091192D80938B279093F5
:10E300008C27A0938D27B0938E2788819981AA812D
:10E31000BB8180938F2790939027A0939127B093F0
:10E320009227898D84FF05C01092A2271092A12701
:10E3300006C084E08093A12788ED8093A22780E423
:10E3400080938727809177279091782790938127D2
:10E35000809382271092A6271092A5271092A427B7
:10E360001092A3270E940569809590959093A42709
:10E370008093A32785E480937F27109280271092B3
:10E380008627109285278091841790918517019692
:10E390009093851780938417909383278093842785
:10E3A00010928A27109289270E94F4688095909590
:10E3B00090938A278093892704C01092782710921F
:10E3C000772710927F2CDF91CF911F910F91FF90B3
:10E3D000EF900895382F292FC9010895382F292F3C
:10E3E00040E050E076276727762780E090E0CB0179
:10E3F00077276627262B372B482B592BB901CA01C3
:10E400000895AC01E0917927F0917A2722273327EC
:10E410002E1B3F0B2158334D621773070CF49B01E1
:10E420001216130664F420931A2D30931B2D4E17E9
:10E430005F0729F0CF01BA01A9010E946B7D089501
:10E440000F93DF93CF93CDB7DEB760970FB6F894F5
:10E45000DEBF0FBECDBF002309F459C029833A8324
:10E460004B835C836D837E838F839887E0E2E01B20
:10E4700029813A814B815C811E16BCF019861A866F
:10E480001B861C868E2F992787FD909590958195E8
:10E490009F4F04C0220F331F441F551F8A95D2F788
:10E4A0002D873E874F87588B2AC0CA01B901002E9D
:10E4B00004C0660F771F881F991F0A94D2F76987D7
:10E4C0007A878B879C87DA01C90104C0B695A79526
:10E4D00097958795EA95D2F72D813E814F81588592
:10E4E00004C0220F331F441F551F0A95D2F7822BF9
:10E4F000932BA42BB52B8D879E87AF87B88B29854F
:10E500003A854B855C856D857E858F85988960967B
:10E510000FB6F894DEBF0FBECDBFCF91DF910F9144
:10E520000895A0E1B0E0E7E9F2E70C94BE7A298310
:10E530003A834B835C836D837E838F839887A98620
:10E54000BA86CB86DC86ED86FE860F87188B2D81FA
:10E550003E814F8158858D859E85AF85B889281766
:10E5600039074A075B07C8F082179307A407B50766
:10E5700090F029813A814B815C8189859A85AB85B0
:10E58000BC85281739074A075B0738F082179307BD
:10E59000A407B50720F482E003C080E001C081E059
:10E5A0006096EAE00C94DA7A2F923F924F925F9253
:10E5B0006F927F928F929F92AF92BF92CF92DF9293
:10E5C000EF92FF920F931F93DF93CF93CDB7DEB7F8
:10E5D00063970FB6F894DEBF0FBECDBF6C017F8787
:10E5E0006E87FC0117821682838181FD04C06FC390
:10E5F0004C855D8504C01E010894211C311CF60168
:10E600009381EE85FF8593FD859193FF8191FF872F
:10E61000EE87882309F457C3853241F493FD859131
:10E6200093FF8191FF87EE87853259F490E0B60120
:10E630004A8B5B8B0E94BE7D4A895B895D874C87D4
:10E64000D7CF10E0FF2400E00032B0F48B3269F045
:10E650008C3228F4803251F0833271F40BC08D3249
:10E6600039F0803349F401602CC00260046029C095
:10E67000086027C0006125C007FD2EC0282F205349
:10E680002A3098F406FF08C0812F880F182F110F29
:10E69000110F180F120F15C08F2D880FF82EFF0CB9
:10E6A000FF0CF80EF20E00620CC08E3221F406FD53
:10E6B0000AC3006406C08C3611F4006802C08836B4
:10E6C00059F4EE85FF8593FD859193FF8191FF8736
:10E6D000EE87882309F0B8CF982F9554933018F41B
:10E6E0000061805E06C0982F9556933008F09BC15C
:10E6F0000F7E06FF16E06FE3E62EE022853619F462
:10E70000F0E4EF2A07C0863619F420E8E22A02C0B6
:10E7100011111150E7FE06C01C3340F4912E939462
:10E7200027E00BC0183030F4212F06C027E03CE36F
:10E73000932E03C027E017E09924CA0104969D8711
:10E740008C87FA016081718182819381A101092DF9
:10E750000E947B7C5C016980262D30E0398B288B00
:10E7600060FE03C0388933FF06C0E1FC06C0E2FE4C
:10E7700006C000E205C00DE203C00BE201C000E0EC
:10E78000888999898C7090700097C1F1002311F0ED
:10E7900084E001C083E08F1558F4F81AE3FC09C047
:10E7A00080E290E0B6010E94BE7DFA94C9F701C0F4
:10E7B000FF24002329F0802F90E0B6010E94BE7D47
:10E7C000888983FD03C001E010E10EC00DEF1FE05A
:10E7D0000BC0A114B10409F0805290E0B6010E9470
:10E7E000BE7D0F5F1F4F05C0AE2CBB2490E1A92258
:10E7F000BB24F8018491882361F762C2E7FE0EC052
:10E800009A0CF889F4FF04C08A81813309F49A9440
:10E81000191454F5292D293050F52DC0E6FC2BC0D4
:10E82000812F90E08A159B054CF03CEFA3163FEF3B
:10E83000B30624F080E8E82A01C01150112349F002
:10E84000E2E0F0E0EC0FFD1FE10FF11D808180336D
:10E85000A1F3E7FE10C0912E9394812F90E0A816AB
:10E86000B90644F41A1907C09924939404C098E097
:10E87000992E01C010E0E7FE07C01A141B043CF4F7
:10E8800095012F5F3F4F05C025E030E002C021E039
:10E8900030E0002311F02F5F3F4F112329F0812F2B
:10E8A00090E00196280F391F8F2D90E02817390727
:10E8B00014F4F21A01C0FF244E2C5524C2018970B1
:10E8C0009070009749F406C080E290E0B6010E9483
:10E8D000BE7DFA94FF20C1F7002329F0802F90E03D
:10E8E000B6010E94BE7D43FC09C006C080E390E0F3
:10E8F000B6010E94BE7DFA94FF20C1F7E7FE46C034
:10E900003501B7FE02C06624772425010894411C16
:10E91000511C46185708420C531CF501E919F1091E
:10E920004F01812F90E000271127081B190BFFEFE3
:10E930006F16FFEF7F0629F48EE290E0B6010E9489
:10E94000BE7DA614B70434F0861497041CF4F201BB
:10E95000808101C080E30894610871080894411C1B
:10E96000511C601671062CF090E0B6010E94BE7D2D
:10E97000DECF6A147B0441F49A81963320F49533F8
:10E9800019F4F889F4FF81E390E049C08A8181336A
:10E9900011F02FEE622290E0B6010E94BE7D11239D
:10E9A00089F08EE290E0B6010E94BE7D02E0F101A6
:10E9B000E00FF11D0F5F808190E0B6010E94BE7DE7
:10E9C0001150A9F744FE03C085E490E002C085E63B
:10E9D00090E0B6010E94BE7DB7FC05C0A114B10451
:10E9E00041F464FE06C0B094A194B108B3948DE2E2
:10E9F00001C08BE290E0B6010E94BE7D80E305C0BD
:10EA00008F5FE6EFFFEFAE0EBF1EFAE0AF16B10468
:10EA1000BCF790E0B6010E94BE7DC501C096B6016C
:10EA20000E94BE7D4DC1833631F0833789F0833536
:10EA300009F059C022C09A012E5F3F4F3D872C87B5
:10EA4000FA0180818983310181E0A82EB12C13C0A5
:10EA50009A012E5F3F4F3D872C87FA0160807180BD
:10EA600006FF03C0612F70E002C06FEF7FEFC301AC
:10EA70000E94847D5C010F7714C09A012E5F3F4F86
:10EA80003D872C87FA016080718006FF03C0612FEB
:10EA900070E002C06FEF7FEFC3010E945B7D5C01FD
:10EAA000006803FD1CC006C080E290E0B6010E9431
:10EAB000BE7DFA948F2D90E0A816B906A8F30FC07A
:10EAC000F30107FD859107FF81913F0190E0B601B9
:10EAD0000E94BE7DF110FA940894A108B108A11417
:10EAE000B10471F7EDC0843611F0893661F507FF86
:10EAF0000BC09A012C5F3F4F3D872C87FA01608144
:10EB00007181828193810CC09A012E5F3F4F3D87B6
:10EB10002C87FA0160817181882777FD8095982F75
:10EB20000F7697FF08C090958095709561957F4FFF
:10EB30008F4F9F4F0068A1012AE030E00E94D07EF5
:10EB4000982E921841C0853721F40F7E2AE030E0DC
:10EB500020C0097F8F36A9F0803720F4883509F06E
:10EB6000B2C00BC0803721F0883709F0ACC001C0BB
:10EB7000006104FF09C0046007C004FF08C006600C
:10EB800006C028E030E005C020E130E002C020E10E
:10EB900032E007FF0AC0CA0104969D878C87FA01FC
:10EBA000608171818281938109C0CA0102969D872B
:10EBB0008C87FA016081718180E090E0A1010E9460
:10EBC000D07E982E92180F7706FF09C00E7F9116FF
:10EBD00030F404FF06C002FD04C00F7E02C0E92C21
:10EBE00001C0E12E802F90E004FF0CC0FE01E90D72
:10EBF000F11D2081203311F4097E09C0E39402FF46
:10EC000006C004C086789070009709F0E394A02EA7
:10EC1000BB2403FD14C000FF0FC0EF1428F4192D0E
:10EC20001F0D1E19EF2C08C0192D06C080E290E0C0
:10EC3000B6010E94BE7DE394EF14C0F304C0EF144C
:10EC400010F4FE1801C0FF24A4FE0FC080E390E082
:10EC5000B6010E94BE7DA2FE1FC0A1FE03C088E5D2
:10EC600090E010C088E790E00DC0C50186789070F4
:10EC7000009791F0A1FC02C080E201C08BE207FD89
:10EC80008DE290E0B6010E94BE7D06C080E390E078
:10EC9000B6010E94BE7D11509116C0F39A94F10105
:10ECA000E90DF11D808190E0B6010E94BE7D9920A2
:10ECB000A9F706C080E290E0B6010E94BE7DFA94FA
:10ECC000FF20C1F795CCF6012681378102C02FEFD6
:10ECD0003FEFC90163960FB6F894DEBF0FBECDBFFC
:10ECE000CF91DF911F910F91FF90EF90DF90CF9028
:10ECF000BF90AF909F908F907F906F905F904F905C
:10ED00003F902F9008955058BB27AA270ED0CBC113
:10ED1000BCD130F0C1D120F031F49F3F11F41EF48A
:10ED20008CC10EF4E095E7FB82C1E92FCDD180F3D1
:10ED3000BA17620773078407950718F071F49EF5F8
:10ED4000E5C10EF4E0950B2EBA2FA02D0B01B901F1
:10ED500090010C01CA01A0011124FF27591B99F051
:10ED6000593F50F4503E68F11A16F040A22F232F5D
:10ED7000342F4427585FF3CF469537952795A795AD
:10ED8000F0405395C9F77EF41F16BA0B620B730B54
:10ED9000840BBAF09150A1F0FF0FBB1F661F771FC5
:10EDA000881FC2F70EC0BA0F621F731F841F48F47A
:10EDB000879577956795B795F7959E3F08F0B3CF00
:10EDC0009395880F08F09927EE0F979587950895EA
:10EDD0005CD158F080E891E009F49EEF5DD128F015
:10EDE00040E851E059F45EEF09C027C18FC1E92F17
:10EDF000E0786AD168F3092E052AC1F32617370790
:10EE00004807590738F00E2E07F8E02569F0E0258D
:10EE1000E0640AC0EF6307F8009407FADB01B90168
:10EE20009D01DC01CA01AD01EF9347D03CD10AD06E
:10EE30005F91552331F02BED3FE049E450FD49EC63
:10EE400063CF0895DF93DD27B92FBF7740E85FE3F5
:10EE50001616170648075B0710F4D92F5ED19F934B
:10EE60008F937F936F930FD2E0E2F1E0E9D01BD153
:10EE70002F913F914F915F9163D1DD2349F09058DD
:10EE8000A2EA2AED3FE049EC5FE3D0785D274DDF51
:10EE9000DF9109C1A8D008F481E008950CD003C126
:10EEA000FBD040F0F2D030F021F45F3F19F0BFC04A
:10EEB00051112DC1C2C008D198F39923C9F355232C
:10EEC000B1F3951B550BBB27AA276217730784075D
:10EED00038F09F5F5F4F220F331F441FAA1FA9F313
:10EEE00033D00E2E3AF0E0E830D091505040E69505
:10EEF000001CCAF729D0FE2F27D0660F771F881F66
:10EF0000BB1F261737074807AB07B0E809F0BB0B54
:10EF1000802DBF01FF2793585F4F2AF09E3F510578
:10EF200068F085C0F4C05F3FECF3983EDCF3869553
:10EF300077956795B795F7959F5FC9F7880F911DEE
:10EF40009695879597F90895E1E0660F771F881FDA
:10EF5000BB1F621773078407BA0720F0621B730B8D
:10EF6000840BBA0BEE1F88F7E0950895E89409C06A
:10EF700097FB3EF490958095709561957F4F8F4FEC
:10EF80009F4F9923A9F0F92F96E9BB279395F69502
:10EF9000879577956795B795F111F8CFFAF4BB0F80
:10EFA00011F460FF1BC06F5F7F4F8F4F9F4F16C0E4
:10EFB000882311F096E911C0772321F09EE8872F6E
:10EFC000762F05C0662371F096E8862F70E060E02A
:10EFD0002AF09A95660F771F881FDAF7880F9695A3
:10EFE000879597F90895990F0008550FAA0BE0E847
:10EFF000FEEF16161706E807F907C0F012161306FB
:10F00000E407F50798F0621B730B840B950B39F43A
:10F010000A2661F0232B242B252B21F408950A26A0
:10F0200009F4A140A6958FEF811D811D089597F9E0
:10F030009F6780E870E060E008959FEF80EC08959E
:10F04000DF93CF931F930F93FF92EF92DF927B0199
:10F050008C01689405C0DA2EEF0172D0FE01E894AD
:10F06000A5912591359145915591AEF3EF015DDE66
:10F07000FE019701A801DA9479F7DF90EF90FF90F5
:10F080000F911F91CF91DF91089500240A941616D5
:10F09000170618060906089500240A941216130686
:10F0A000140605060895092E0394000C11F4882314
:10F0B00052F0BB0F40F4BF2B11F460FF04C06F5F30
:10F0C0007F4F8F4F9F4F089557FD9058440F551F06
:10F0D00059F05F3F71F04795880F97FB991F61F0DA
:10F0E0009F3F79F087950895121613061406551F51
:10F0F000F2CF4695F1DF08C0161617061806991FBD
:10F10000F1CF86957105610508940895E894BB27B1
:10F1100066277727CB0197F908959B01AC0160E042
:10F1200070E080E89FE3BACE0BD0BDCFAEDF28F011
:10F13000B3DF18F0952309F07ACF7FCF1124E7CF02
:10F14000C3DFA0F3959FD1F3950F50E0551F629F49
:10F15000F001729FBB27F00DB11D639FAA27F00D30
:10F16000B11DAA1F649F6627B00DA11D661F829F57
:10F170002227B00DA11D621F739FB00DA11D621F3C
:10F18000839FA00D611D221F749F3327A00D611D59
:10F19000231F849F600D211D822F762F6A2F11243B
:10F1A0009F5750408AF0E1F088234AF0EE0FFF1F8E
:10F1B000BB1F661F771F881F91505040A9F79E3FC5
:10F1C000510570F034CFA3CF5F3FECF3983EDCF3F2
:10F1D000869577956795B795F795E7959F5FC1F702
:10F1E000FE2B880F911D9695879597F90895FA0142
:10F1F000EE0FFF1F30962105310599F1611571055C
:10F2000061F48038BFE39B0749F168949038810529
:10F2100061F08038BFEF9B0741F0992342F5FF3F33
:10F22000E1053105210511F1E8940894E795D9012C
:10F23000AA2329F4AB2FBE2FF85FD0F310C0FF5FD5
:10F2400070F4A695E0F7F73950F019F0FF3A38F46A
:10F250009F779F930CD00F9007FC905808953EF035
:10F26000ECCE60E070E080E89FE308954FE79F7781
:10F270005F934F933F932F9375D02F913F914F9171
:10F280005F9152DF08C09B01AC014ECF19F40EF024
:10F29000CECE3CCFD2CE20DFC8F39638C0F707F8E9
:10F2A0000F92E8942BE33AEA48EB5FE74BDF0F92CB
:10F2B0000F920F924DB75EB70F9294D0EDE4F1E04C
:10F2C000BFDE4F915F91EF91FF91E595EE1FFF1F1C
:10F2D00049F0FE57E0684427EE0F441FFA95E1F726
:10F2E0004195550B06D00F9007FE17CF08959FCE7E
:10F2F000ACC0F2DEE8F39923D9F3940F511DBBF3B0
:10F300009150504094F059F0882332F0660F771FE7
:10F31000881F91505040C1F79E3F510544F7880F18
:10F32000911D9695879597F908955F3FACF0983EAB
:10F330009CF0BB27869577956795B79508F4B160E3
:10F340009395C1F7BB0F58F711F460FFE8CF6F5FDB
:10F350007F4F8F4F9F4FE3CFDACE0EF076C06DCE4A
:10F36000689465CEB9DEC8F39923D1F3C6F3DF9371
:10F37000CF931F930F93FF92C92FDD2788232AF085
:10F380002197660F771F881FDAF720E030E040E80A
:10F390005FEB9FE3883920F0803E30F021968F7735
:10F3A000B3DCE5E7F1E003C0AFDCE2EAF1E048DE20
:10F3B0008B01BE01EC01FB2E6F5771097595771F0C
:10F3C000880B990BD5DD28E132E741E35FE3B8DE36
:10F3D000AF2D9801AE01FF900F911F91CF91DF915A
:10F3E000A4DC61CEFA01DC01AA0FBB1F9B01AC01BA
:10F3F000BF5728F422273327442750781FC0B7511E
:10F4000088F4AB2F0024469537952795011CA395CA
:10F41000D2F3002069F0220F331F441FB395DAF3B3
:10F420000DD071CC61307105A0E88A07B94630F47F
:10F430009B01AC016627772788279078309621F0CA
:10F44000208331834283538308959F3F31F091504D
:10F4500020F4879577956795B795880F911D9695B8
:10F46000879597F90895629FD001739FF001829F5D
:10F47000E00DF11D649FE00DF11D929FF00D839F43
:10F48000F00D749FF00D659FF00D9927729FB00DE0
:10F49000E11DF91F639FB00DE11DF91FBD01CF01F3
:10F4A00011240895AA1BBB1B51E107C0AA1FBB1F53
:10F4B000A617B70710F0A61BB70B881F991F5A9500
:10F4C000A9F780959095BC01CD01089597FB092E71
:10F4D00007260AD077FD04D0E5DF06D000201AF415
:10F4E000709561957F4F0895F6F7909581959F4FA0
:10F4F0000895A1E21A2EAA1BBB1BFD010DC0AA1F75
:10F50000BB1FEE1FFF1FA217B307E407F50720F08C
:10F51000A21BB30BE40BF50B661F771F881F991F07
:10F520001A9469F760957095809590959B01AC0150
:10F53000BD01CF01089597FB092E05260ED057FD7A
:10F5400004D0D7DF0AD0001C38F450954095309590
:10F5500021953F4F4F4F5F4F0895F6F79095809557
:10F56000709561957F4F8F4F9F4F08952F923F92D7
:10F570004F925F926F927F928F929F92AF92BF92C3
:10F58000CF92DF92EF92FF920F931F93CF93DF936F
:10F59000CDB7DEB7CA1BDB0B0FB6F894DEBF0FBECC
:10F5A000CDBF09942A88398848885F846E847D8419
:10F5B0008C849B84AA84B984C884DF80EE80FD801B
:10F5C0000C811B81AA81B981CE0FD11D0FB6F89491
:10F5D000DEBF0FBECDBFED010895AF92BF92CF92B7
:10F5E000DF92EF92FF920F931F93CF93DF93EC0183
:10F5F000688179818A819B816115710581059105F9
:10F6000021F464E279ED8BE597E02DE133EF41E001
:10F6100050E00E949B7A79018A0127EA31E440E0B8
:10F6200050E00E94337A5B016C01C801B7012CEEF7
:10F6300034EF4FEF5FEF0E94337A6A0D7B1D8C1D14
:10F640009D1D97FF04C061507040804090486883C2
:10F6500079838A839B837F77CB01DF91CF911F9141
:10F660000F91FF90EF90DF90CF90BF90AF900895F3
:10F670000E94ED7A089587ED96E00E94ED7A089554
:10F68000A0E0B0E08093D7069093D806A093D90667
:10F69000B093DA0608952F923F924F925F926F9245
:10F6A0007F929F92AF92BF92CF92DF92EF92FF92A2
:10F6B0000F931F93CF93DF933B01EA01611571050F
:10F6C00019F0FB0180839183209739F09E0122502D
:10F6D00030402332310508F0D5C0C82ED92EF601AE
:10F6E00011916F017F01812F90E00E94537D00975F
:10F6F000B1F71D3231F4F60111917F0199249394F1
:10F7000006C01B3219F4F60111917F01992420974C
:10F7100019F0C031D105D1F4103389F4F70180819B
:10F72000883711F0883559F4F701118182E090E0B3
:10F73000E80EF91E92E0992AC0E1D0E007C02097B8
:10F7400029F41033B1F0CAE0D0E02BC0CA30D105A3
:10F7500041F1C031D10521F0C830D105A9F409C06B
:10F760002FEFA22E2FEFB22E2FEFC22E2FE0D22E90
:10F7700020C0C8E0D0E09FEFA92E9FEFB92E9FEFE9
:10F78000C92E9FE1D92E15C09E01442737FD409513
:10F79000542F6FEF7FEFCB010E94797A59016A01F4
:10F7A00008C089E9A82E89E9B82E89E9C82E89E11F
:10F7B000D82E60E020E030E0A9011E01442437FC8F
:10F7C0004094542C012F00530A3060F0812F815453
:10F7D0008A3110F4075006C0812F81568A3150F5C6
:10F7E000012F0755802F90E08C179D071CF56F3F68
:10F7F000E9F0A216B306C406D506A8F0CA01B901FD
:10F80000A20191010E94337A9B01AC01802F90E00C
:10F81000A0E0B0E0280F391F4A1F5B1F28173907E7
:10F820004A075B0710F46FEF01C061E0F701119127
:10F830007F01C8CF6114710481F0662339F0089408
:10F84000E108F108F301F182E08207C091FE05C0F2
:10F85000C7010297F3019183808390FE07C0509502
:10F860004095309521953F4F4F4F5F4F67FF0DC03B
:10F8700082E290E09093A52D8093A42D2FEF3FEF8F
:10F88000A90103C020E030E0A901B901CA01DF915C
:10F89000CF911F910F91FF90EF90DF90CF90BF908D
:10F8A000AF909F907F906F905F904F903F902F9080
:10F8B0000895662777270C94697FFC01882799278C
:10F8C000E89421912032E9F3293010F02E30C8F36A
:10F8D0002B3241F02D3239F4689404C00E94B67D79
:10F8E000820F911D219120532A30C0F31EF4909570
:10F8F00081959F4F0895283008F027E03327DA01DB
:10F90000990F311D87FD916000966105710539F4ED
:10F9100032602E5F3D9330E32A95E1F708959F3FD3
:10F9200030F080387105610509F03C5F3C5F3D9324
:10F93000913008F08068911DDF93CF931F930F9350
:10F94000FF92EF92192F987F9695E92F96959695AD
:10F95000E90FFF27E15AFF4E99273327EE24FF24B2
:10F96000A701E70105900894079428F4360FE71ED5
:10F97000F81E491F511D660F771F881F991F069497
:10F98000A1F70590079428F4E70EF81E491F561FAB
:10F99000C11D770F881F991F661F0694A1F7059058
:10F9A000079428F4F80E491F561FC71FD11D880F52
:10F9B000991F661F771F0694A1F70590079420F4FE
:10F9C000490F561FC71FD81F990F661F771F881F23
:10F9D0000694A9F784911095177041F0D695C795B4
:10F9E00057954795F794E7941A95C1F7E5E0F0E14C
:10F9F00068941590159135916591959105907FE2E8
:10FA00007395E118F10A430B560BC90BD009C0F7E7
:10FA1000E10CF11E431F561FC91FD01D7EF4703329
:10FA200011F48A95E6CFE894015030F0080F0AF4FB
:10FA30000027021708F4202F2395022F7A3328F08D
:10FA400079E37D932A95E9F710C07D932A9589F68D
:10FA5000069497956795379517951794E118F10ACD
:10FA6000430B560BC90BD00998F023957E917395E3
:10FA70007A3308F070E37C932013B8F77E917061BD
:10FA80007D9330F0839571E37D9370E32A95E1F7E0
:10FA90001124EF90FF900F911F91CF91DF91992743
:10FAA00087FD909508959111A2C3803219F0895075
:10FAB0008550D0F70895FC01059061507040011009
:10FAC000D8F7809590958E0F9F1F089548E857E1CD
:10FAD0000E948F7D0895FB01DC0102C001900D9210
:10FAE00041505040D8F70895DC0101C06D9341505A
:10FAF0005040E0F70895FB01DC018D9101908019E1
:10FB00000110D9F3990B0895FC01615070400190E8
:10FB10000110D8F7809590958E0F9F1F0895FA01D8
:10FB2000A191B081009719F41097E1F0CD01DC01AB
:10FB3000CD010D90002011F4C00113C0FB012191F3
:10FB4000222319F02015D9F7F3CFFB0121912015BD
:10FB500019F41E92119606C02223C1F70D900020C1
:10FB6000A1F7D001FA01A193B08308957AE0979F9D
:10FB7000902D879F802D910D112408950F931F9331
:10FB8000CF93DF938C01EB018B8181FF1BC082FF40
:10FB90000DC02E813F818C819D812817390764F427
:10FBA000E881F9810193F983E88306C0E885F98546
:10FBB000802F0995009731F48E819F8101969F8354
:10FBC0008E8302C00FEF1FEFC801DF91CF911F910D
:10FBD0000F910895DF93CF93CDB7DEB7FE01359631
:10FBE000619171918091A02D9091A12DAF010E9402
:10FBF000D472CF91DF910895DF93CF93CDB7DEB765
:10FC0000FE013596619171918091A02D9091A12D69
:10FC1000DC0113962C911397286013962C93AF0157
:10FC20000E94D472E091A02DF091A12D2381277F15
:10FC30002383CF91DF9108956091A02D7091A12D24
:10FC40000E94BE7D0895EF92FF920F931F93CF9372
:10FC5000DF938C01E091A02DF091A12D838181FF94
:10FC60001FC0C0E0D0E00AC0DB011896ED91FC9106
:10FC700019970995009711F0CFEFDFEFF801819107
:10FC80008F016091A02D7091A12D882369F7DB0170
:10FC90001896ED91FC9119978AE00995009711F05B
:10FCA000CFEFDFEFCE01DF91CF911F910F91FF904A
:10FCB000EF9008950F931F93DF93CF93CDB7DEB7E7
:10FCC0002E970FB6F894DEBF0FBECDBF0D891E89EB
:10FCD0008F89988D26E02C831A83098397FF02C0B1
:10FCE00080E090E801979E838D839E01255E3F4FC3
:10FCF000CE010196698D7A8DA9010E94D4724D8141
:10FD00005E8157FD0AC02F813885421753070CF4D6
:10FD10009A01020F131FF80110822E960FB6F89465
:10FD2000DEBF0FBECDBFCF91DF911F910F91089520
:10FD30000F931F93DF93CF93CDB7DEB72E970FB6F8
:10FD4000F894DEBF0FBECDBF8C01CB01BA0146E0F7
:10FD50004C831A83098397FF02C080E090E80197E3
:10FD60009E838D83CE010196A9010E94D4724D819C
:10FD70005E8157FD0AC02F813885421753070CF466
:10FD80009A01020F131FF80110822E960FB6F894F5
:10FD9000DEBF0FBECDBFCF91DF911F910F910895B0
:10FDA000FA01AA27283051F1203181F1E8946F93AC
:10FDB0006E7F6E5F7F4F8F4F9F4FAF4FB1E03ED052
:10FDC000B4E03CD0670F781F891F9A1FA11D680FF0
:10FDD000791F8A1F911DA11D6A0F711D811D911D23
:10FDE000A11D20D009F468943F912AE0269F112498
:10FDF0003019305D3193DEF6CF010895462F4770FC
:10FE0000405D4193B3E00FD0C9F7F6CF462F4F7056
:10FE1000405D4A3318F0495D31FD4052419302D0B4
:10FE2000A9F7EACFB4E0A69597958795779567955A
:10FE3000BA95C9F700976105710508959B01AC015A
:10FE40000A2E06945795479537952795BA95C9F781
:10FE5000620F731F841F951FA01D0895DC01CB0145
:10FE6000FC01F999FECF06C0F2BDE1BDF89A3196CA
:10FE700000B40D9241505040B8F70895F999FECF63
:10FE800092BD81BDF89A992780B50895A8E1B0E0A8
:10FE900042E050E00C94307FDC01CB0103C02D9197
:10FEA0000E94577F41505040D0F70895262FF9996E
:10FEB000FECF1FBA92BD81BD20BD0FB6F894FA9A4D
:10FEC000F99A0FBE019608950E94567F272F0C9431
:10FED000577F6F927F928F929F92AF92BF92CF92F5
:10FEE000DF92EF92FF920F931F93DF93CF930F92C6
:10FEF000CDB7DEB75B016115710521F0DB018C9395
:10FF000011969C93482F592F6A01F601E1906F01D9
:10FF10008F018E2D90E00E94537D0097B1F7FE2D4A
:10FF2000FD3229F4D601ED908D0121E007C0BE2DF0
:10FF3000BB3219F4F601E1908F0120E068010894CA
:10FF4000C108D108C6016FEF70E143E050E029839A
:10FF50000E94FA802981009711F572E0E72EF12CBA
:10FF6000E00EF11EC70162E071E145E050E00E9441
:10FF7000FA802981009729F467E0E62EF12CE00E43
:10FF8000F11EA114B10421F0D5011196FC92EE925C
:10FF900020FF0FC130E020E090E88FEF12C1C601D2
:10FFA00067E071E143E050E029830E94FA802981F3
:10FFB000009731F060E070E0CB01662477240AC03E
:10FFC000A114B10409F4F9C00E5F1F4FF5011183AC
:10FFD0000083F3C03E2D30533A30A0F52260E22F6B
:10FFE000F0E0AF014870507022FF07C04115510585
:10FFF00071F50894611C711C2AC04115510519F056
:020000021000EC
:100000000894610871086B017C0152E0CC0CDD1C86
:10001000EE1CFF1C5A95D1F76C0D7D1D8E1D9F1D8A
:10002000660F771F881F991F630F711D811D911D1A
:100030006839F9E97F07F9E98F07F9E19F0738F097
:10004000246005C03E3F39F423FD3FC02860D8013D
:10005000ED908D01BFCF353311F03531B1F5F80199
:1000600031913D3211F4206102C03B3241F4D8019C
:1000700011963C911197319642E050E002C041E068
:1000800050E030533A3020F08F01041B150B1DC097
:1000900040E050E0BCE040385B075CF4DA01AA0FB6
:1000A000BB1FAA0FBB1F4A0F5B1F440F551F430FF7
:1000B000511D319130538F013A3060F324FF03C05A
:1000C000509541955F4F640E751EC22EDD2421FFB1
:1000D00008C0A114B10429F001501040F5011183AA
:1000E00000830E94B6777B018C01F3E0CF22DD24F0
:1000F00033E0C316D10421F417FB109517F91095BE
:10010000C801B70120E030E0A9010E944A778823A6
:1001100009F44AC077FE09C04EE1C42E41E1D42E55
:10012000709461947108739404C036E3C32E31E176
:10013000D32E26E0822E912C90E2A92EB12C0FC056
:10014000F6012591359145915491C801B7010E945E
:100150009478E62EF72E082F192F6A187B086A1458
:100160007B0474F7B594A7940894810891088114CE
:10017000910429F08CEF9FEFC80ED91EF0CFB70184
:10018000C801282F220F292F221F2F3F39F020E0EE
:1001900030E0A9010E944A77882331F482E290E09E
:1001A0009093A52D8093A42D3E2D2F2D902F812F40
:1001B00008C030E020E090E803C030E020E090ECA0
:1001C0008FE7F901AC016F2F722F852F942F0F90BD
:1001D000CF91DF911F910F91FF90EF90DF90CF9023
:1001E000BF90AF909F908F907F906F9008959927C8
:1001F00088270895FB01DC014150504088F08D9123
:1002000081341CF08B350CF4805E659161341CF0F8
:100210006B350CF4605E861B611171F3990B0895C8
:08022000881BFCCFF894FFCF0E
:10022800263A202573205B414444523D252D642EF7
:10023800252D64205345513D252D642052535349A3
:100248003D252D75204C51493D252D752044525092
:100258003D252D642E253032645D0A00523D252D42
:1002680075204C3D252D7520533D252D64200054C7
:10027800696D656F757420414444523D252D642E87
:10028800252D64205345513D252D64205253534953
:100298003D252D75204C51493D252D750A002845D1
:1002A800787450777229000065756936343D0025E9
:1002B80030327800253032780A00736E3D00413ABA
:1002C800202564202564202564200A00433A20253F
:1002D8006420256420256420613D25352E31660A79
:1002E800007374617475733D3078253032780A2054
:1002F80000312E30204669726D776172652056652F
:10030800722E2053322D342E3120323031332D309D
:10031800382D303900656570726F6D006F6E006F33
:100328006666004F6E006131007265736574006E19
:100338006F6E6500613200765F696E0031003200D1
:100348003300340035003600636820706B74730026
:1003580025327520252D3130750A006175746F00BE
:10036800666C75736800414444523D252D642E2502
:100378002D64205345513D252D6420525353493D4A
:10038800252D75204C51493D252D750A006465655C
:100398007000666F7263655F69646C65007472698A
:1003A8006D00746573740043683D252D642054788E
:1003B8005077723D252D640A004572726F72205481
:1003C80058204C656E6774683D25640A0049443DB1
:1003D800004536343D002050533D25640020543DEF
:1003E800252D362E3266002054313D252D362E32ED
:1003F800660020545F4D43553D252D352E3166004E
:1004080020565F4D43553D252D342E326600205031
:10041800303D252D6C58002050305F543D252D3738
:100428002E3366002050313D252D6C580020503168
:100438005F543D252D372E3366002055503D252D20
:100448006C58002052483D252D342E316600205628
:100458005F494E3D252D352E32660020565F4131CD
:100468003D252D352E32660020565F41323D252D23
:10047800352E32660020565F41333D252D352E300E
:10048800660020503D252D6C64002050413D252DEF
:10049800372E326600263A2025730A0054582070F9
:1004A8006B74206C656E203D2025640A002530326F
:1004B80058006C656E3D25640A000100D734EF3C96
:1004C80022FFCC3B22FFCC3B1A20090D00A9046176
:1004D80062636465666768696A6B6C6D6E6F7026C7
:1004E8009400003C000A001A636D642070726F6308
:1004F800657373000000C80463350000000073745E
:1005080064696E2070726F63657373000000DE04A7
:100518008B0F0000000062726F6164636173742066
:1005280070726F63657373000000F6044336000051
:100538000000536C6565702070726F63657373009B
:10054800000012057D1000000000506572696F649C
:1005580069632070726F636573730000002A057900
:100568001700000000D404EC0408053B0520050032
:1005780000070900001D0040001207520710000084
:1005880000B73EAB3E1810000000004576656E745B
:100598002074696D65720000006B05C2420000009E
:1005A800004374696D65722070726F6365737300C0
:1005B80000008105004400000000020306070A0B42
:1005C8000E0F020306070A0B0E0F284329203230AC
:1005D8003132204865726A756C66005574766563B9
:1005E8006B6C696E6720202020202000436F6E749A
:1005F800696B6920322E35000000000200000000FF
:100608003B5200000000C600C500C400C100C20083
:10061800000000CE00CD00CC00C900CA00000000D8
:1006280052463233302064726976657200000000E9
:1006380006F256000000006355E15441578B5804F8
:100648005694540253FC528354E5530001010101AE
:1006580001010101010101010101010052696D65FA
:10066800003C06065ACD5961646174612E6E756D41
:1006780020776179206F75742074686572653A20F7
:1006880025640A00485B475B515D805EB85C00806A
:10069800C0E0F0F8FCFEFF6E756C6C6D616300776E
:1006A80006335F185F1E5F245F2A5F305F736963DC
:1006B800736C6F776D6163008D065460B55F4B5F37
:1006C800345F3A5F485FBA0008001111191135000C
:1006D8000200E916EB165443502F495020737461F9
:1006E800636B000000B606AE62000000000208FF5F
:0C06F800FFFFFF000000000100000000F8
:00000001FF
